:10100000808702209DE5000037CF010089E50000C0
:1010100089E5000089E5000089E500000000000086
:1010200000000000000000000000000049E7000090
:1010300089E5000000000000B5E6000089E5000039
:1010400005EA00005934010005EA000005EA000045
:1010500005EA000005EA000005EA000005EA0000D4
:1010600005EA0000D1600100E160010005EA00002E
:1010700005EA000005EA000005EA000005EA0000B4
:1010800005EA000005EA000005EA000005EA0000A4
:10109000BD34010005EA000005EA000005EA000091
:1010A00005EA000005EA000005EA000005EA000084
:1010B00005EA000005EA000005EA000005EA000074
:1010C00005EA000005EA000005EA000005EA000064
:1010D00005EA000005EA000005EA000005EA000054
:1010E00005EA000005EA000005EA000005EA000044
:1010F00005EA000005EA000005EA000005EA000034
:1011000001F0FF01102A2BDB10F0070F08D010F8B8
:10111000013B013A8B422DD010F0070F42B3F6D1BC
:10112000F0B441EA012141EA014122F007047FF0D5
:1011300000070023F0E80256083C85EA010586EA2C
:10114000010685FA47F5A3FA87F586FA47F6A5FA68
:1011500087F68EB9EED1F0BC01F0FF0102F0070274
:1011600032B110F8013B013A83EA010313B1F8D11F
:101170000020704701387047002D06BF3546033800
:10118000073815F0010F07D1013015F4807F02BF39
:10119000013015F4C03F0130F0BC0138704700BF8A
:1011A00018B1034B1860002070474FF0FF307047B4
:1011B00000050020014B1B689B68184700050020B4
:1011C000014B1B681B69184700050020014B1B6879
:1011D0005B69184700050020014B1B689B69184795
:1011E00000050020014B1B68DB6918470005002043
:1011F000014B1B681B6A184700050020014B1B6848
:101200009B6A18470005002010B4034C2468E4686A
:10121000A4465DF8044B604700050020014B1870A0
:10122000704700BFA8300020914208B503B20AD031
:10123000072804D940F2A331074800F0B9FA980012
:101240006030C0B208BD072802D940F29B31F3E7F5
:1012500098003030F5E700BFD7250200F8B50B7ACB
:101260000022C0E9002205460E46A3B31A4B0360D4
:101270008C7A04714F7A20463946FFF7D5FF012258
:10128000687139462046FFF7CFFFA871A000737937
:10129000327900F1804000F5C04003F01F0343EABB
:1012A0004213D0F8102522F4991222F4F852C0F813
:1012B0001025D0F8102587F001071B0242EA0752DB
:1012C00003F47C531343C0F81035D0F8103543F0C5
:1012D0000303C0F81035F8BD00600040024B1868E9
:1012E000003818BF01207047AC30002010B4034C08
:1012F0002468A4465DF8044B604700BFAC30002072
:10130000024B5B6803B11847704700BFAC30002048
:1013100000220F4938B50446134644FA02F0C007CC
:10132000D5B248BF581C02F1010244BFCD54C3B22C
:10133000042AF2D1064DC3F10402042BD2B24FF0BD
:10134000FF0188BF0022E81800F0BCFA2C7138BDFC
:10135000B430002038B5054D2B7983420C4601D1BD
:10136000285D38BDFFF7D4FFFAE700BFB430002096
:1013700090F83030FF2B10B515D00B4C01229A405D
:10138000C4F80825DA0002F1804202F5F83203F5CC
:1013900011730021C2F81015C2F8141544F8231077
:1013A000FF2380F8303010BD00F001402DE9F843F4
:1013B00099460546089B18B94321672000F002FAB8
:1013C000007DA8B36E7DFF2E01D14721F5E793F88C
:1013D0003000FF2820D183F830600A442F785379F9
:1013E0000A6834B202EB03086FB3012F4ED1E2005A
:1013F00002F1804202F5F8322549D2F81435E3B102
:1014000006F5117341F82380012303FA06F6C1F8AB
:1014100004650020BDE8F883864206D11C4806F525
:10142000117350F82330002BD7D06FF01500F1E77F
:101430000AB11E7FD1E75E7FCFE76B68C2F8103537
:10144000C2F81485E0E7287C08B97521B5E739466C
:10145000FFF780FFE200696802F1804200F150036B
:1014600002F5F83201EB8303C2F81035012303FAC9
:1014700006F6074BC2F81485C3F80465EB6800F55F
:10148000A870A3EB090341F82030C2E7892194E753
:1014900000F0014010B518B99621672000F092F9CC
:1014A000037DC3B1437D0F4C01229A40C4F8082547
:1014B000DA0002F1804202F5F83203F511730021DF
:1014C000C2F81015C2F8141544F823100378012B44
:1014D00006D9AC21E1E709B1137FE4E7537FE2E7E6
:1014E000084610BD00F00140017FCA0070B402F14F
:1014F0008042124C012505FA01F302F5F83201F59C
:101500001171C4F808350023C2F81035C2F814353B
:1015100044F82130417FCA0002F180428D4002F53B
:10152000F83201F51171C4F80855C2F81035C2F847
:10153000143544F8213070BCFFF71ABF00F00140A9
:10154000836B10B50446DBB190F84C300E4A02EBC9
:10155000C301012003F500734860002142F8231005
:1015600004F134002246FFF795FF20B14FF4CE710D
:10157000672000F027F9FF2384F84C30A06310BDEA
:101580004FF0FF30FBE700BF00F001400148FFF7DC
:10159000D7BF00BFBC300020014A01F001B900BF35
:1015A000BC3000200148FFF79FBF00BFBC300020C7
:1015B000014801F0D9B800BFBC300020014801F05B
:1015C000B7B800BFBC300020014A01F08FB800BF9F
:1015D000BC300020014A01F067B800BFBC300020D9
:1015E0001FB50446CDE902210193FFF777FE019B69
:1015F000039930B1029A204604B0BDE8104001F0D2
:1016000014B8044A92F90820204604B0BDE81040FE
:1016100000F0FBBFBC300020084B5A6910B522B166
:10162000C40742BF597E01245450DA6822B18107B1
:1016300042BF5B7C0121D15010BD00BFBC300020F7
:10164000034AD3680BB192F909300370704700BFA9
:10165000BC300020074B1A6A4AB95A6A3AB99A6AEA
:101660002AB9D86A003818BF0120404270474FF0AD
:10167000FF307047BC30002008B50146044801F037
:10168000BAF820B9BDE808400248FFF789BD08BD97
:10169000BC3000204405002030B50246114890F9C6
:1016A0001C3093421ADD90F92430934218DAD31A91
:1016B000856A0D4CE85C235693420ED00E34002907
:1016C0000CBF0346431CA542D8B206D129B1013A4A
:1016D000D2B2012A01D80130C0B230BD0D20FCE7E2
:1016E0000020FAE7982B002034E5010008B5054BEF
:1016F00093F91C30984203DAFFF7CEFF024B1B56DA
:10170000184608BD982B002034E5010010B51C4C8C
:1017100094F82C3073B9012384F82C3000F0A8F829
:1017200048B1184BA362D823236284F824300823DD
:10173000A361237710BD00F0B1F80028F1D100F0CB
:10174000B7F80028EDD100F075F838B10E4BA36260
:10175000D823236284F824300423E9E700F074F8E6
:101760000028F3D100F07AF80028EFD100F08AF8D1
:101770000028EBD14FF4DF71742000F023F800BF94
:10178000982B00206FE5010042E50100BFF34F8F69
:101790000549064BCA6802F4E0621343CB60BFF30D
:1017A0004F8F00BFFDE700BF00ED00E00400FA0529
:1017B00008B572B6024B5B6803B19847FFF7E6FFC6
:1017C000283000201FB572B6134B5D688DB9FFF746
:1017D000DDFFB2FBF6F2DCB20133002AF9D104F1ED
:1017E00010036B4403F80C2C0A2234B901A8A84753
:1017F000EDE7024600230A26EDE7631E04AEDCB2E5
:1018000056FA83F3B0FBF2F602FB1600303003F811
:101810000C0C3046E9E700BF283000204FF0805222
:10182000034BD2F830111960D2F834215A60704756
:1018300064300020034B1868A0F10F035842584150
:10184000704700BF64300020034B1868A0F10A0302
:1018500058425841704700BF64300020034B18685D
:10186000A0F10E0358425841704700BF6430002079
:10187000034B1868A0F1100358425841704700BF4D
:1018800064300020044B1868062803D0431C5842DB
:10189000584170470120704764300020034B18689E
:1018A000A0F10D0358425841704700BF643000203A
:1018B000034B1868A0F1080358425841704700BF15
:1018C000643000202DE9F04184075FFA81FE5FD08B
:1018D000002A59D0034601E0002A55D003F801EB55
:1018E000990702F1FF32F7D14EEA0E24032A44EAA7
:1018F00004443ED9151FAE08172D06F10106C3F3A7
:10190000800147D99846002940D048F8044B771AFF
:1019100003EB810C79080CEBC101CCE900440CF11C
:10192000080C6145F9D127F0010C08EB8C016745E3
:10193000CCEB8C7805EB880517D02F1F032F0C609C
:1019400013D9A5F10807032F4C600ED9A5F10C0798
:10195000032F8C6009D9A5F11007032FCC6004D99F
:10196000143D032D0C6188BF4C6102F0030203EBB0
:1019700086034AB1013A83F800E005D0012A83F8D2
:1019800001E018BF83F802E0BDE8F0811546BEE72C
:101990000346A9E719461546CFE700BF81F000418D
:1019A00002E000BF83F0004330B54FEA41044FEA44
:1019B000430594EA050F08BF90EA020F1FBF54EADF
:1019C000000C55EA020C7FEA645C7FEA655C00F07B
:1019D000E2804FEA5454D4EB5555B8BF6D420CDD4C
:1019E0002C4480EA020281EA030382EA000083EACF
:1019F000010180EA020281EA0303362D88BF30BD6F
:101A000011F0004F4FEA01314FF4801C4CEA1131C4
:101A100002D0404261EB410113F0004F4FEA033323
:101A20004CEA133302D0524263EB430394EA050FAE
:101A300000F0A780A4F10104D5F1200E0DDB02FA1D
:101A40000EFC22FA05F2801841F1000103FA0EF2B1
:101A5000801843FA05F359410EE0A5F120050EF177
:101A6000200E012A03FA0EFC28BF4CF0020C43FAA8
:101A700005F3C01851EBE37101F0004507D54FF0B5
:101A8000000EDCF1000C7EEB00006EEB0101B1F505
:101A9000801F1BD3B1F5001F0CD349085FEA30004B
:101AA0004FEA3C0C04F101044FEA445212F5800F56
:101AB00080F09A80BCF1004F08BF5FEA500C50F1F3
:101AC000000041EB045141EA050130BD5FEA4C0CD6
:101AD000404141EB0101013C28BFB1F5801FE9D233
:101AE00091F0000F04BF01460020B1FA81F308BF56
:101AF0002033A3F10B03B3F120020CDA0C3208DD22
:101B000002F1140CC2F10C0201FA0CF021FA02F1FC
:101B10000CE002F11402D8BFC2F1200C01FA02F16C
:101B200020FA0CFCDCBF41EA0C019040E41AA2BF91
:101B300001EB0451294330BD6FEA04041F3C1CDA59
:101B40000C340EDC04F11404C4F1200220FA04F079
:101B500001FA02F340EA030021FA04F345EA030123
:101B600030BDC4F10C04C4F1200220FA02F001FAE5
:101B700004F340EA0300294630BD21FA04F0294667
:101B800030BD94F0000F83F4801306BF81F4801100
:101B90000134013D4EE77FEA645C18BF7FEA655C73
:101BA00029D094EA050F08BF90EA020F05D054EA45
:101BB000000C04BF1946104630BD91EA030F1EBF4A
:101BC0000021002030BD5FEA545C05D1400049414E
:101BD00028BF41F0004130BD14F580043CBF01F541
:101BE000801130BD01F0004545F0FE4141F4700127
:101BF0004FF0000030BD7FEA645C1ABF1946104602
:101C00007FEA655C1CBF0B46024650EA013406BF02
:101C100052EA033591EA030F41F4002130BD00BFC1
:101C200090F0000F04BF0021704730B54FF480647E
:101C300004F132044FF000054FF0000150E700BFFF
:101C400090F0000F04BF0021704730B54FF480645E
:101C500004F1320410F0004548BF40424FF000014B
:101C60003EE700BF42004FEAE2014FEA31014FEA8E
:101C700002701FBF12F07F4393F07F4F81F06051DD
:101C8000704732F07F4208BF704793F07F4F04BF28
:101C900041F40021704730B54FF4607401F0004505
:101CA00021F000411CE700BF50EA010208BF704765
:101CB00030B54FF000050AE050EA010208BF704756
:101CC00030B511F0004502D5404261EB41014FF4BF
:101CD000806404F132045FEA915C3FF4D8AE4FF0C7
:101CE00003025FEADC0C18BF03325FEADC0C18BFAA
:101CF000033202EBDC02C2F1200300FA03FC20FAFB
:101D000002F001FA03FE40EA0E0021FA02F1144447
:101D1000BDE600BF70B54FF0FF0C4CF4E06C1CEA60
:101D200011541DBF1CEA135594EA0C0F95EA0C0FD1
:101D300000F0DEF82C4481EA030621EA4C5123EA44
:101D40004C5350EA013518BF52EA033541F4801173
:101D500043F4801338D0A0FB02CE4FF00005E1FB26
:101D600002E506F00042E0FB03E54FF00006E1FB70
:101D700003569CF0000F18BF4EF0010EA4F1FF04B3
:101D8000B6F5007F64F5407404D25FEA4E0E6D41F3
:101D900046EB060642EAC62141EA55514FEAC52004
:101DA00040EA5E504FEACE2EB4F1FD0C88BFBCF580
:101DB000E06F1ED8BEF1004F08BF5FEA500E50F131
:101DC000000041EB045170BD06F0004646EA0101F7
:101DD00040EA020081EA0301B4EB5C04C2BFD4EB29
:101DE0000C0541EA045170BD41F480114FF0000E22
:101DF000013C00F3AB8014F1360FDEBF002001F090
:101E0000004170BDC4F10004203C35DA0C341BDC09
:101E100004F11404C4F1200500FA05F320FA04F0DB
:101E200001FA05F240EA020001F0004221F000410F
:101E300010EBD37021FA04F642EB06015EEA430E82
:101E400008BF20EAD37070BDC4F10C04C4F12005B2
:101E500000FA04F320FA05F001FA04F240EA020065
:101E600001F0004110EBD37041F100015EEA430E36
:101E700008BF20EAD37070BDC4F1200500FA05F256
:101E80004EEA020E20FA04F301FA05F243EA0203D5
:101E900021FA04F001F0004121FA04F220EA0200E4
:101EA00000EBD3705EEA430E08BF20EAD37070BD2A
:101EB00094F0000F0FD101F00046400041EB01010A
:101EC00011F4801F08BF013CF7D041EA060195F0EC
:101ED000000F18BF704703F00046520043EB0303A6
:101EE00013F4801F08BF013DF7D043EA0603704793
:101EF00094EA0C0F0CEA135518BF95EA0C0F0CD09E
:101F000050EA410618BF52EA4306D1D181EA0301E3
:101F100001F000414FF0000070BD50EA410606BFDD
:101F20001046194652EA430619D094EA0C0F02D122
:101F300050EA013613D195EA0C0F05D152EA033667
:101F40001CBF104619460AD181EA030101F0004185
:101F500041F0FE4141F470014FF0000070BD41F0CE
:101F6000FE4141F4780170BD70B54FF0FF0C4CF4A8
:101F7000E06C1CEA11541DBF1CEA135594EA0C0FC7
:101F800095EA0C0F00F0A7F8A4EB050481EA030E14
:101F900052EA03354FEA013100F088804FEA0333FB
:101FA0004FF0805545EA131343EA12634FEA0222C9
:101FB00045EA111545EA10654FEA00260EF000418A
:101FC0009D4208BF964244F1FD0404F5407402D2DC
:101FD0005B084FEA3202B61A65EB03055B084FEA6D
:101FE00032024FF480104FF4002CB6EB020E75EB6A
:101FF000030E22BFB61A754640EA0C005B084FEA92
:102000003202B6EB020E75EB030E22BFB61A75460E
:1020100040EA5C005B084FEA3202B6EB020E75EB59
:10202000030E22BFB61A754640EA9C005B084FEAD1
:102030003202B6EB020E75EB030E22BFB61A7546DE
:1020400040EADC0055EA060E18D04FEA051545EACD
:1020500016754FEA06164FEAC30343EA52734FEA76
:10206000C2025FEA1C1CC0D111F4801F0BD141EAEF
:1020700000014FF000004FF0004CB6E711F4801F54
:1020800004BF01430020B4F1FD0C88BFBCF5E06F34
:102090003FF6AFAEB5EB030C04BFB6EB020C5FEA44
:1020A000500C50F1000041EB045170BD0EF0004E99
:1020B0004EEA113114EB5C04C2BFD4EB0C0541EACB
:1020C000045170BD41F480114FF0000E013C90E6C8
:1020D00045EA060E8DE60CEA135594EA0C0F08BF8C
:1020E00095EA0C0F3FF43BAF94EA0C0F0AD150EA8B
:1020F00001347FF434AF95EA0C0F7FF425AF10461E
:1021000019462CE795EA0C0F06D152EA03353FF445
:10211000FDAE1046194622E750EA410618BF52EAC2
:1021200043067FF4C5AE50EA41047FF40DAF52EA96
:1021300043057FF4EBAE12E74FF0FF3C06E000BF33
:102140004FF0010C02E000BF4FF0010C4DF804CD40
:102150004FEA410C7FEA6C5C4FEA430C18BF7FEA00
:102160006C5C1BD001B050EA410C0CBF52EA430C2E
:1021700091EA030F02BF90EA020F0020704710F1AE
:10218000000F91EA030F58BF994208BF90422CBF3D
:10219000D8176FEAE37040F0010070474FEA410C36
:1021A0007FEA6C5C02D150EA013C07D14FEA430C54
:1021B0007FEA6C5CD6D152EA033CD3D05DF8040BC5
:1021C000704700BF8446104662468C4619466346F7
:1021D00000E000BF01B5FFF7B7FF002848BF10F1CE
:1021E000000F01BD4DF808EDFFF7F4FF0CBF012013
:1021F00000205DF808FB00BF4DF808EDFFF7EAFF8F
:1022000034BF012000205DF808FB00BF4DF808ED49
:10221000FFF7E0FF94BF012000205DF808FB00BF3E
:102220004DF808EDFFF7CEFF94BF012000205DF8C8
:1022300008FB00BF4DF808EDFFF7C4FF34BF0120D5
:1022400000205DF808FB00BF4FEA4102B2F1E04315
:1022500024BFB3F5001CDCF1FE5C0DD901F0004C8D
:102260004FEAC0024CEA5070B2F1004F40EB8300DD
:1022700008BF20F00100704711F0804F21D113F109
:102280003872BCBF01F00040704741F480114FEA42
:102290005252C2F11802C2F1200C10FA0CF320FACB
:1022A00002F018BF40F001004FEAC1234FEAD323E8
:1022B00003FA0CFC40EA0C0023FA02F34FEA430352
:1022C000CCE77FEA625307D150EA01331EBF4FF0DB
:1022D000FE4040F44000704701F0004040F0FE40F6
:1022E00040F40000704700BF80F0004002E000BFF3
:1022F00081F0004142001FBF5FEA410392EA030FF1
:102300007FEA226C7FEA236C6AD04FEA1262D2EB3A
:102310001363C1BFD218414048404140B8BF5B423F
:10232000192B88BF704710F0004F40F4000020F0D8
:102330007F4018BF404211F0004F41F4000121F0EE
:102340007F4118BF494292EA030F3FD0A2F1010238
:1023500041FA03FC10EB0C00C3F1200301FA03F176
:1023600000F0004302D5494260EB4000B0F5000F99
:1023700013D3B0F1807F06D340084FEA310102F158
:102380000102FE2A51D2B1F1004F40EBC25008BF0A
:1023900020F0010040EA03007047490040EB0000D4
:1023A000013A28BFB0F5000FEDD2B0FA80FCACF1D5
:1023B000080CB2EB0C0200FA0CF0AABF00EBC25002
:1023C00052421843BCBFD0401843704792F0000FF0
:1023D00081F4000106BF80F400000132013BB5E743
:1023E0004FEA41037FEA226C18BF7FEA236C21D0B9
:1023F00092EA030F04D092F0000F08BF084670471E
:1024000090EA010F1CBF0020704712F07F4F04D1EB
:10241000400028BF40F00040704712F100723CBFFE
:1024200000F50000704700F0004343F0FE4040F428
:10243000000070477FEA226216BF08467FEA2363E6
:102440000146420206BF5FEA412390EA010F40F4D1
:10245000800070474FF0000304E000BF10F000431D
:1024600048BF40425FEA000C08BF704743F0964304
:1024700001464FF000001CE050EA010208BF70471F
:102480004FF000030AE000BF50EA010208BF7047A6
:1024900011F0004302D5404261EB41015FEA010CBB
:1024A00002BF84460146002043F0B64308BFA3F1B3
:1024B0008053A3F50003BCFA8CF2083AA3EBC25395
:1024C00010DB01FA02FC634400FA02FCC2F12002B4
:1024D000BCF1004F20FA02F243EB020008BF20F0EB
:1024E0000100704702F1200201FA02FCC2F1200251
:1024F00050EA4C0021FA02F243EB020008BF20EA46
:10250000DC7070477BB972B90029BEBF00204FF064
:10251000004106E008BF00281CBF6FF000414FF0EB
:10252000FF3000F057B8ADF1080C6DE904CE00297A
:1025300009DB002B1ADB00F09DF9DDF804E0DDE992
:10254000022304B07047404261EB4101002B1BDBCA
:1025500000F090F9DDF804E0DDE9022304B0404228
:1025600061EB4101524263EB43037047524263EB1C
:10257000430300F07FF9DDF804E0DDE9022304B055
:10258000404261EB41017047524263EB430300F06C
:1025900071F9DDF804E0DDE9022304B0524263EB97
:1025A0004303704753B94AB9002908BF00281CBF2C
:1025B0004FF0FF314FF0FF3000F00CB8ADF1080CD8
:1025C0006DE904CE00F056F9DDF804E0DDE9022300
:1025D00004B07047704700BF10F8012B11F8013BA1
:1025E000012A28BF9A42F7D0D01A7047034613F841
:1025F000012B002AFBD1181A0138704708B5FFF7E4
:102600000DF9BDE80840FFF781B870B5841A04F3EE
:1026100007040E4660B259B21546FFF767F800236B
:1026200030702844737040B270BD13B50C4611462B
:1026300001AAFEF75BFE9DF804309DF906002370A9
:102640009DF80530637002B010BD00230360704731
:102650007047002070474FF0FF3070474FF0FF3059
:10266000704770474FF0FF307047002070470020E0
:1026700070470023037070470022FFF7C6BF002099
:1026800070474FF0FF3070474FF0FF3070474FF00A
:10269000FF30704770478B8C8383FF2380F8303086
:1026A00080F84C3000207047536973B506460D46DC
:1026B0001446B3B140B10092136804F11401012231
:1026C000FEF774FE58B9266275B1236800940022A3
:1026D00004F114012846FEF769FE00B9656202B0F4
:1026E00070BD4FF0FF30FAE72846F8E7D36873B5BE
:1026F00006460D461446B3B140B10092536804F14A
:102700000C010122FEF752FE58B9A66275B163684A
:102710000094002204F10C012846FEF747FE00B9A0
:10272000E56202B070BD4FF0FF30FAE72846F8E7E7
:10273000436910B50446A3B1006A28B122460121BD
:10274000FEF7A8FE60B92062606A28B12246002127
:10275000FEF7A0FE20B960622046FEF709FE0020C9
:1027600010BD4FF0FF30FBE7C36810B50446A3B1BE
:10277000806A28B122460121FEF78CFE60B9A06272
:10278000E06A28B122460021FEF784FE20B9E0620B
:102790002046FEF7EDFD002010BD4FF0FF30FBE7B7
:1027A00073B50123144682F8343004F13406002254
:1027B0000D46A063236884F84820009404F11401B6
:1027C0003046FEF7F3FD50B902466368009404F109
:1027D0000C013046FEF7EAFD08B984F84C5002B00F
:1027E00070BD0323036070477047002070470020CE
:1027F00070470020704737B50C460546502200212F
:10280000FFF760F8637A6B7263686B60237A2B72F0
:102810002146284651F8183B40F80C3BFEF71EFDB8
:1028200005F1140004F10C01FEF718FD28462146BD
:10283000FFF731FF054650B994F90830ADF80500AF
:102840008DF8070001A88DF80430FEF759FD2846E1
:1028500003B030BD00280CBF6FF01500002070479A
:102860000020704707230370002070470020704746
:10287000002070472DE9F04786468C460846089EA2
:10288000154674461946002B40F0C2808542B2FAC4
:1028900082F245D94AB1C2F1200300FA02FC2EFAB5
:1028A00003F3954043EA0C0C94404FEA154EA8B24E
:1028B000BCFBFEF8230C0EFB18CC08FB00F943EA26
:1028C0000C43994528D9EB1808F1FF3704D29945F4
:1028D00002D9A8F102072B44A3EB0903A4B2B3FB6E
:1028E000FEFC0EFB1C330CFB00F044EA0344A04248
:1028F00014D92C190CF1FF3304D2A04202D9ACF147
:1029000002032C44241A43EA07401EB1D44000239A
:1029100034607360BDE8F0874746DDE76346F1E762
:1029200092BB431B01214FEA154EAFB2B3FBFEFC35
:10293000200C0EFB1C330CFB07F840EA03439845C0
:1029400062D9EB180CF1FF3004D2984502D9ACF1F2
:1029500002002B44A3EB0803A4B2B3FBFEFC0EFB66
:102960001C330CFB07F744EA0344A7424ED92C1949
:102970000CF1FF3304D2A74202D9ACF102032C447C
:10298000E41B43EA0040C0E7C2F1200320FA03F150
:10299000954090402EFA03F303434FEA154EAFB231
:1029A000B1FBFEFC0EFB1C10190C0CFB07F841EAF6
:1029B0000041884504FA02F422D969180CF1FF306D
:1029C00004D2884502D9ACF102002944A1EB0801E8
:1029D0009BB2B1FBFEFC0EFB1C110CFB07F743EA9C
:1029E00001439F420ED9EB180CF1FF3104D29F42F4
:1029F00002D9ACF102012B44DB1B41EA004192E712
:102A00006046E3E76146F7E76046A3E76346B7E75A
:102A1000834206D916B9002108467BE7C6E900E0E3
:102A2000F9E7B3FA83F78FB9834201D3724508D827
:102A3000BEEB020460EB030301209C461EB900219B
:102A400068E73846FAE7C6E9004CF8E7C7F1200C1A
:102A5000BB4022FA0CF41C432EFA0CF120FA0CF3C2
:102A6000B84001434FEA14490EFA07F5B3FBF9F8F1
:102A70001FFA84FE09FB18300B0C08FB0EFA43EA20
:102A800000439A4502FA07F240D9E31808F1FF30F3
:102A900004D29A4502D9A8F102002344A3EB0A0309
:102AA00089B2B3FBF9F809FB183308FB0EFE41EAC3
:102AB00003418E452CD9611808F1FF3304D28E45AD
:102AC00002D9A8F10203214443EA0040A0FB029886
:102AD000A1EB0E014145CE46434602D306D14D45FA
:102AE00004D2B9EB020E68EB04030138002EA6D025
:102AF000B5EB0E0261EB030101FA0CFC22FA07F3BD
:102B00004CEA0303F940C6E9003198E74046C5E7BF
:102B10004346D9E7000000002DE9F04F2DED028B70
:102B2000A1B00AF029FF08F0A9FD002840F0DB80E1
:102B3000002140F6CD4015F0D7FCB548DFF88C8376
:102B400019F0CDFA35231321CDE90131032340F2E9
:102B5000EA710A22AF480093012319F0C0FAAE4887
:102B600019F0BDFAAD4819F0BAFAAD4819F0B7FA44
:102B7000AC4819F0B4FAAC4819F0B1FAAB4819F006
:102B8000AEFAAB4819F0ABFAAA4819F0A8FAAA486D
:102B900019F0A5FAA94B18681B798DF82430A84BB9
:102BA00008909A8818689B798DF85630A54B149038
:102BB00018681B798DF82C30A34BADF854200A907F
:102BC0009A8818689B798DF85E30A04B0493A04BCF
:102BD0001690ADF85C2018689A889B798DF866305D
:102BE0009C4B189018681B798DF834309A4B0C90D8
:102BF0001868ADF864200E901B798DF83C30974B27
:102C0000186812909B889648ADF84C3019F067FA16
:102C1000944B9548059319F062FA944B18681090FC
:102C20001B7993488DF8443019F059FA914819F0FE
:102C300056FA914819F053FA904819F050FA904812
:102C400019F04DFA8F4819F04AFA8F4819F047FAEF
:102C50008E4819F044FA8E4819F041FA8D4819F05F
:102C60003EFA8D4B18689A889B798DF86E308B4BA5
:102C7000069365A7D7E9006705331A90ADF86C2075
:102C800007930AF061FE0024054601460A7872BBEC
:102C9000052208A928461AF0D1FE002846D180480E
:102CA00019F01DFA35231322CDE9013203230A223C
:102CB00040F2EA7100935748012319F010FA79485D
:102CC00019F00DFA784819F00AFA784819F007FA5D
:102CD0004FF080527648D2F8A830D2F8A4209BB2A8
:102CE00019F0FDF9CDE7012015F03AFC1BE718F8C3
:102CF00002004B7800F00300012804D120320A7052
:102D00000A46511CC2E7202AFAD1002CF8D10C70D7
:102D100018F8032002F00302012A08BF2033DBB2B7
:102D20004A1C4B70002B18BF1446EAE7072214A96F
:102D300028461AF083FEB0BB1AF040FE5D4AA0FBA5
:102D4000020302FB0131C00B40EA41405A4A1423FE
:102D5000C90BFFF7D7FB0446194610463B463246DF
:102D6000FFF7D0FB0546194610460023534AFFF7EC
:102D7000C9FB81461946104600234E4AFFF7C2FBA5
:102D800082461946104600234FF47A72FFF7BAFBC9
:102D9000CDF800A0CDE901024B4649482A4621461C
:102DA00019F09DF96DE704A9042228461AF046FEA1
:102DB0000146F8B91022204616F086FE414ACDE9B8
:102DC000000181460D461CA80D2119F095F959EA1C
:102DD00005030BD00D2221461CA81AF02FFE28B99E
:102DE00001224846294603F0CFFB4AE7364819F04E
:102DF00076F946E7072218A928461AF01FFE002890
:102E000066D103F06BFC3CE700A493D60000000001
:102E100035F1010069F10100CCF1010001F201007E
:102E200031F2010062F2010096F20100CAF20100E3
:102E3000FBF201002CF301005CF30100B408020076
:102E400056FE01005DFE010062FE01006164640047
:102E500072F0010069FE01006EFE010073FE0100C8
:102E60008FF3010064667500C2F30100D1FE01001A
:102E7000E6F301002BF401006FF40100BFF4010040
:102E800008F501004AF501008DF50100D6F50100B5
:102E900015F601004CF6010079FE01006869640036
:102EA0008AF60100B6F60100CDF60100DCF601005D
:102EB000FCF6010040420F000060D71D008793031D
:102EC00016F701003BF7010043F70100042402005C
:102ED00005220AA928461AF0B1FD8146B0B9A248D8
:102EE000A24DDFF810A319F0FAF84C46DFF808936A
:102EF0002A78E3B29A427FF6C4AE09EBC303D3E962
:102F00000023504619F0EBF80134F1E7072216A927
:102F100028461AF093FD48B909F00EFD4FF4004021
:102F2000002115F0E1FA012007F0D4FA042207A9E4
:102F300028461AF083FD50BB5CB18D490322204620
:102F40001AF07CFDC8B9012005F082FA002005F0D6
:102F5000A5FD05F083FA874D874C00280CBFA946D4
:102F6000A14605F0A1FD494600280CBF2A4622468D
:102F7000824819F0B4F8824839E782490422204691
:102F80001AF05CFD0028E4D105F062FAE1E70422C2
:102F900006A928461AF052FDE0B99CB17A490422EC
:102FA00020461AF04BFD054660B97849204616F0D8
:102FB00035FC7649284616F031FC18B11AF03AFD76
:102FC00005F020FA05F02AFA0146714819F087F851
:102FD00070480CE707221AA928461AF02FFD00288E
:102FE00040F07882002C40F093806B48614D624C39
:102FF0009FED6A8A19F073F805F056FD00280CBFA2
:1030000029462146664819F06AF805F07BFD00283C
:103010000CBF29462146634819F061F805F072FD9E
:10302000B8B105F091FD60EE087A17EE900AFEF750
:1030300019FE02460B465C4819F051F805F09AFD5E
:1030400010EE100AFEF70EFE02460B46574819F026
:1030500046F85748474C19F042F805F0A1FD464B99
:10306000002818BF1C4605F0D1FD10EE100AFEF72F
:10307000F9FD82468B4605F0CFFD10EE100AFEF7F3
:10308000F1FD5246CDE900015B462146494819F061
:1030900026F805F0E3FD60EE087A17EE900AFEF7D9
:1030A000E1FD04460D4605F02DFD58BB424B43485B
:1030B000009322462B4619F012F805F0E9FC10EEB9
:1030C000100AFEF7CFFD02460B463D4819F007F8FF
:1030D0003C4819F004F83C4819F001F83B4818F056
:1030E000FEFF3B4818F0FBFF3A4818F0F8FF3A485B
:1030F00018F0F5FF394818F0F2FF394818F0EFFFE3
:10310000384874E605F04CFD0028CFD1364BCEE7A9
:103110001749032220461AF091FC054638B90120D0
:1031200005F0EAFC284605F035FD30485FE6154914
:10313000042220461AF082FC054600285ED105F0E4
:10314000DBFC284605F026FD05F088FDDFED137A4F
:1031500060EE277A17EE900AFEF784FD02462448B7
:103160000B4618F0BCFF8CE554F70100C138022073
:10317000EC130200EFF00100ECF0010069F7010030
:1031800094F7010065F70100E6F70100EC0C02007E
:10319000EBF701002FF8010063F8010000007A440A
:1031A00083F80100A2F80100C0F80100D4F8010082
:1031B000790C0200EEF801000CF1010027F9010082
:1031C00051F9010072F9010078F90100BDF901001F
:1031D00002FA010042FA01007BFA0100B8FA01008C
:1031E000EBFA01002FFB0100F3F0010066FB010088
:1031F0008EFB01000DF70100A04D0020BF49052204
:1032000020461AF01BFC0546A8BBBD49204616F017
:1032100005FBBB49284616F001FB50B1B949032212
:103220001AF00CFC18BB012005F0B4FC012005F0DD
:1032300063FC05F0B5FCB44CB44B002818BF1C4629
:1032400005F0E4FC10EE100AFEF70CFD82468B46FA
:1032500005F0E2FC10EE100AFEF704FD5246CDE93F
:1032600000015B46AA48214618F039FF09E52846C7
:1032700005F090FCDDE7A749072220461AF0DEFBA7
:103280000546002839D19E49204616F0C7FA9C49C8
:10329000284616F0C3FA9A498146284616F0BEFA27
:1032A0000446B9F1000F12D088B148461AF0C2FBAB
:1032B00008EE100A20461AF0BDFBB8EEC88A00EEF0
:1032C000900AB0EE480AF8EEE00A05F06FFC05F04F
:1032D0009DFC10EE100AFEF7C5FC04460D4605F0F5
:1032E0009BFC10EE100AFEF7BDFC2246CDE9000162
:1032F0002B46894818F0F3FEC3E48849062220468D
:103300001AF09CFB054600BB7D499FED858A20464F
:1033100016F084FA7A49284616F080FA48B11AF075
:1033200089FB00EE100AB8EEC00A80EE080A05F02C
:10333000EFFB05F009FC60EE087A17EE900AFEF745
:1033400091FC02460B4677480BE777490522204659
:103350001AF074FB0546D0B96949204616F05EFAAA
:103360006749284616F05AFA38B11AF063FB00EEA6
:10337000100AB8EEC00A05F0EDFB05F0FBFB10EEFD
:10338000100AFEF76FFC02460B466848E9E66849FA
:10339000032220461AF052FB054678BB58499FEDA0
:1033A000608A204616F03AFA5549284616F036FA51
:1033B00048B11AF03FFB00EE100AB8EEC00A80EEEA
:1033C000080A05F02FFC05F049FC60EE087A17EEBC
:1033D000900AFEF747FC04460D4605F03FFC554AAF
:1033E000554B5648B5EEC00AF1EE10FA88BF1346A9
:1033F000009322462B4618F072FE42E45049072201
:1034000020461AF01BFB0546E8B93D49204616F058
:1034100005FA3B49284616F001FA38B1394903222A
:103420001AF00CFB68B9012005F038FB05F03CFBF5
:10343000354A3649002808BF1146424818F04FFE69
:103440001FE40020F0E74049072220461AF0F6FA70
:10345000054680BB2A49204616F0E0F9284900209D
:1034600016F0DCF98146E0B11AF0E4FA2E210446A8
:1034700048461AF009FB18B101301AF0DBFA05468C
:103480006423002C04FB03F3B8BF6D422B4400EE11
:10349000103ADFED2E7AB8EEC00A80EE270A05F06A
:1034A00049FA05F0F5FA10EE100AFEF7DBFB0246CA
:1034B0000B46274855E62146264818F010FE2648B8
:1034C00018F00DFE254818F00AFE254818F007FEF2
:1034D00024488CE405220CA928461AF0AFFA18B942
:1034E00003F006FAFFF7CDBB05220EA928461AF015
:1034F000A5FAC8BB03F00AFAFFF7C3BBD0FB010073
:10350000EC0C0200EC130200EFF00100ECF0010003
:10351000D5FB01000AFC010011FC01003CFC01008C
:1035200000007A4442FC0100E6F7010069FC01005A
:10353000A2FC01007A0C02002EF10100A6FC0100A1
:10354000CBFC0100D2FC0100EFFC01000000C842EE
:10355000F6FC01000FFD01002CFD010060FD0100E3
:1035600090FD0100CEFD0100062212A928461AF0A6
:1035700065FA18B903F0D0F9FFF783BB042205A957
:1035800028461AF05BFAE0B92548436881681B6851
:1035900002691B030AD4234923484FF47F7218F0B1
:1035A00011FE20484FF47F7118F003FE136823F4D6
:1035B000002313600B684FF4C02213219847FFF7D4
:1035C00060BB052210A928461AF038FA20BB1AF071
:1035D000F5F94FF4C3620023FEF794FF1046194635
:1035E0004E220023FEF78EFF0446194610460023A4
:1035F0000D22FEF787FF0D4B0D49D2B2C0B253F832
:1036000022300C4AE4B252F8202051F824100A4823
:1036100018F065FDFFF735BB0848FFF7E8BB00BFB2
:10362000E4DF0100F7FD010025FE0100D8E50100FF
:1036300024E601000CE601003DFE010045FE01000C
:103640002DE9F04F2DED048BA7B002AF04F08AFAFC
:103650001023BB62EFF3118C402383F31288BFF376
:103660006F8F254EDFF89C9096F80138BB63082BCE
:10367000A8BF0823984696F800E80023FB64FB6C7B
:103680000EEB0304984504F03F0425D1BB6BFA6CA4
:1036900086F800489B1A86F801388CF31188BFF32E
:1036A0006F8F0023DFF860B0FB63FB6BFA6C934213
:1036B0002CD1BB6B072B03D9BB6A013BBB62C9D1C1
:1036C0000E4B5B687B640E4B1878002840F09F859A
:1036D00004F07EFA00F0C9BFFB6C06EB441409EB62
:1036E00043150FCC0FC594E80F0085E80F00FB6C65
:1036F0000133FB64C3E700BF986F0020001000E0B7
:10370000C23F0220A0550020AA550020A94B9BF8DB
:1037100007201A709BF806303B63A74B3A6B1A7070
:10372000DBF80E30BB64DBF812307B6418F073F901
:10373000A24B7963D3E900211BF8096C38640A4372
:1037400004BF02461A601BF80A1C04BF7A6B5A6059
:10375000304603F089FE1BF80A8CB8F1000F6BD1DC
:10376000DFF868A20625754306EB46030AEB05045D
:103770007B620AEB4303FB626379ABF10509002B23
:103780004BD0F86A052249461AF058F9002844D06F
:103790008B4A13680133032B13603ED863783B6276
:1037A000A378FB61E378BB6123797B611BF8053C5F
:1037B0001AF805201BF8011C3B6112201BF8043C81
:1037C0001BF8035C1BF8024C7A60FB60B96007F0E1
:1037D0003FFFE0B17B4B7A68B968C261C0E905364A
:1037E0003B6A0362FB694362BB6983627B69C362B4
:1037F0003B690363FB68C463C0E90D350D230164B5
:10380000037480F8118080F8128080F813806E496C
:1038100000234FF4D14219F079F97A6AD9F80030CF
:103820004AF81230FA6A99F804301371674B06228D
:1038300002FB063301225A71604B3A6CD3E9005304
:10384000501B7A6B41F2883162EB0303884273F1BB
:1038500000030546C0F2F880F862EFF311824024BD
:1038600084F31288BFF36F8F594BD3F80418F960B3
:1038700093F8011893F8088883F8081882F31188E0
:10388000BFF36F8F534B54481B687B62534B1B68CD
:103890003B624B4B1968524B79601A68514BBA60C6
:1038A0001B68FB6103685048BB61D0F800A04F481B
:1038B000D0F800904E4803684E487B6106684E4839
:1038C00003683B61162007F0C3FE00B34B4B7968D9
:1038D000BA68C461C0E90538FB6803627B6A436269
:1038E0003B6A8362FB694363BB69C162C0E90E3A0C
:1038F0007B690263C0E911363B69C0F84090C0E9BA
:10390000133511230374002343748374C3742E4945
:10391000002348F6C00219F0F9F8364A0023136074
:10392000334A1360344A13602E4A13602C4A1360E2
:103930002A4A1360274A1360214A13602B4A1360F6
:10394000294A1360244A07F1700007F180011360CF
:1039500004F070FD04F062FD3B6F2DB14FF47A72FC
:103960005A43B2FBF5F2FA62254A264C1178264AF0
:10397000264D274ED7F8809000290CBFA4469446C8
:10398000244C2A687A62E84690B0D4F800E03168A6
:1039900002AAD361FB6ADFF884A0C2E908397B6A16
:1039A000C2E90C3140F2046313871B4BC2E905A046
:1039B00036E000BFC0380220BF380220A0560020E9
:1039C000C0D401206605020054E40100C238022080
:1039D000986F0020BCD4012070D40120B8D40120FD
:1039E000B4D40120B0D401206CD4012068D40120CB
:1039F000CCF80120C8F80120C4F80120B20502006B
:103A0000A9280020EFF00100ECF00100D4F801201B
:103A1000D0F80120D8F801200A000001AE0602000B
:103A2000C2E90ACE42F8103F0023CF4845F2C04118
:103A300007F0B4FF002333602B602360CB4B3A6C5C
:103A40001A607A6B5A60C5461BF80A4C072C00F2C4
:103A500064826FF09606264116F0010640F05D8202
:103A6000ABF10A031022314607F16000C7E9156681
:103A70003B64FE651AF000F8012C02D0042C40F0E3
:103A8000CD813BF9020CFEF7DBF800224FF07C53AE
:103A9000FEF740F9FEF7D8FB38663BF9080CFEF755
:103AA000CFF800224FF07C53FEF734F9FEF7CCFB41
:103AB00078663BF9060CFEF7C3F800224FF07C5302
:103AC000FEF728F9FEF7C0FBB8663BF9040CFEF7D9
:103AD000B7F800224FF07C53FEF71CF9FEF7B4FB59
:103AE000F8661BF80A1C1BF8090CA14C07F16002D0
:103AF00003F03CFD1BF8093C9E4A04EB03142146ED
:103B000007F1600002EB031805F076FC414607F16F
:103B10006000B0EE408A05F06FFCD4ED007AF5EE5F
:103B2000407AF1EE10FAF0EE408A15D1D4ED017A28
:103B3000F5EE407AF1EE10FA0ED1D4ED027AF5EE00
:103B4000407AF1EE10FA07D1D4ED037AF5EE407A1F
:103B5000F1EE10FA00F0A581B6EE007AB4EEC78A55
:103B6000F1EE10FA40F39D81DFED837AB4EEE78A3F
:103B7000F1EE10FA40F19581F4EEC78AF1EE10FAF9
:103B800006DDF4EEE78AF1EE10FA4CBF01260026BE
:103B90007A4ADFED7B7A13681BF809AC1BF80A9CA4
:103BA00068EE277A01331360FCEEE77A754A17EE68
:103BB000903A11688B4288BF1360734B03EBCA03C2
:103BC00093ED009B714B102053F82A307B6307F074
:103BD0003FFD0546C8B16E4B436180ED069BC0E9D1
:103BE00008A918EE100AFEF73DF8C5E90A0118EE1B
:103BF000900AFEF737F87B6BAB63C5E90C010B232A
:103C00002B7400236B74AB74EB7428465649002365
:103C10004FF4B14218F07AFF5C4B1BF8095C53F883
:103C2000252002F1010C43F825C007F160030FCBFA
:103C300088E80F0036BBBCF1020F23DD524B0A208F
:103C400003EBC503D3E9008907F002FD48B1514BEE
:103C50004361C0E9068905230562037446748674CE
:103C6000C674414900234FF4225218F04FFF1BF84D
:103C7000092C464B002143F8221007F160030FCBBB
:103C800084E80F001BF80A6C012E0AD0072E00F200
:103C900044819423F340DC0740F13F81301F4642CA
:103CA0004641D7E911321BF8090C07F1600100F019
:103CB000DBFD04F0F9FE002800F000811BF8090C80
:103CC00007F1700104F0FCFE002800F0268197ED5A
:103CD0001D6AD7ED1C7AD7ED1E6A97ED1F7A9FED0E
:103CE0002E5A66EE065A47EEA75A46EEA65A47EEF9
:103CF000075AF4EEC55AF1EE10FA40F30E819FED2B
:103D0000275AF4EEC55AF1EE10FA40F10681002E62
:103D100000F02A829FED225ADFED225A26EE056A34
:103D2000B4EEE56AF1EE10FA00F3DC81DFED1E4A35
:103D3000B4EEE46AF1EE10FA00F1D781BDEEC66A86
:103D400016EE103A1BB266EE856A2BF8083CF4EECC
:103D5000E56AF1EE10FA00F3CA819FED136AF4EE02
:103D6000C66AF1EE10FA21E054E40100A0560020EA
:103D70004016002040060020C3F5B840BCD4012006
:103D800000007A44B8D40120A04D0020C4D4012002
:103D900045070200860702006666663FCDCC8C3F71
:103DA0000000004700FEFF46000000C700F1A281AE
:103DB000FDEEE66A16EE903A1BB227EE057A2BF876
:103DC000063CB4EEE57AF1EE10FA00F395815FED72
:103DD0000A6AB4EEE67AF1EE10FA00F19081BDEED7
:103DE000C77A17EE103A1BB267EE857A2BF8043CBF
:103DF000F4EEE57AF1EE10FA00F383811FED167A06
:103E0000F4EEC77AF1EE10FA00F17E81FDEEE77A6A
:103E100017EE903A1BB22BF8023C7EE03B6CD3F8D5
:103E20000540C4F30900FDF7FBFEB84B0022FDF787
:103E300071FFFEF709FA07EE900A77EEA77AB7EE60
:103E4000008A77EEC87AC4F38A20C7ED157AFDF7A9
:103E5000E7FE00224FF07D53FDF75CFFFEF7F4F91B
:103E600007EE900A77EEA77A600D77EEC87AC7ED75
:103E7000167AFDF7D5FE00224FF07D53FDF74AFF7D
:103E8000FEF7E2F907EE900A77EEA77A07F16001F4
:103E900077EEC87A07F15400C7ED177A05F018FBE2
:103EA0001FE61BF8092C9A4B002107F1600543F827
:103EB000221095E80F0088E80F00E1E6954B1B788B
:103EC0005BB31BF8094C002E40F08E800BF1FF3ADB
:103ED0003B6EC7F880307B6EC7F88430BB6EC7F886
:103EE0008830FB6EC7F88C3023018B4D7B638B4B86
:103EF00003EB04182B5D002B78D107F1900313E935
:103F00000F0088E80F00864BB96C43F8341003EBC0
:103F1000C4027B6C536001232B55824CABF10A0524
:103F20000BF1060622462B4603CBB34220606160AC
:103F30001D4604F10804F6D11BF80A1C012903D020
:103F400004291CBF3B6BD373774C784D20782B78BA
:103F5000DFF808E292F801C0002402019C422BDA4B
:103F600002F110061EF80680E04540F04D81704CCD
:103F7000A65C072E12D86FF0960C4CFA06FC1CF0CB
:103F8000010F0BD1B14209D0072903D89626CE40A4
:103F9000F10703D4674E316801313160664E3168F4
:103FA000013131605F49224401F1100451F8046B82
:103FB00042F8046BA142F9D1642B0ED85C49594AEE
:103FC000184401EB001002F1100152F8044B40F8C4
:103FD000044B8A42F9D101332B70FB6B0133FB6335
:103FE0000BF1200BFFF761BBDA4671E7534A135D13
:103FF0002BB153490B6801330B600023135507F1B4
:104000008001404617F015FDB5EEC00AF1EE10FA3A
:104010005CD4434B03EBC40253F834505368BA6C7E
:10402000551B7A6C62EB0309464A0023AA4273EBE4
:104030000901BCBF9946154642F210739D4279F1C1
:10404000000207F1800107F170024046B6EE000A57
:10405000BCBF1D464FF0000904F0BEFA3A4B7A6B24
:104060001A4407F1800394460FCB8CE80F00374BBE
:10407000DAF8000004EB440203EB420143F81200BB
:10408000BAF804308B806D08BB6C314A45EAC975BB
:10409000ED187B6C42F8345002EBC40143EB69032A
:1040A0004B60264B01221A5507F180030FCB88E89D
:1040B0000F001B4BB96C43F8341003EBC4027B6C4C
:1040C0005360244A13680133136000E607F180034C
:1040D0000422D3ED007A013AF1EE677AE3EC017A3B
:1040E000F7D196E747F6FF732DE61B4B2BE647F615
:1040F000FF7362E6184B60E647F6FF7374E6164BF3
:1041000072E647F6FF7386E6134B84E60000503FE5
:10411000C4D40120A9280020C3460220DC080220C4
:10412000985F0020C6570220C4470220C5470220DE
:10413000C6470220B4D40120B0D40120C3450220D8
:10414000D0F8012080380100DCF80120C33F0220B4
:1041500098570020D8F801200080FFFFB7470220C1
:10416000000000450000804407F18001C7E9206697
:10417000C7F8886007F1700005F05EF9D7ED216A95
:104180005FED095AB7EE006A76EE866AB6EE007AFF
:1041900066EE876AF0EE477A46EEA57A40F2FF7146
:1041A000D7ED226A76EE866AFDEEE77A66EE876ADA
:1041B00017EE902AF0EE477A46EEA57A22EAE272EE
:1041C0008A425FED186AFDEEE77AA8BF0A4617EE4D
:1041D000903AD7ED207A77EE867A23EAE37367EE9A
:1041E000877A8B4207EEA67AA8BF0B465B0543EAA7
:1041F0008223FDEEC77A17EE902A82F30A02134358
:104200003A6CC2F8053088E601343246A6E6A84C7E
:104210002378002B00F02982A64D2B7823B117F0CC
:10422000FAFBA54BC3E9000104F03EFCB0B919F05C
:10423000C5FBA24B1B78002B40F0E5802B78CBB957
:1042400017F0E9FB9E4BD3E90023633861F10001CD
:1042500082428B410EDB0120FFF73ABA17F0DBFBFD
:10426000954AD2E90032C01A61EB0201652871F16A
:104270000001DCDA17F0CFFB914BC3E900012B788A
:10428000BB64904BBFF35B8F53E8002F42F00101FA
:1042900043E800100028F7D1BFF35B8F12F0010A4A
:1042A00040F0DF8295F800B004F0FEFB002800F03B
:1042B0003A8119F083FB844A844EDFF82082DFF8CC
:1042C0002092A0FB020302FB0131C40BCB0B44EA9A
:1042D0004144D6E90001201A63EB0101FB64FDF7BC
:1042E000EBFC71A3D3E90023FDF73EFEFDF7ACFF25
:1042F000FB6C7749346008EE100A736056462B78E1
:10430000B34200F3A1800026694B1A78B3B29A42F7
:1043100040F20981BBF1020F00F305816C49DFF81F
:10432000BC816C4B0D781B883344B3FBF2F002FB6D
:104330001039604B1FFA89F093F800E0002208EB77
:104340000513964500F39E80634BD3F800C0BCF183
:10435000000F40F0CD80614A4FF07F0C0CEB05035D
:1043600003F07F03190102EB031393F801E0864584
:1043700040F08181515C01F1FF3EBEF1010F04D993
:10438000042902D0072940F076815D444FEA051CDC
:1043900002EB0515284603F1100E53F8048B40F884
:1043A000048B7345F9D18423CB40DB0715D5D5F8B1
:1043B0000900B5F80D30A7F88430012302F80C305D
:1043C0008046C7F880000E220021A81C19F054FB7B
:1043D000B7F88430C5F80A80EB81FB6C2246B0EE5A
:1043E000480A284603F09AFC3D4B03EBC90243F808
:1043F0003940FB6C53603B4A1368013313600BF187
:10440000010B013680E7304A94F800E0364CA0FBFF
:10441000020302FB0131C30B344A43EA4143002645
:10442000C90BB0B286457FF609AF14F8010B40B155
:104430005068F86410688342F86C71EB0000BFF6B6
:1044400019AF01360832ECE708783044030108EB75
:10445000001018F80320072A0BD86FF096031341B9
:10446000DA0706D4437809EBC30249F83340FB6C02
:104470005360FB6C2246B0EE480A03F04FFC013655
:1044800013493CE793F801C0844507D193F800C075
:10449000BCF1010F40D0BCF1040F3DD0013210330C
:1044A0004FE700BFAFF300800000000080842E4182
:1044B000C1380220C547022088050020A928002015
:1044C00090570020E818022040420F008857002033
:1044D000C447022054370220E4180220C6470220B5
:1044E00098670020E0180220C3450220985700205A
:1044F000B04A02EBC90352F839205B68B4EB020EF4
:10450000FA6C62EB0303E64573F10003BFF623AFD9
:10451000A94A136801331360A84B01361A78B3B265
:104520009342FFF4FEAEA64B1B78002B3BD004F069
:10453000BBFA002837D119F041FAA24ADFF87C9281
:10454000A0FB020302FB0131C60BCB0B46EA41463E
:104550003B6499F800301FFA8AF2934223D9BBF1E9
:10456000020F20DCDFF8B082974A15885544B5FB6E
:10457000F3F203FB125518F80530002B00F003810D
:10458000924B53F8352003EBC50196424B683A6CC9
:1045900072EB030374DA99F800300AF1010A1FFA8A
:1045A0008AF29A42E0D38A4D8A4E8749DFF86CC27C
:1045B000DFF808925C464FF0FF084FF0000E032C26
:1045C000287840F32D8106EB00118348834E006864
:1045D00007F1800340220AF007FF814B31785B68C6
:1045E00001907A6C9B1A9B0900935A460446042357
:1045F000B86C03F0FFFA3278042A19D979487A4B5B
:10460000E8468AB0111F052A18BF034602AA774858
:10461000D36140F201331384754BC2E9050142F8BE
:10462000103F744800234FF4135107F0B7F9C54603
:104630002B78327813440333DBB2812B28BF00235D
:104640002B700025357084B1062007F001F830B1D9
:10465000694B43610223037445748574C5746549CD
:1046600000234FF4825218F051FA9437BD46BDEC46
:10467000048BBDE8F08FBCF1010CBFF46FAEC0E657
:10468000534B1C785C442301FB64524B03EB041432
:104690000F220021601C19F0EFF9F96C4D4BDFED92
:1046A000576A9FED577A01225A54564A657002EBB9
:1046B0000512D2ED017A67EEA67AF4EEC77AF1EE32
:1046C00010FA63DC9FED506AF4EEC67AF1EE10FA50
:1046D0005FD4FDEEE77A17EE903A1BB2D2ED027A84
:1046E000638067EEA67AF4EEC77AF1EE10FA52DC38
:1046F0009FED456AF4EEC67AF1EE10FA4ED4FDEE67
:10470000E77A17EE903A1BB2D2ED037AA38067EEF8
:10471000A67AF4EEC77AF1EE10FA41DC9FED3A6A20
:10472000F4EEC67AF1EE10FA3DD4FDEEE77A17EE1C
:10473000903A1BB2D2ED007AE38067EEA67AF4EEEF
:10474000C77AF1EE10FA30DC9FED2F7AF4EEC77ADB
:10475000F1EE10FA2CD4FDEEE77A17EE903A1BB288
:104760002A4A238106236B439918D358C4F80A3088
:10477000274A8B88E381002308F80530136801334A
:1047800013600BF1010B0AF1010AE2E647F6FF7331
:10479000A4E7204BA2E747F6FF73B5E71D4BB3E74D
:1047A00047F6FF73C6E71B4BC4E747F6FF73D7E72F
:1047B000184BD5E798670020DC180220C13802208A
:1047C000A928002040420F005437022098570020AB
:1047D000C4470220C6470220EC180220C547022029
:1047E000001000E0BEF801007A0C0200A8070200E9
:1047F0000400000154E40100BC070200000000476F
:1048000000FEFF46DCF80120000000C7C33F022085
:10481000D4F801200080FFFFC3450220A04D0020F6
:1048200002190B884FEA021A06EB021206F80A80F8
:104830000CEBC30A5CF83300C2F80200BAF80400BB
:104840005370D080C2F808E0C2F80CE0013399F848
:1048500000209BB2B3FBF2F002FB10330B8001345B
:10486000ADE60220FEF734BF2DE9F04F2DED048BAD
:104870009A466F4B1B7887B080460D461746002B33
:1048800065D0002963D0D1ED017AD1ED008AD1ED58
:10489000026A91ED037A67EEA77A48EEA87A46EEAF
:1048A000A67A47EE077AB6EE007AF4EEC77AF1EE12
:1048B00010FA4CD4B7EE087AF4EEC77AF1EE10FA9B
:1048C00045DCDFF87C914FF4A876464309EB0604FB
:1048D00004F1400B94F84C30002B3DD1C4ED008A1C
:1048E0004B6863608B68A360CB68E3600B682361EF
:1048F0004B6863618B68A361CB68E3610B682362DB
:104900004B6863628B68A362CB68E3620B682363C6
:104910004B6863638B68A363CB68E3632264CBF863
:1049200004A00B68C4F890304B68C4F894308B68CE
:10493000C4F89830CB68C4F89C304FF48073A4F866
:1049400030310123C4F81021A26484F84C3007B040
:10495000BDEC048BBDE8F08F236CDBF80420FB1A60
:1049600000936AEB0203194600980193FDF7A4F93E
:104970002DA3D3E90023FDF7F7FAFDF765FC2D4BD6
:104980002D49D3ED000A2D4B08EE100A0098D3ED07
:10499000009A814201994FF0000306F1100273EB77
:1049A00001014A444EDAC4ED0C8A69686163A96862
:1049B000A163E9680092B0EE480AE1632764CBF88E
:1049C00004A003F0C7FEF0EE690AF0EE408AB0EEF4
:1049D000480A03F0BFFE2946B0EE408A2046B0EEFA
:1049E000680A03F0EDFE009AB0EE480A1046214630
:1049F00003F0E6FE2269C4F890206269C4F89420AE
:104A0000A269C4F898200023E269C4F89C2084F8C5
:104A100064304FF480720023C4F81071A4F8302180
:104A2000236594E7AFF300800000000080842E41EE
:104A3000D858022050260020400D03004C260020AC
:104A4000A877002006F1300327644B44CBF804A07C
:104A5000D3ED017A95ED016A93ED005AD5ED005A38
:104A6000D5ED026A95ED037A009266EE277A45EE5F
:104A7000857A4FF4A87A0AFB089593ED025A46EE20
:104A8000857A93ED035A47EE057AB0EE480AF5EEC3
:104A9000C07AF1EE10FA41BFF1EE655AB1EE466A06
:104AA000F1EE666AB1EE477ACDED025A8DED036AFA
:104AB000CDED046A8DED057AC5ED0C5A85ED0D6AD4
:104AC000C5ED0E6A85ED0F7A03F044FEF0EE690A3B
:104AD000B0EE409AB0EE480A03F03CFE2046F0EEFD
:104AE000408A02A9B0EE490A03F06AFE009A214604
:104AF0001046B0EE680A03F063FE95F83031474C7B
:104B0000D5ED049A95ED059AD5ED068AD5F81CB039
:104B1000009A013303F00703152101FB083109EB6B
:104B20000110542185F8303101FB083344330AFB6E
:104B3000084A49F8237095F83131C0ED249A072BC3
:104B40009CBF013385F831319AF8643080ED259AA5
:104B5000C0ED268AC0F89CB0002B5BD054362644AA
:104B6000D2ED016A96ED010A96ED007AD2ED007A57
:104B700020EE260A07EE270A96ED027AD2ED027A97
:104B800007EE270A96ED037AD2ED037A07EE270A9D
:104B9000F7EE007AB5EEC00AF1EE10FA48BFB1EEBA
:104BA000400AB4EE670AF1EE10FAC8BFB0EE670A29
:104BB00015F0EAFDDFED1A7ADFED1A6AB4EEE78A46
:104BC000F1EE10FAC5BF30EE000ADFED177A9FED67
:104BD000177A20EE270A4FF4A873C8BF80EE087A30
:104BE00003FB0843D3ED147A37EE677A47EE267A53
:104BF0004FF4A87303FB08430122C3ED147AC3EDFD
:104C0000159A83ED169AC3ED178AC3F860B083F83E
:104C100064209CE6DFED057AEAE700BFA877002074
:104C2000BD378635CDCCCC3EE12E6542000000007C
:104C30002DE9F04F2DED088B97B005460593BF4B3E
:104C4000289C1B780293B0EE408A1746002B00F098
:104C50006F81002C00F03C83B94E4FF4A87202FB28
:104C6000006292F84C300293002B00F06181059BAA
:104C70003B4303BFDFEDB37A926C60EE277A3B468D
:104C800002BFFCEEE77A17EE903A9B184FF4A87239
:104C9000424306EB02080392C8F84830AA4BD3ED12
:104CA000000A03F057FD039B2033F3180693039B80
:104CB000069803F11001314403F082FDA34B93F8F1
:104CC00000B0A34BBBF1000F00F0458298F8319182
:104CD00093F800A0B9F1010F00F24C81BAF1000F76
:104CE00040F07082F7EE008ADFED9A0A944EB0EE43
:104CF000480A03F02FFD4FF4A87303FB0563D3EDBF
:104D00001B7A78EEE78A48EE807AF5EEC07AF1EE0B
:104D100010FAB0EE670A00F17382F7EE007AB4EE93
:104D2000670AF1EE10FAC8BFB0EE670A4FF4A87335
:104D3000B5EEC00A03FB0562F1EE10FA82ED1B0A24
:104D400003D9BAF1000F40F05E8203FB05631A6AD3
:104D500022605A6A62609A6AA260DB6AE3607E4BF4
:104D600093ED007A059BB5EEC07AF1EE10FAD8BF4C
:104D70009FED7A7A3B4340F05B82B5EEC08AF1EE5C
:104D800010FA00F19A82DFED767AB4EE678AF1EEDE
:104D900010FAC8BFB0EE678A4FF4A87303FB05632F
:104DA000D3ED1D8ADFED6F7A47EE088A4FF4A873C2
:104DB00003FB056367EE277A12AFF4EE678AF1EE24
:104DC00010FAC8BFF0EE678AF5EEC08AF1EE10FA6D
:104DD00048BFDFED658A04F1100CC3ED1D8A234640
:104DE000186859683A4603C2083363451746F7D135
:104DF0004FF4A87303FB056394ED00BA93F88C306D
:104E0000002B00F08380F5EEC08AF1EE10FA94EDED
:104E1000018AD4ED02AA94ED03AADFED549AB7EE0D
:104E2000009A45D9039F7C37374497ED010AD7EDA7
:104E3000007A28EE000A0BEE270AD7ED027A0AEE76
:104E4000A70AD7ED037A0AEE270AF7EE007AB5EE45
:104E5000C00AF1EE10FA48BFB1EE400AB4EE490ABA
:104E6000F1EE10FAC8BFB0EE670A15F08DFC30EE17
:104E7000000A20EE290AB4EEE80AF1EE10FA17D97A
:104E8000DFED3B7AF4EEE78AF1EE10FA40F118829A
:104E9000234607F1100257F8041B43F8041B9742FE
:104EA000F9D14FF4A87303FB056393F88C306BB30F
:104EB00094ED017AD4ED007A28EE070A0BEE270A6A
:104EC000D4ED027A0AEEA70AD4ED037A0AEE270A95
:104ED000B5EEC00AF1EE10FA01D5B1EE400AB4EE1B
:104EE000490AF7EE007AF1EE10FAC8BFB0EE670A91
:104EF00015F04AFC4FF4A87303FB0563D3ED1D7A4C
:104F000030EE000A40EE697AC3ED1D7A4FF4A873C3
:104F100003FB05632268DA676268C3F88020A26831
:104F2000C3F88420E268C3F88820012283F88C202B
:104F3000029817B0BDEC088BBDE8F08FD85802205E
:104F4000A87700200024744948260020AA280020C1
:104F5000D65802200AD7233C0019022000007A44C8
:104F60009A99193ECDCC4C3D00000000E02E6542E0
:104F7000BD378635059B3B433FF4B0AEBE4BD3ED0A
:104F8000007AF5EEC07AF1EE10FAD4BFD8F87000CE
:104F900017EE900AFCF766FE4FF4A87303FB056654
:104FA000012396F830610493CDE9000154236B434B
:104FB00006F108080793D8F1000202F0070208F092
:104FC000070358BF5342DAB20A92079A52FA83F3A0
:104FD0004433AA4A52F82300381AFCF721FEA2A350
:104FE000D3E90023FCF7C0FF08F1FF3802460B4667
:104FF000CDE90C23D8F1000202F0070208F0070304
:1050000058BF5342079A5FFA83FC52FA83F3443342
:105010009A4ACDF82CC052F823300893DDE90023DA
:10502000FDF7F4F890B1089BF81AFCF7F9FD8EA390
:10503000D3E90023FCF798FF02460B46CDE908238D
:10504000DDE90023FDF7ECF8002838D1049B01339B
:105050004B450493AFDB542303FB05634433DFF874
:105060001C8258F82300381AFCF7DAFD7EA3D3E936
:105070000023FCF779FFDDE90023FDF7DBF850B9E9
:105080000936A6EB0906734203F0070306F007068C
:1050900058BF5E42F6B2152303FB056608EB061304
:1050A00008EB0618D3F890300E93D8F894300F938D
:1050B000D8F898301093D8F89C3011933CE0DDE993
:1050C0000C23DDE90801FCF76DFC69A3D3E900239B
:1050D00080468946FDF7AEF898B3DDE90023DDE9A7
:1050E0000801FCF75FFC42464B46FCF73DFF0022FF
:1050F000002380468946FDF77FF810BB604B0022F5
:1051000040464946FDF796F800BB09234946152657
:10511000404616FB0536FDF797F80A990B9BDFF81A
:105120005CC13144334400EE100A0EAA0CEB0111AD
:105130000CEB031003F096FBBAF1000F10D1DA4626
:10514000D0E54FF000084FF00009DEE7DFF83091BE
:105150004FF00008D9E793F800A0BAF1000F2ED065
:10516000464A48494FF4A87303FB0523D1ED006A72
:1051700093ED147AB4EEE67AF1EE10FA4FF00001F6
:1051800023DBD3ED1A7A9FED406AF4EEC67AF1EE96
:1051900010FA03D577EE887AC3ED1A7A3B4BD3ED3C
:1051A000007A3B4BB4EEE77AF1EE10FA0FD500200F
:1051B00058554FF4A87303FB05239966DA46DFEDD3
:1051C000378A91E54FF0000BCAE79966E6E7B4EE3F
:1051D000E67AF1EE10FA03D55B5D002BEED0AEE778
:1051E0004FF4A87101FB052292ED1A7ADFED267AC1
:1051F000B4EEE77AF1EE10FAEEDB01225A559EE7A3
:105200009FED260A92E5F7EE007AB4EEE70AF1EE9A
:1052100010FA07DB0E9B23600F9B6360109BA3605B
:10522000119B9BE5069822460EA916F01BFC96E5FD
:105230004FF4A87303FB05639B6F8BBBB5EEC08A6D
:10524000F1EE10FA36D4DFED137AB4EE678AF1EEA0
:1052500010FAC8BFB0EE678A4FF4A87303FB05636A
:105260009F6799E5AFF300800000000080842E4125
:1052700095D626E80B2E113E04190220A8770020AF
:105280000000F03F442600200AD7A33C402600201F
:10529000D65702209A99193E002474490000000054
:1052A000FB1A07EE903A5FED046AF8EE677A87EE34
:1052B000A68AC8E71FED078ACEE71FED088A6BE5CF
:1052C00088EE800A22462146384603F0CBFAE8E50C
:1052D00002942DE6000000002DE9F04FD0E90063B4
:1052E00089B087680393838905930D46B368039952
:1052F0005B6806AA30469847002831DBDDE9064B9B
:10530000A7FB042307FB0B3804920498DFF8609096
:1053100015A3D3E900234146FDF744F9049B4FF060
:10532000FF3A9A4579EB0803074619D3A5FB0443D6
:1053300005FB0B3529460CA3D3E900232046FDF7D6
:1053400031F9A24579EB0505034609D38742B268D6
:1053500006D305990091146803993A463046A04750
:1053600009B0BDE8F08F00BF00CA9A3B0000000002
:10537000FFC99A3B000000002DE9F04F9FB0824624
:10538000039117461C460025387810B9284600F0CE
:10539000A6BD252809D00399D0470028C0F29F85D3
:1053A0007B1C01350593059FEEE71822002110A80C
:1053B00018F062FB7B78252B00F0BC800023791C61
:1053C00098469E469C4618460E4611F8012B2B2AFD
:1053D00000F0E38000F2DA80202A00F0E180232A46
:1053E00000F0E1802BB19DF8483043F040038DF888
:1053F0004830B8F1000F05D09DF8483043F0200345
:105400008DF84830BEF1000F05D09DF8483043F0CC
:1054100010038DF84830BCF1000F05D09DF84830DE
:1054200043F008038DF8483028B19DF8483043F028
:1054300004038DF848309DF8483003F044014429B6
:1054400003D16FF386138DF848309DF848300E96DF
:1054500043F080032A2A8DF8483040F0A9809DF857
:10546000493043F001038DF84930731C1A782E2A15
:105470009DF849200CBF0121002161F341028DF804
:1054800049200CD15A1C0E925A782A2A40F0A0804A
:105490009DF8492042F004028DF8492002331A7821
:1054A0006C2A00F0C18000F2A380682A00F0A98075
:1054B0006A2A00F0C2804C2A00F0C78013F8012B42
:1054C0000593782A8DF84B2000F209816D2A00F2AD
:1054D000C980692A00F20381572A00F2E280412A3A
:1054E00004D0A2F14503022B00F2F9809DF84A3066
:1054F00002F0DF020421A2F1410961F30203D9F1B4
:1055000000029DF849108DF84A3042EB090262F31F
:10551000C7110A068DF84910CBB200F11F8103F0C4
:105520007802182A40F009816FF3C6038DF84930DC
:105530000023F8E08DF84B30BB1C05939DF84930F3
:105540009DF84A20DE0702F0070040F1098154F877
:10555000041B0491002908DA9DF8481041F0040169
:105560008DF84810049949420491590740F100818F
:1055700054F8046B002E80F2FF809DF849306FF3E1
:1055800041038DF849304FF0FF36F5E02D2A0DD05C
:10559000302A7FF427AF012316E74FF0010C13E701
:1055A0004FF0010E10E74FF001080DE701200BE767
:1055B0000EA804F0F1FC0E9BB3423FF457AF9DF8E8
:1055C00048201390C00F60F341028DF848204DE74A
:1055D0000EA804F0E1FC9DF848301490C3F340029B
:1055E00042EAD07262F341038DF848300E9B56E7D1
:1055F000742A26D07A2A7FF461AF9DF849200621CB
:105600000CE05A78682A9DF8492006D1012161F3FF
:10561000C6028DF84920023350E7022161F3C60229
:105620008DF84920013349E75A786C2A9DF84920C2
:1056300001D10421EBE70321F0E79DF84920052182
:10564000ECE79DF849200721E8E7BDF8482022F45F
:10565000F04222F0020242F4804242F00202ADF82F
:105660004820DFE76E3AD3B201229A4040F28243EB
:105670001A429DF8493039D112F0240F61D1D10777
:105680002DD59DF84A2003F07803A3F140080321AB
:1056900061F30202D8F100038DF84A2043EB0803BE
:1056A00041E0A2F15801C9B2012000FA01F111F460
:1056B000624F7FF41BAF40F6010319429DF8493059
:1056C0001AD111F4043F0AD09DF84A2060F3020277
:1056D00003F07803402B8DF84A207FF429AF9DF822
:1056E000483043F001038DF8483021E79DF84A2007
:1056F000022161F30202EBE79DF84A10022003F059
:10570000780360F30201402B8DF84A1002BF9DF828
:10571000481041F001018DF84810632A7FF408AF6A
:10572000003B18BF01239DF84820C2F340010B4302
:1057300063F341028DF8482000E713F0380FCED113
:10574000F6E69DF84A20032113F0780F61F3020278
:105750008DF84A2014BF01230023E4E70123E2E788
:105760009DF948100029B4BF13994FF0FF31FBE6B3
:105770009E077FF508AF149E00230428CDE913335C
:105780009DF8493007D1990705D49DF949100029A2
:10579000ACBF06260D2602F00702012AC3F3C3039D
:1057A00032D1DA1E042A04D8DFE802F02045452071
:1057B00020002268012B4FEAE271CDE910211BD1B4
:1057C0009DF94020D117CDE9102104349DF84820DF
:1057D000069292074FD0059B03993A46504616F021
:1057E000D1FC0028C0F27B830544DCE554F8042B8F
:1057F000D117CDE91021E9E7022BE6D111B242F32E
:10580000C032CDE91012E0E7022A24D1DA1E042AC0
:1058100004D8DFE802F0181010181800012B54F813
:10582000042B4FF0000114D0022BCDE91021CDD173
:1058300092B21092CAE7073424F00704F4E8020198
:10584000CDE91001C2E754F8042B10920022119206
:10585000BCE7D2B2CDE7042A08D1073424F007040C
:10586000D4E900010834CDE91001AFE7032AADD136
:1058700054F8042BDDE79DF84B80B8F1780F3FF624
:1058800092ADB8F1570F5CD8B8F1250F00F0A480A5
:10589000B8F1240F7FF687ADB8F1410F04D0A8F11D
:1058A0004503022B3FF67FADDDE91023002BC0F24C
:1058B0004D810699080700F14C81C1F300194FEAA8
:1058C0004919C3F30A51C3F31303002940F044817B
:1058D00052EA030014BF4FF0010C4FF0000CD80245
:1058E00040EA5250D702CDE90C70B8F1460F47EAB2
:1058F000010740EAE17008BF4FF06608384300F046
:10590000B881BCF1000F10D01B0343EA12531703F8
:105910003A4618464FF0000C002880F25681BCF140
:10592000000F40F05981CDE90C730D9B43F000430B
:10593000A1F2FE3B0D930021DDE90C230F4605206B
:1059400060E1A8F15802202A3FF62DAD01A151F8DF
:1059500022F000BF1F5B0000A7530000A753000008
:10596000A7530000A7530000A7530000A75300004F
:10597000A7530000A7530000A9580000A753000038
:10598000CB5A0000DF5A0000A9580000A9580000B7
:10599000A9580000A7530000DF5A0000A7530000D9
:1059A000A7530000A7530000A7530000255B000089
:1059B0001F5B00006F5A0000A7530000A7530000B0
:1059C000E9590000A75300001F5B0000A753000027
:1059D000A75300001F5B000003994046D0470028F2
:1059E000C0F27D820135DEE4002E109F3BDB3146A4
:1059F000384618F069F8002F3FF4D5AC3E18F31B79
:105A00004FF000099DF84A2012F01001069100F0B5
:105A10005B82023312F04002DDF84C80089218BF1E
:105A2000149ACDF81C80434418BF9B18049A002A8E
:105A300040F36582D31A9DF8482004935007C2F3BF
:105A4000800B00F15C82510640F14C82B9F1000FED
:105A500007D003994846D0470028C0F2408201355C
:105A6000D94630223FE23846FCF7C0FDC6E7109821
:105A7000002800F024820DF17503009312AA17ABE1
:105A8000002104F09FFABDF84A3003F0EF0343F41D
:105A9000F04343F010030746ADF84A304FF00009D9
:105AA000002E0CDB9DF848200DF17503DB1B6FF316
:105AB00086129E428DF8482001D9F31A1393002FC5
:105AC0003FF471AC0DF175066DE0109B8DF85C3004
:105AD0004FF000090DF15D0617AF012392E7069B19
:105AE0001F0758BFC3F30019DDE9102354BF4FEA65
:105AF00049194FF02B09002B06DA524263EB43039E
:105B0000CDE910234FF02D090DF175030093DDE968
:105B1000100117AB12AA04F055FA0746C0E74FF080
:105B20000009F1E7109A072B3FF63DACDFE803F0E0
:105B30000C04060C08080C0C157034E4158032E4D3
:105B4000EB17C2E900532EE415602CE44FF02D0949
:105B5000B7E64FF02B09B4E640F2FF70814231D135
:105B600008F10108A2495FFA88F8134311F80810F8
:105B700001F003011ED101290BBF492369234E21E6
:105B80006E210CBF462266228DF85C309DF84830AD
:105B90008DF85D106FF386138DF85E208DF8483018
:105BA0000DF15F0617AFF31BB9F1000F3FF42AAFF9
:105BB000013327E7012915BF6E234E2361214121BF
:105BC0001A46E1E74FF0000C89E6921801F1FF3127
:105BD00040414FF0010C9FE6CDE90C20A5E65208AC
:105BE00042EAC3725B08B3F1333F59460BF1010B34
:105BF000F5D200FB03FCA2FB002301F1020B63447E
:105C0000013F01211BF1020FE9DB09B1CDE90C23B2
:105C1000BBF1000FDDE90C322EDCCBF10401A1F168
:105C200020000BF11C0B02FA0BFB22FA00F0CA4019
:105C3000CB40079208F0DF0243EA0B03472A43EA0E
:105C400000037DD1F91C01DBBE422BDAA8F102086A
:105C5000002E5FFA88F87CDD9DF84820920606F158
:105C6000FF3676D4B6F1000B18BF4FF0010B721C53
:105C700027E04FF0000B5EE6023342F100020CA871
:105C8000CDE90C3216F04FFADDE90C320BF1FF3B97
:105C90000137DB185241002A0BF1FF3BF9DACDE95D
:105CA0000C32B5E79DF848209006A6EB07064DD4C8
:105CB000B6F1000B18BF4FF0010BF2194FF0660858
:105CC0004AD4102AA8BF10229FED477B8DED0E7B92
:105CD00010200B90DDE90E01002A3FD1079A1B1816
:105CE00042EB0101B1F1805F47D2CDE90C31069B57
:105CF000B8F1660F03F0200240F0C180002F47DCAE
:105D000030238DF85C30002A74D1002E40F3BA8124
:105D10002E238DF85D3087B17B42B342A8BF334656
:105D20009DF84A201393002BA6EB0306D4BF002353
:105D3000012363F345128DF84A200DF15E0340E024
:105D4000B8F1660F4FF0000BB7D090E74FF0000BA3
:105D5000B3E74FF0000B8AE70022B5E7400840EABE
:105D6000C1704908CDE90E010EA8CDE9082316F04F
:105D7000DAF9089A099B013AACE75B0843EAC17378
:105D80000CA84908CDE90C31013716F0CCF9AEE783
:105D900017AB0B9900290BDD0BA90CA8CDE9063236
:105DA00016F0D9F9069B079A03F8010B013FF0D1D1
:105DB0001397AAB9002E40F363812E2103F8011B2B
:105DC0000027002E1FDD0B9A002A1CDD0BA90CA852
:105DD000069316F0C0F9069B013E03F8010BF0E7AD
:105DE0002E2203F8012BEBE7000000000000000862
:105DF000032402002E238DF85D30002F9DD0002E4D
:105E00008ADC0DF15E03BBF1000F4CD114961E46E7
:105E100008F0DF03452B21D1002FBABF7F422D238D
:105E20002B23632FC8BF64227370C2BFB7FBF2F38A
:105E300003F1300102FB13774FF00A0286F800806D
:105E4000CABFB17002360336B7FBF2F303F130017B
:105E500002FB13733033317073700236139B002BC7
:105E60002BDC149B002BD4BF002301239DF84A2078
:105E700063F3861200238DF84A20337092E60BA953
:105E80000CA8069216F067F9069A8DF85C00302887
:105E900018BF07F1FF3712B9002E40F3F3802E230D
:105EA0008DF85D3049E71E46013B16F8012C302A7B
:105EB000F9D02E2A08BF1E46AAE70123D6E7734E63
:105EC0008146771F05239DE5110748BF0133A1E5F2
:105ED000104609920399D0470028099A05DA1FB0A5
:105EE000BDE8F08F2022DDF810B0594600290BF1F3
:105EF000FF3BEDDC049BCDF810B02B445D1AB9F1EB
:105F0000000F05D003994846D0470028E7DB01354C
:105F1000089B002B79D09DF94930002B29DBDFF855
:105F200070913B46187819F8002052079B4603F100
:105F300001033FD49DF84A30EF1B98065F4407D415
:105F40004246002A08F1FF383BDC079B3B449F1A7E
:105F50009BF800002E280AD10399D0470028BEDB09
:105F6000B8F1000F07F1010731DC0BF1010B5D46C1
:105F700038E0B94699F800007028C84609F10109CF
:105F800013D1EF1B149D47443D44EB1B002B34DC25
:105F9000039933464246504616F0F4F800289EDB3B
:105FA0003844049E0546064465E00399D04700281E
:105FB000E0DA94E706930399D0470028069BB1DA0C
:105FC0008DE703993020D0470028B9DA87E7039995
:105FD0003020D04708F1FF38C0E70399D0470028A8
:105FE000FFF67DAF287819F800305907A84605F16B
:105FF0000105F2D4A7EB0B07C4E703993020D04783
:106000000028FFF66CAF0137BFE79DF84A30DA068B
:1060100001D41B0706D503993020D0470028FFF68E
:106020005EAF0135069B3BB103999DF84B00D0470D
:106030000028FFF654AF0135A84406E0039930204C
:10604000D0470028FFF64BAF0135A8EB0503002B26
:10605000F4DC039933463A46504616F093F800288C
:10606000FFF63DAF28449CE703992020D047002845
:10607000FFF635AF0135731B002BF5DCFFF793B945
:106080001746C0E60DF15D03BDE600BF0C0A020035
:10609000042402002DE9F047464D474F002605F144
:1060A000050844480DF08CFF10F13D0F04466FD0F9
:1060B00000285AD12B78082B06F101061AD0102B94
:1060C000EFD13E4B95F8069093F800A0D1452DD323
:1060D000082005F0BDFA48B1394BC0F81CA0C0E952
:1060E00005390423037444748474C47400234FF486
:1060F000025217E0D8F800303B60D8F804307B60DB
:106100007B78013B012BCCD9062005F0A1FA30B1F8
:106110002C4B43610223037444748474C4740023BD
:106120004FF48652284916F0F1FCBAE7274A12F8D4
:1061300009300F2B03D8013302F80930B1E76B792E
:10614000DF2BAED8224B2A791A70224BA978224C29
:1061500019702248D4F8049002F086F96068A0EB28
:106160000900800901F0E8F99BE7082005F070FAC2
:1061700040B11B4BC0E9053403230374002343746F
:106180008374C374104900234FF4C25216F0BEFC4E
:10619000144A1368012E03F10103136081BF124AF0
:1061A000136801331360114B1A68964288BF1E6052
:1061B000BDE8F0879938022091380220C1380220CA
:1061C00057EE010044EE01002CE40100913702205B
:1061D000C0380220BF380220001000E09E380220A4
:1061E0007DEE010070D401206CD4012068D4012020
:1061F00070B5062005F02CFA38B1214B436102231B
:106200000374002343748374C3741E4C1E4900231B
:106210004FF4865216F07AFC23786BB300250620E3
:10622000257005F015FA30B1184B43610223037451
:1062300045748574C574002313494FF4865216F0D3
:1062400065FC0A2015F0C9FB23789BB1062005F0F8
:10625000FFF938B10E4B43610223037400234374EA
:106260008374C374BDE87040074900234FF486521D
:1062700016F04CBC0DF09EFC0023237070BD00BFD7
:106280009FEE0100803702202CE40100BAEE0100ED
:10629000CDEE010010B50C484FF48072002117F0CC
:1062A000EBFB00244FF47A7015F097FB064A0023AD
:1062B00012F8011B01330F2998BF02F8014CB3F506
:1062C000807FF5D1EEE700BF9137022030B5002086
:1062D00085B00BF043FB0446A8B9062005F0B8F9D9
:1062E00030B12C4B43610223037444748474C4742E
:1062F000294900234FF4825216F008FC6FF0050480
:10630000204605B030BD002501236946019503955F
:10631000029304F0B9FA041E12DA082005F098F985
:1063200038B11E4B4574C0E90534032303748574EA
:10633000C574194900234FF4C25216F0E7FBDFE79A
:1063400042F21174029D15F0030518D0013CF9D1F9
:10635000082005F07DF948B1114B43616FF00A0345
:1063600083610323037444748474C4740A4900234E
:106370004FF4C45216F0CAFB6FF00A04C0E7039C46
:10638000002CBDD0082005F063F90028D1D0054BC2
:10639000C8E700BFE7EE01002CE4010007EF0100B1
:1063A0003FEF010020EF01002DE9F0413D4E86B0A6
:1063B000337800AF80468BB1062005F049F938B13B
:1063C000394B436102230374002343748374C37401
:1063D000364900234FF4845216F098FB344D0FCD0C
:1063E0003C1D0FC42B682360324BB8F1000F32D034
:1063F000BB6000233B737B82012308223B752E4B3D
:10640000BA7340F201126C4688B0FA826A462B4990
:10641000C2E905134FF400739383294B42F8103FF0
:10642000224800234FF4E65105F0B8FA381DA5467E
:106430000DF0F8FB0446B8B1082005F009F938BBA7
:106440001A4900234FF4C25216F060FB01210220CA
:1064500002F0B0FE17E00122BB600823BB737A7123
:10646000184B87F80C80CCE764200DF0FBFE164833
:106470000DF09CFE15480DF0B3FE154808210DF0F7
:10648000C9FE0123337020461837BD46BDE8F081B0
:10649000104BC0E905340323037400234374837451
:1064A000C374CDE7803702206AEF01002CE40100BD
:1064B00020E50100CFB9010068EF010082EF010083
:1064C00003000001221502008D37022089370220C7
:1064D000813702209DEF0100074B08491A68084BDD
:1064E0001A60084B1A68084B1A60084A0B68136058
:1064F0004B685360704700BFBBEF0100C0EF010065
:106500008D370220C9EF0100893702208137022030
:1065100010B5194B93E8030086B04FF080530090FC
:10652000ADF8041093F8A9400023CDE90433CDE978
:1065300002000DF10F02E1180133082B02F8011FD0
:10654000F9D102A9102211F8013B1BB1552B01D042
:10655000AA2B02D1083301F8013C013AF3D1074AD2
:10656000029B1360064A136004AB03CB054A10601C
:10657000516006B010BD00BFA40000108D3702208E
:1065800089370220813702202DE9FF47DFF83C815F
:10659000DFF8449198F8003006460D4686468A4654
:1065A0001746002A77D0CC461C460022934264DC72
:1065B000A34272D10A2005F04BF850B1414BC0E91B
:1065C0000865C0E90534062303740023437483740B
:1065D000C3743D4900234FF4435216F097FA09EB78
:1065E000C402E01C0823002180B249F834605560E1
:1065F00002F0E2FE98F80030344A013388F80030A7
:1066000001230021184602F0D7FE9FB3062202A9FB
:106610000720CDE900650296ADF80C5002F09EFF10
:106620004FF08053061E4FF0080008BF0826D3F82D
:10663000A470D3F8A85005F00BF8A8B1E217244BCA
:106640004361120242EA14622B04240243EA174314
:1066500044EA0744134334430022C0E906430423B9
:10666000037442748274C274174900234FF40352B6
:1066700016F04CFA04B0BDE8F0875EEA0A0106D0D5
:10668000DCE90001514508BF704508BF14460132DE
:106690000CF1080C8AE71C468CE7082004F0D8FFB0
:1066A00040B10C4BC0E90534032303740023437449
:1066B0008374C374044900234FF4C65216F026FABB
:1066C000A4E700BFCEEF01002CE40100C138022096
:1066D0001AF00100F9EF0100A04D00202DE9F04172
:1066E0001B4D2C7824B301231846013C2A46002177
:1066F0002C7002F061FE2C78164B0A2003EBC403C9
:10670000D3E9006704F0A4FF50B1134BC0E9086758
:10671000C0E9053406230374002343748374C374EF
:1067200000234FF44352BDE8F0410C4916F0EEB996
:10673000062004F08DFF30B1094B4361022303743E
:1067400044748474C47400234FF48452EBE700BF94
:10675000C1380220A04D002037F001002CE40100D8
:1067600064F001002DE9F84F062004F071FF38B104
:10677000544B436102230374002343748374C37432
:1067800000234FF486525049DFF8588116F0BEF9C5
:106790000020FFF7A1FE0024FFF706FE0DF060FCCD
:1067A0004FF0805388F80340D3F8A400474AC8F854
:1067B00007009288A8F80B200820D3F8A460D3F82B
:1067C000A85004F045FF48B1ADB2414B4361C0E968
:1067D00006650423037444748474C47400233A4922
:1067E000DFF804913B4DDFF804A14FF4035216F09B
:1067F0008DF90221032002F001FB012389F800300A
:10680000FF236B7099F800303BB90221012002F0A0
:10681000F5FABDE8F84FFFF7EBBC2F4B187818B925
:10682000FFF7C2FD0DF01CFC6B78022B36D0FF2B5E
:1068300034D00DF091FC2C686F689AF800C0274E98
:10684000240C44EA0744E3463F0C002262452BDB5C
:1068500006222349072002F081FE2A78061E08BF7F
:106860000826B2420FD154EA07020CD09AF8002051
:106870005A4508D1204639460022FFF785FE0021FF
:10688000082002F0BBFA2A78164888F806B096422B
:1068900018BF002288F805200DF0F8FAFF23012028
:1068A0006B7015F09AF8ADE754EA070107D0D6E906
:1068B00000018F4208BF844208BF1FFA82FB0132E9
:1068C0000836C3E779F001002CE40100A4000010B1
:1068D00081F001009138022080370220A04D002075
:1068E00093380220842800207F370220C1380220FC
:1068F00008B5FFF77DFC034B00221A70024BFF2204
:106900005A7008BD7E37022091380220014B0022C8
:106910001A7070477F37022010B50E4A00240123F9
:1069200018462146147002F047FD062004F090FE40
:1069300030B1094B43610223037444748474C474FA
:10694000064900234FF4865216F0E0F8BDE81040E7
:10695000FFF7CEBFC138022099F001002CE40100FE
:1069600008B5FFF7D5FD024B01221A7008BD00BF24
:106970007E370220F8B5254DFFF7A8FC01222946F5
:10698000104602F029FD2B7813B1214B01221A7019
:10699000204E00242F78A7422EDC082004F058FE59
:1069A00058B11D4BC0E905374FF48073C361042310
:1069B0000374002343748374C374154C1749002374
:1069C0004FF4035216F0A2F8237833B1FFF7C8FF53
:1069D0000020FFF7E9FC0DF043FB257845B9FFF7F0
:1069E000C1FEFFF7BDFF2846FFF7DEFC0DF038FBC8
:1069F000642014F0F2FFF0E7E01C3146082280B278
:106A000002F0EAFC01340836C4E700BFC1380220B6
:106A10007E370220A04D0020A3F001002CE40100ED
:106A200008B52DED088BD1ED00AA90ED02AA90EDEE
:106A300000BA90ED018AD1ED029AD1ED01BA90ED44
:106A4000039AD1ED038A2AEE8A0A1BEE290A2AEE5E
:106A5000887A1BEE2B7A0BEEC90A6AEE897A0AEE67
:106A6000687A5BEE287A08EE280A09EE897A48EE01
:106A7000697A20EE000A4BEE8A7A07EE070A07EEE3
:106A8000A70A13F027FF68EE2B0A4BEE2A0A4AEEFC
:106A9000290A49EE280AF0EEE00A17F008FABDECE0
:106AA000088B30EE000ADFED027A20EE270A08BDDF
:106AB000E12E654210B590ED016A91ED017A90EDFD
:106AC000005AD0ED027AD1ED026AD0ED034AD1ED41
:106AD000035A2DED068B91ED008A66EE079A45EE7E
:106AE000089A144668EE278A28EE069A55EE268AFA
:106AF00047EEA69A15EE079A47EE648A28EE248A96
:106B000044EEA59A07EEE59A15EE258A46EE258A0B
:106B100006EEA49A06EE668AF5EEC09AF1EE10FA39
:106B200007EE278A44BFF1EE688AB1EE499A28EE53
:106B3000A80A09EE090A48BFB1EE488A08EE080A19
:106B400048BFF1EE699A13F0C5FEDFED137AB4EE9B
:106B5000E70AF1EE10FAB0EE40AA1AD4F0EE690A94
:106B600017F0A5F930EE000AC0EE0A7A9FED0B7A15
:106B700067EE877A29EE279A68EEA78A28EE278A99
:106B800084ED009AC4ED018A84ED028ABDEC068B87
:106B900010BDF0EE007AE9E795BFD633E12E6542ED
:106BA0002DE9F04F2DED0A8B95B014F026FF1C4B0C
:106BB0001D1F543306460E9300214FF4203011F070
:106BC00093FC14F01AFF174B04901C78002C35D15D
:106BD000154A01261E70D2F8FC3043F08073C2F8CB
:106BE000FC30124B5C601A6832431A60104B0A206A
:106BF0001F7804F02DFD58B10E4BC661C0E9053475
:106C00000823C0E908370623037444748474C474E9
:106C1000094900234FF4435215F078FF049ECBE757
:106C200094340020BE38022000ED00E0001000E0A7
:106C3000C138022047FF01001CE40100BD4C049B49
:106C4000D4E900799E1B012E38BF0126B9F1000F4F
:106C500000F02782A368B3FBF9F8E36800930C20E7
:106C6000D4E904BA04F0F4FCA8B1B34A009B426131
:106C70004FF47A72C0E9093B57430823B7FBF6F794
:106C8000C0E9067903740023C0F82080C0F82CA066
:106C900043748374C374A949002344F2C00215F0FD
:106CA00035FFE3690093D4E908B30193A36D029320
:106CB000E36D0393236E0593636E0693A36EA16B3E
:106CC000E26B07931820E36AD4F81880A76AD4F817
:106CD00030A0D4F88C900A91646B0992089304F068
:106CE000B7FC00282DD0964B0A99099A01624FF4FF
:106CF0007A7CC0E905380CFB08F8B8FBF6F3C361F1
:106D0000009B4262C0E90A3B019BC0E90C37029B31
:106D1000C363039B0364059B4364069B8364079BD7
:106D2000C364089BC0E9143A142303740023C0E928
:106D300016940CFB07F743748374B7FBF6F787636D
:106D4000C3744AF2C0027D49002315F0DFFE794A80
:106D5000976C17B1D36CB3FBF7F7946FD2E9143B80
:106D6000002C00F0A081D66FB6FBF4F60E20D2E91D
:106D700020A9D2F88880009304F06AFC88B1009BB7
:106D8000704AC0F83480C0E9073BC0E905270A23F0
:106D9000C0E9096AC0E90B49037400234374837492
:106DA000C3740023654945F2C00215F0AFFE664882
:106DB0000378002B00F0A980C37A0093037B019332
:106DC000437B0293837B0393C37B0593037C0693EE
:106DD000437C4168827A0793837C90ED0E8A067A21
:106DE000447A90ED06CAD0ED07BA90ED08BAD0ED1E
:106DF00009AA90ED0AAAD0ED0B9A90ED0C9AD0ED6D
:106E00000D8A90F813B00A910992089390F814A093
:106E100090F8159090F81680C77D242004F018FC97
:106E2000002868D0FDEEC87A484BC0ED077AF8EE2E
:106E3000E77A436138EE678ADFED457A009B836528
:106E4000B0EEC88A28EE278ADFED427A019BC3653F
:106E50002CEE277A029B0366BDEEC77A039B80ED7A
:106E60000B7A2BEEA77A4366BDEEC77A059B80EDC1
:106E70000C7A2BEE277A8366BDEEC77A069B80EDEF
:106E80000D7A2AEEA77ABDEEC88ABDEEC77A0A99B6
:106E900080ED0E7A2AEE277A099AC366BDEEC77A8C
:106EA000079B80ED0F7A29EEA77AC0E90964BDEE51
:106EB000C77AC0E9136480ED107A29EE277A68EE6C
:106EC000A77ABDEEC77AFDEEE77A816180ED088A88
:106ED00080ED117AC0ED127A42650367089BC0E924
:106EE0001FA9C0E91D3BC0E921871F2303740023AC
:106EF00043748374C37400234FF680020F4915F066
:106F000005FE114B00221A705A60134B0024CDE984
:106F10001244D3F8E00012A916F0DEFC11F084FB55
:106F200013A916F0D9FC0A20DDE9127604F090FBD3
:106F300014E000BF90340020B5FF01001CE4010004
:106F400002000200D100020074D4012055010200A9
:106F50000000C84200007A4468D2012058B1534B67
:106F60004474C0E905374FF40063C0E907360523D0
:106F700003748474C4744FF0000B4D494D4C0023CE
:106F80004FF4235215F0C2FDCDE900BBDA464A4B5F
:106F90001B78534547DDD4F83C310293D4F838319F
:106FA0000393029BD4F83071042B00F28B80009B7A
:106FB000039A13440093019B3B4401930BF1010B93
:106FC0000AF1010A00230022BAF1100FC4E951337B
:106FD000C4E94F33C4E95333C4E95733C4E94B33ED
:106FE000C4E92033C4E92533C4E93C33C4F838315B
:106FF00084F85431C4F85831C4F87831C4F83431C5
:10700000C4F88820C4F88C20C4F89020C4F89C30C0
:10701000C4F8EC30C4F8FC20C4F8F820C4F80031FF
:1070200004F5C474B3D1BBF1000F16D00A2004F0EC
:107030000FFB60B1214BC0E9053B009BC361019B85
:10704000036205230374002343748374C3741849D3
:1070500000234FF4235215F059FD0024184B0E98CD
:107060009C6014222146C3E90044C5E90C44C5E9EB
:107070000444C5E90A44C5E90844C5E90644C5E92C
:107080000E44C5E91244C5E914442C6016F0F4FC22
:10709000C5E91E44C5E92144C5F88040C5F88C40C7
:1070A000BCE5C846D9E5264660E600BF36020200C8
:1070B0001CE4010020350020C138022077040200C2
:1070C00094340020D4F82C61D4F8EC80BE191EBF93
:1070D00064237B43B3FBF6F6B8F1000F00F0768132
:1070E000D4F8F03064225343B3FBF8F1D4F83431D0
:1070F0000593D4F840310693D4E951320792D4E98C
:107100002620D4F850910890D4F8840094ED229A67
:10711000D4ED238AD4ED249A0990B9F1000F03D05D
:10712000D4F84C01B0FBF9F90F9394F854310A9359
:10713000D4F800310B93D4F8F4300C932020D4F819
:10714000583194ED3E8A0D93CDE9102104F080FA78
:10715000002865D09E4B109A11994662FDEEC96ACF
:10716000BDEEE87AC0E9053A039BC0ED126AC0E9BA
:107170000737F8EEE66A059B80ED147AB8EEC77A19
:107180008362029BC36239EE669A069BDFED916AC9
:10719000036378EEC78A0F9B4363B0EEC99A079BDF
:1071A0008363F0EEE88A4FF47A7329EE269AB2FBF5
:1071B000F3F268EEA68AC263089A0264099A4264EE
:1071C000FDEEC87A0A9AC0F85C90BDEEC99AFDEE51
:1071D000E88AFDEEE99AC0E9182880ED139AC0ED1F
:1071E000158AC0ED169A8166C0ED1D7AF8EEE77A31
:1071F0000B9AB2FBF3F338EE678AC366B0EEC88A27
:107200000C9B036728EE268A0D9BC367BDEEC88AD8
:107210001C230374002380ED1E8A43748374C3749B
:1072200000236D494EF2C00215F070FC94F8C8308E
:10723000002B00F08D80D4F85C3100265A1C022B04
:1072400084F8C860C4F85C2100F2828094F8B4101D
:1072500094F8B52094ED28AAD4ED299A94ED2A9AB1
:10726000D4ED2B8A94ED2C8A94F8B69094F8B780DC
:1072700094F8B87003911620029204F0E9F90028FE
:1072800060D0FDEECA7AFDEEE95ABDEEC96AFDEEA8
:10729000E86ABDEEC87AC0ED077AC0ED095AF8EE8B
:1072A000E77AF8EEE55A80ED0B6AC0ED0D6AB8EEAC
:1072B000C66AF8EEE66A80ED0F7AB8EEC77A3AEE63
:1072C00067AA79EEE59A39EE469A78EEE68A38EEC4
:1072D000478ADFED407A029A404B03994164B0EE51
:1072E000CAAAF0EEE99AB0EEC99AF0EEE88AB0EEDA
:1072F000C88A2AEE27AA69EEA79A29EE279A68EE8D
:10730000A78A28EE278ABDEECAAAFDEEE99ABDEE4D
:10731000C99AFDEEE88ABDEEC88AC0E91229C0E923
:107320001487C0E9053A122380ED08AAC0ED0A9A35
:1073300080ED0C9AC0ED0E8A80ED108A03744674BD
:107340008674C6742449002349F2800215F0DEFBDE
:1073500094F81031002B3FF433AED4F8603100269E
:107360005A1C022B84F81061C4F860213FF628AE45
:107370000C20D4E9468994ED458AD4F8807104F054
:1073800067F9E0B1FDEEC87A154BC0ED077AF8EE6B
:10739000E77AC0E9099838EE678ADFED0E7AC762AE
:1073A000B0EEC88A28EE278AC0E9053ABDEEC88A41
:1073B000082380ED088A037446748674C6740649EF
:1073C00000234FF4814215F0A1FBF9E541468DE61B
:1073D000720202000000C8421CE40100A80302007F
:1073E00010040200F8B50E46044611463046154614
:1073F000FFF716FBF1EE047AB4EEE70AF1EE10FAAD
:107400002AD4164F7B6801337B60234603F1100CAE
:1074100007F1080418685968224603C20833634517
:107420001446F7D10E4C3346103618685968224678
:1074300003C20833B3421446F7D10A4C2A4610352A
:1074400010685168234603C30832AA421C46F7D18C
:10745000012387ED0E0A3B70F8BD00BF74D40120F4
:107460008CD401209CD40120F8B52F4A13680F2832
:1074700003F101030446136047D814F0BEFA064630
:107480002A484FF4C47303FB04030F46D3F83811A2
:107490000131C3F8381126490D7893F82911C3E951
:1074A0005A6705F00305A1B193F82811691A01F094
:1074B000030102292AD1D3F830110131C3F8301168
:1074C0004FF4C47303FB0403D3F82C110131C3F848
:1074D0002C114FF4C47303FB0400012380F82931FD
:1074E000144BD0F84C211B7880F828511A44C0F86E
:1074F0004C21D0F850210132C0F8502190F854218D
:10750000D9B29A4238BF80F85411F8BD032903D18B
:10751000D3F830110231D1E70029D1D1D3F8341199
:107520000131C3F83411CBE790340020203500201E
:10753000C0380220BF3802200B4B5A6801325A6013
:107540009A6802449A60DA68904288BFD860C82876
:1075500009D91A69B0F5FA7F02F101021A6182BFF6
:107560005A6901325A617047903400202DE9F04F7A
:107570002DED028B93B00F2806468846059200F247
:10758000A181DFF8B8934FF4C47202FB0093B8F105
:10759000010FD3F83C1101F10101C3F83C1103D0F4
:1075A000B8F1040F40F0938102FB0693D3F8402119
:1075B0000132C3F8402114F020FA4FF4C47474432C
:1075C00009EB0407C7E95C0116F0F8F9D84AA0FBFB
:1075D000025302FB013115F5804541F10001EB0B2F
:1075E00043EA41430193CB0B049304F140034B4422
:1075F000029397F87D30002B60D005990298FFF731
:107600000FFAD7E91C01019BD7ED237A181A049BC6
:10761000B4EEE70A63EB0101F1EE10FAC8BF87EDA3
:10762000230A012871F10003B0EE408A46DB4FF4D3
:10763000C47707FB06970029D7F89830D4BF0246D5
:107640004FF0FF329A424AF6C87388BFC7F89820B5
:107650009A4208D94FF4C47202FB0692D2F89C30C9
:107660000133C2F89C30C82871F1000326DBFAF719
:107670000BFFDFEDB07A07EE100A27EE277A4FF402
:10768000C473C8EE077A03FB069393ED247AF4EEF5
:10769000C77A9FEDA97AF1EE10FAF4EEC77AC8BF67
:1076A000C3ED247AF1EE10FA08DD4FF4C47303FB46
:1076B0000693D3F894200132C3F8942004F17803A0
:1076C00009EB040B4B4404F1500ECE445F46039388
:1076D0009946DC464FF0000A65460CF1100C9CE818
:1076E0000F0085E80F00DEE90223EEE802230AF12D
:1076F000010A99F8013009F8013BBAF1040FEBD106
:10770000059BDDF808C003F1100E18685968624641
:1077100003C2083373459446F7D1DFF82092019AEB
:107720004FF4C47A0AFB06930AFB069A1A67049A76
:107730005A6793F87D2083F87C80042A9CBF01322D
:1077400083F87D20DAF880300133CAF880309AF867
:107750007D30042B40F2B68004F12008C84406AA0C
:1077600059464046FFF7A6F904F1100109AA494419
:107770004046FFF79FF904F130010CAA4944404606
:10778000FFF798F90FAA02996C4D4046FFF792F95E
:10779000DDED097A9DED067A9DED070A9DED0B6AF8
:1077A000F1EE006A07EEE67ADDED0C7A07EEE67A96
:1077B000DDED0F7A37EE277ADDED0A7A07EEE60A7D
:1077C000DDED0D7A07EEE60ADDED107A30EE270AE0
:1077D000DDED087A46EE667A9DED0E6A46EE667A33
:1077E00020EE000ADDED116A07EE070A77EEA67AB1
:1077F00007EEA70A13F06EF8F1EE087A02995846E0
:1078000080EE278AFFF70CF9DAE91401019B181AB8
:10781000049B63EB0101F0EE408AFAF735FE9FED21
:10782000457ADFED476A07EE900A67EE877A4FF4F4
:10783000C473F4EEC77AF1EE10FACCBF88EEA77AE3
:107840009FED407AF0EE007A47EE267AB4EEE78AB2
:10785000F1EE10FA78DD03FB0653D3ED227AB4EE95
:10786000E78AF1EE10FAC8BF83ED228A4FF4C473A1
:1078700003FB065393F87E60002E3AD1D3F88420A0
:1078800083ED288A01210A4483F87E1083F8C8100A
:10789000D3E91801C3E9300104F1A408C3F8842036
:1078A000A844384610373946FFF7BAF80136042E97
:1078B000A8EC010AF5D1039AB43492E803002B191D
:1078C0002851197113B0BDEC028BBDE8F08FB8F1EF
:1078D000020F05D1D3F844210132C3F844216AE6EE
:1078E000B8F1070F02BFD3F848210132C3F848218D
:1078F00061E6D3ED287AB4EEE78AF1EE10FAE1DD25
:10790000D3E91801C3E9300104F1A40683ED288A04
:107910002E444FF00008384610373946FFF780F8FC
:1079200008F10108B8F1040FA6EC010AF3D1C2E78F
:1079300040420F00BD3786350000FA442035002054
:107940000AD7A33B0000000003FB0655002385F87F
:107950007E30B7E72DE9F04F2DED028B0F2885B073
:107960000746914600F2AE80794DDFED7A7A4FF40A
:10797000C47606FB005220EE270AD2F87831D2F8FE
:107980005811FCEEC07A0133C2F8783117EE903A04
:107990004643994206F1D00A38BFC2F85831AA448A
:1079A00016F00CF86C4B2E44A0FB034803FB018837
:1079B00014F5804496F8E83048F10008E40B44EAF6
:1079C00048444FEAD838002B53D049465046FFF779
:1079D00027F8D6E93832D6ED3E7AD6F8EC00B4EB8B
:1079E000030BB4EEE70A68EB0201F1EE10FA00F1C6
:1079F0000100C8BF86ED3E0ABBF1C80FC6F8EC0017
:107A000071F10000B0EE408A1DDB5846CDE902322C
:107A10000191FAF739FD9FED517A039A07EE900A2A
:107A200067EE877A4FF4C47088EE277A00FB075020
:107A3000DDE90113D0ED3F7AB4EEE77AF1EE10FA0A
:107A4000C8BF80ED3F7ADFED467AB4EEE78AF1EE0B
:107A500010FA4FF4C4703AD500FB0750D0F8F0107C
:107A60000131C0F8F010D0E94261314301D1C0E9E1
:107A7000423209F11002D9F80000D9F80410534637
:107A800003C309F1080991459A46F4D14FF4C4762D
:107A900006FB0756012386F8E83096F81031C6E950
:107AA00038487BB113F0A9FFD6E95C3253EA0204EF
:107AB0004AD0C01A61EB02014FF4C47303FB0755AF
:107AC000C5E9600105B0BDEC028BBDE8F08F00FB9D
:107AD0000752D2E9426356EA030C33D0A61B68EB87
:107AE0000303002BD2F80031B8BF00269E4288BFA6
:107AF000C2F8006100FB075000220023C0E94223C6
:107B0000F0EE007AB4EEE78AF1EE10FAB1DD4FF450
:107B1000C47202FB07520029D2F8F43082ED458A84
:107B200003F10103C2F8F4304FF0010382F8103181
:107B3000ACBF5B460023C2E94734C2F81861C2F803
:107B4000248196E70026DBE74FF0FF300146B3E7DC
:107B50002035002000007A4440420F00BD378635B2
:107B60006F12033B38B515F029FF174CA0FB043208
:107B700004FB0121154A906901309061D2E910049B
:107B800013F5804341F10001DB0B50EA040543EAA1
:107B900041434FEAD13113D0181A61EB0404012894
:107BA00074F100050CDB956BA84240F2D17588BFDB
:107BB0009063A84274F10004A2BFD06B0130D0637F
:107BC000C2E9103138BD00BF40420F0090340020A0
:107BD000074B18B9DA690132DA61704701280BBF27
:107BE0001A6A5A6A013201320CBF1A625A6270472D
:107BF0009034002070B5194B9E6A01369E629E6CCF
:107C0000DDE9044501369E64DE6C2644DE641E6DAB
:107C1000B44288BF1C65B4F5617F82BF5C6D0134DE
:107C20005C6581421EBFD96A0131D9620428C2BF96
:107C3000196B01311963D3F88C10814238BFC3F836
:107C40008C0015B1596B01315963042A9FBF16325C
:107C500053F82210013143F8221070BD90340020F7
:107C600038B515F0ABFE1E4CA0FB043204FB01211D
:107C70001C4AD2E91C0413F5804341F10001DB0BDF
:107C800050EA040543EA41434FEAD13125D0181A9E
:107C900061EB0404012874F100041EDB946F0134CD
:107CA0009467D46F0444D467D2F88040A04288BF60
:107CB000C2F88000B0F5FA6F0FD9B0F5FA5FD2F8CC
:107CC000844088BFD2F8880004F1010488BF0130E5
:107CD000C2F8844088BFC2F88800C2E91C3138BDB0
:107CE00040420F009034002001480FF0C5BB00BF98
:107CF000F018022008B5054804F05CFF0449054867
:107D00000FF048FB044B01221A7008BD6982000085
:107D100041360000F0180220C23F02202DE9F04158
:107D20002DED088B017807298EB0044600F24081C2
:107D30006FF096070F4117F0010740F0398106AE4A
:107D400000964078FCF774FF002800F031819DED2B
:107D5000076ADDED067ADDED086A9DED097A9FED93
:107D6000CB5A66EE065A47EEA75A46EEA65A47EE9B
:107D7000075AF4EEC55AF1EE10FA00F119819FEDA1
:107D8000C45AF4EEC55AF1EE10FA00F311812378CB
:107D900094F801E0CDED0A7A022B8DED0B6ACDED62
:107DA0000C6A8DED0D7A0AAD00F00781072B00F00B
:107DB0000481DFF80883B74F18F80E20B64B002A6D
:107DC00040F00C8103EB0E1C95E80F008CE80F00CF
:107DD00096E80F0007EB0E1787E80F00012308F85D
:107DE0000E302378012B02D0042B40F06D819FEDE3
:107DF000AB5ADFEDAB5A26EE056AB4EEE56AF1EE5A
:107E000010FA00F32F81DFEDA74AB4EEE46AF1EE39
:107E100010FA00F12A81BDEEC66A16EE103A1BB2C6
:107E200066EE856A6380F4EEE56AF1EE10FA00F31F
:107E30001E819FED9C6AF4EEC66AF1EE10FA00F125
:107E40001981FDEEE66A16EE903A1BB227EE057A2E
:107E5000A380B4EEE57AF1EE10FA00F30D81DFEDC8
:107E6000916AB4EEE67AF1EE10FA00F10881BDEE07
:107E7000C77A17EE103A1BB267EE857AE380F4EE0C
:107E8000E57AF1EE10FA00F3FC809FED867AF4EECD
:107E9000C77AF1EE10FA00F1F780FDEEE77A17EEFF
:107EA000903A1BB223812378012B02D0042B40F09F
:107EB0005881B4F90800F9F7C3FE00224FF07C5353
:107EC000F9F728FFFAF7C0F90A90B4F90200F9F7B8
:107ED000B7FE00224FF07C53F9F71CFFFAF7B4F914
:107EE0000B90B4F90400F9F7ABFE00224FF07C537D
:107EF000F9F710FFFAF7A8F90C90B4F90600F9F7B2
:107F00009FFE00224FF07C53F9F704FFFAF79CF92B
:107F10000D90DDED06AA9DED0CAA9DED0ABA9DED32
:107F20000B8ADDED089ADDED07BA9DED0D9ADDEDCA
:107F3000098A677894F800802AEE8A0A1BEE290ADB
:107F40002AEE887A1BEE2B7A0BEEC90A6AEE897A42
:107F50000AEE687A5BEE287A08EE280A09EE897A3A
:107F600048EE697A20EE000A4BEE8A7A07EE070A9D
:107F700007EEA70A12F0AEFC68EE2B0A4BEE2A0AB7
:107F80004AEE290A49EE280AF0EEE00A15F08FFFC2
:107F9000DFED457A30EE000A2A464146384620EEAB
:107FA000270AFFF7D7FC2A4631462046FFF71AFA80
:107FB0000EB0BDEC088BBDE8F081F5EEC07AF1EEB5
:107FC00010FA7FF5F6AE2B46D3ED005A0137F1EEED
:107FD000655A042FE3EC015AF6D1EAE607EB0E12DC
:107FE000D2ED015A92ED005A66EE255A47EE855AB7
:107FF00092ED025A46EE855A92ED035A03EB0E12A9
:1080000092ED014AD2ED004A47EE055A9DED0B5A1A
:1080100025EE045A9DED0A4A04EE245AD2ED024A96
:108020009DED0C4A04EE245AD2ED034A9DED0D4A13
:1080300004EE245AB5EEC05AF1EE10FA44BF1B49C3
:108040000A68F5EEC05A44BF01320A60F1EE10FA38
:1080500041BF17490A6801320A6016490A680132AD
:108060000A60AFE647F6FF73DAE6134BD8E647F649
:10807000FF73EBE6104BE9E647F6FF73FCE60E4BA9
:10808000FAE647F6FF730DE70B4B0BE76666663FB4
:10809000CDCC8C3FC4D80120C4E8012000000047AB
:1080A00000FEFF46000000C7E12E6542CCF801202B
:1080B000C8F80120C4F801200080FFFFC23E022062
:1080C000000000450000804400230A932946C5E9CA
:1080D0000133304601F0B0F9DDED0B6A5FED085A6F
:1080E000B7EE006A76EE866AB6EE007A66EE876ACA
:1080F000F0EE477A46EEA57A40F2FF71DDED0C6AAC
:1081000076EE866AFDEEE77A66EE876A17EE902ACB
:10811000F0EE477A46EEA57A22EAE2728A425FEDF5
:10812000176AFDEEE77AA8BF0A4617EE903ADDED32
:108130000A7A77EE867A23EAE37367EE877A8B42D0
:1081400007EEA67AA8BF0B465B0543EA8223FDEE45
:10815000C77A17EE902A82F30A021343C4F8053057
:10816000A1E6D4F80570C7F30900F9F759FD1D4BD6
:108170000022F9F7CFFDFAF767F807EE900A77EEDD
:10818000A77AB7EE008A77EEC87AC7F38A20CDEDDA
:10819000037AF9F745FD00224FF07D53F9F7BAFD58
:1081A000FAF752F807EE900A77EEA77A780D77EE95
:1081B000C87ACDED047AF9F733FD00224FF07D53F4
:1081C000F9F7A8FDFAF740F807EE900A77EEA77ADC
:1081D000294677EEC87A03A8CDED057A01F078F943
:1081E00097E600BF0000503F034B1B7813B10348D4
:1081F0000FF042B9704700BFC23F0220F0180220C2
:1082000010B5062003F024FA38B1084B436102236D
:108210000374002343748374C374BDE8104004499D
:1082200000234FF4845214F071BC00BFD20402004A
:1082300054E4010008B5FFF713FDBFF35B8F094B52
:1082400053E8002F22F0010143E800100028F7D185
:10825000BFF35B8FD30703D4BDE80840FFF7D0BF5F
:1082600008BD00BFE8180220012810B502D003287D
:1082700004D010BD084B00221A70FAE70B78064CA8
:108280000BB92370F5E72378002BF2D1034B186864
:10829000FFF7D0FF0123F4E7C3470220EC180220C8
:1082A00080B50C4A0C4B00AF88B0002908BF1346BC
:1082B0006A460A49C2E905134FF400739383084BD9
:1082C00042F8103F074800234FF4E65103F066FBE5
:1082D000BD4680BD64FE0100CD0702000605020018
:1082E0000300000154E4010073B53A483A4C0DF024
:1082F000F5FF05462060A0B9062003F0A9F930B1CA
:10830000364B43610223037445748574C574344944
:1083100000234FF4825214F0F9FB6FF0120002B008
:1083200070BD082003F094F940B12E4BC0E905352B
:1083300003230374002343748374C3742849002304
:108340004FF4C65214F0E2FB274B284920680F2255
:1083500007F032F8BFF35B8F254B53E8001F41F065
:10836000010143E80012002AF7D1BFF35B8F15F03B
:1083700025FB204A204EA0FB020302FB0131C00B6B
:1083800040EA4140C90BC6E9000100252122002333
:108390001A48CDE9002310F069FE2068294614F040
:1083A00067FE80B1062003F053F930B1144B4361EE
:1083B0000223037445748574C574094900234FF47E
:1083C000845214F0A3FB206802B0BDE8704014F0A2
:1083D00054BE00BF17050200EC1802201D05020064
:1083E00054E401003705020074E60100F1070200C1
:1083F000E818022040420F0088570020082900207A
:108400004A05020010B1034BB3FBF0F0024B1860B9
:10841000704700BF40420F00E4180220034B186869
:1084200010B1034BB3FBF0F0704700BFE41802201B
:1084300040420F00044B1A680260044802680A6058
:10844000002202601A607047E0180220DC18022047
:10845000014B1870704700BFA9280020014B187805
:10846000704700BFA92800202DE9F047264B1E7851
:1084700005460F46F6B215F0A1FA04468E46EFF314
:10848000118C402383F31288BFF36F8F1F4A92F839
:1084900001383F2B0AD9D2F804380133C2F8043826
:1084A0008CF31188BFF36F8FBDE8F08792F8001846
:1084B0000B4403F03F0802EB481305F1100A28684B
:1084C00069689946A9E80300083555454B46F6D139
:1084D0000F4DA4FB053005FB0E00DB0B02EB481132
:1084E00043EA4043C00BC1E9063092F801380F74EB
:1084F0004E74013392F80818DBB2994282F80138C1
:1085000038BF82F80838CBE7C0380220986F0020C7
:1085100040420F0008B504210D2000F06FFC00F070
:1085200065FAB7EE000A00F005FA9FED090A00F0BF
:1085300011FB9FED080A00F075FB012000F0DCFA4A
:10854000002000F027FB002000F0A8FA002008BD62
:10855000002474490000000010B52DED068B90ED4D
:10856000018A90ED00AA90ED029AD0ED038ADFED2A
:10857000187A28EE080A0AEE0A0A044609EE090AE1
:1085800008EEA80AF7EE009AB4EEE70AF1EE10FA48
:1085900016D412F09FF989EE807A6AEE079A68EE97
:1085A000077A29EE079A68EE878AC4ED009AC4ED2F
:1085B000017A84ED029AC4ED038ABDEC068B10BDEE
:1085C000DFED047AB0EE679AF0EE678AEDE700BF60
:1085D000CCBC8C2B0000000030B52DED088B85B095
:1085E000F0EE40AA13F025FAB5EEC00AF1EE10FA4B
:1085F00091ED00AAD1ED019A91ED029AD1ED038A95
:1086000005461446B0EE408A09D5B1EE4AAAF1EE0D
:10861000699AB1EE499AF1EE688AB1EE408AF5EEB8
:10862000C0AAF1EE10FA8DED00AACDED019A8DED04
:10863000029ACDED038A0BD82B6823606B686360C8
:10864000AB68A360EB68E36005B0BDEC088B30BDA0
:10865000F7EE007AF4EEE7AAF1EE10FA08DB84ED0B
:1086600000AAC4ED019A84ED029AC4ED038AEBE7F7
:108670009FED367AB4EEC78AF1EE10FA07DD224696
:10868000B0EE6A0A6946284613F0ECF9DCE7B4EE6E
:10869000E78AF1EE10FA55DCFFEE007AB4EE678A55
:1086A000F1EE10FA48BFB0EE678AB0EE480A12F059
:1086B0006BF8F0EE40BA12F021F8DFED257AB4EE57
:1086C000E70AF1EE10FAB0EE40BAD8D46AEEABAADF
:1086D000B0EE6A0A12F012F8F0EE40BA28EE2B8AD9
:1086E000B0EE6A0A11F0C6FFC8EE0B7A20468BEE98
:1086F0008B7AD5ED006A70EE677A2AEE07AA07EE4C
:10870000A6AA69EE879A84ED00AAD5ED016A47EE24
:10871000A69A29EE079AC4ED019AD5ED026A07EEF2
:10872000A69A68EE878A84ED029AD5ED036A47EE31
:10873000A68AC4ED038A05B0BDEC088BBDE83040C5
:10874000FFF70ABFB0EE678AAFE700BF3BDF7F3FAE
:10875000CCBC8C2BDFED177AB4EEE70AF1EE10FA01
:1087600008B51DD4DFED147AB4EE670AF1EE10FA05
:10877000C8BFB0EE670AB1EE400A80EE200A12F0E0
:1087800035F8F7EE007A37EEC00AB4EEE70AF1EEFC
:1087900010FA08DCB5EEC00AF1EE10FA06D408BDF6
:1087A000B0EE670AE7E7B0EE670AF8E79FED030A65
:1087B000F5E700BF6F12833A0AD7233D000000009F
:1087C00030B52DED028B89B00D460446B0EE408ADF
:1087D00013F02FF9B5EEC00AF1EE10FA95ED006A2C
:1087E000D5ED016A95ED027AD5ED037A2ED5B1EE7D
:1087F000466AF1EE666AB1EE477A8DED046ACDED18
:10880000056A8DED067AF1EE677AB1EE400ACDED9C
:10881000077ADFED137AB4EEE70AF1EE10FA6A4652
:10882000B0EE480A04A9204617D5FFF7D5FE6846E2
:10883000FFF792FE009B2360019B6360029BA36095
:10884000039BE36009B0BDEC028B30BD8DED046A83
:10885000CDED056A8DED067AD9E713F003F9E6E769
:10886000A4707D3F30B5D0ED017A91ED016AD0ED75
:10887000006A91ED007A67EE867A46EE877A85B0D7
:108880006B46D0ED026A91ED027A46EE877A144685
:1088900001F1100591ED037AD0ED036A46EE877A77
:1088A0001A46BFEE007AF5EEC07AF1EE10FAF7EE56
:1088B000007A58BFB0EE677AF1EC017A67EE877AFA
:1088C000A942E2EC017AF7D1254600F110012246D7
:1088D000F0EC017AB3EC017A37EE677A884247EE22
:1088E000007AE2EC017AF3D194ED010AD4ED006A4A
:1088F00094ED027AD4ED037A20EE000A06EEA60A81
:1089000007EE070A07EEA70A11F0E4FFDFED087A89
:10891000B4EEE70AF1EE10FA08DD103495ED007AB6
:10892000C7EE007AE5EC017AAC42F7D105B030BD74
:108930005F70893008B5DFED247AB4EEE70AF1EE16
:1089400010FA2DED048BF7EE008A3AD4B4EE680AE3
:10895000F1EE10FAC8BFB0EE680A9FED1C7ADFEDA9
:108960001C7A1C4B9FED1C9A83ED000A20EE078AAF
:1089700060EE277A9FED197AF4EE477AF1EE10FA5D
:10898000C8BFF0EE477A9FED167AB4EE478A38EE0C
:10899000E70AF1EE10FA48BFB0EE478A11F064FF23
:1089A000C9EE007A0F4B38EEC80AC3ED007A11F019
:1089B0005BFFC9EE007A0C4BC3ED007ABDEC048B73
:1089C00008BDB0EE670AC8E7CDCCCC3D3333733F6A
:1089D0003333B33F542600200AD7A3BB77BE7F3F73
:1089E0006F12833A502600204C260020F8B5002450
:1089F000224B234D4FF07E500022002600272146B7
:108A00000134B4F5807FC3E9106718605A609A603A
:108A1000DA6018615A619A61DA6118625A629A6280
:108A2000DA6218635A639A63DA63996483F83011DF
:108A300083F831111D675A679967D867C3F880209A
:108A4000C3F88420C3F8882083F88C101A6583F853
:108A5000641058659A65DA651A669A66DA6683F86C
:108A60004C1003F5A873CBD19FED060AFFF762FF08
:108A7000054A01231370054A1370F8BDA87700203A
:108A80008FC2753D3333333FD7580220D858022068
:108A9000014B93ED000A704754260020014B1870DB
:108AA000704700BFD7580220034B187808B1034B1A
:108AB000187800F001007047D7580220D8580220DB
:108AC0000B4B0246187890B181B10A4B4FF4A87055
:108AD00000FB023393F84C0048B11A690A605A69E6
:108AE0004A609A698A60DB69CB60704708467047C4
:108AF000D8580220A8770020014B1870704700BF9B
:108B0000AA280020014B1878704700BFAA2800202F
:108B1000B5EEC00AF1EE10FA0CD4DFED087AB4EE2F
:108B2000670AF1EE10FAC8BFB0EE670A044B83ED96
:108B3000000A70479FED030AF8E700BF9A99193EB3
:108B40000419022000000000014B93ED000A704759
:108B500004190220B5EEC00AF1EE10FA48BF9FEDED
:108B6000030A034B83ED000A704700BF00000000BA
:108B700000190220054B93ED000AB5EEC00AF1EE94
:108B800010FAD8BF9FED020A704700BF00190220FB
:108B900000007A44014B1870704700BFD65802207D
:108BA000014B1878704700BFD6580220B5EEC00AB6
:108BB000F1EE10FA22D4F5EEC00AF1EE10FA1DD44F
:108BC000DFED0F7AB4EEE70AF1EE10FA16DCF4EE00
:108BD000E70AF1EE10FA11DCB4EEE00AF1EE10FA59
:108BE000084B5CBFF0EE607AF0EE400AC3ED000A7D
:108BF000054B58BFB0EE670A83ED000A704700BF0F
:108C00000000FA444426002040260020014B93ED4A
:108C1000000A704744260020014B93ED000A70477C
:108C200040260020B5EEC00AF1EE10FA0CD4DFEDBC
:108C3000087AB4EE670AF1EE10FAC8BFB0EE670A20
:108C4000044B83ED000A70479FED030AF8E700BF6D
:108C5000CDCC4C3D4826002000000000014B93ED98
:108C6000000A70474826002022EAE27221EAE171F8
:108C700051430C22F8B55043104B42F21075B1FB32
:108C8000F5F419581E1864270D48614391FBF5F15E
:108C90007943FCF721FB71680A48614391FBF5F1C8
:108CA0007943FCF719FBB1680748614391FBF5F183
:108CB0007943BDE8F840FCF70FBB00BF8CE601002C
:108CC000DCE60100CCE60100BCE6010010B503467D
:108CD00000681B7902690121994043681B681942A9
:108CE0000AD10A490A4840F28D6213F06BFA07482C
:108CF00040F28D6113F05DFA136819428368BDE894
:108D000010400CBF1B69DB68184700BFF7FD01006E
:108D100025FE010070B503460C46DA880068197913
:108D2000224302F03004302CD0E9013605690AD123
:108D30001849194840F2E23213F044FA40F2E231A5
:108D4000144813F036FA02F00604042C08D1114935
:108D5000114840F2E93213F035FA40F2E931EFE719
:108D60001B6801248C401C4208D10A490A484FF470
:108D70007F7213F027FA4FF47F71E1E72B6812F04E
:108D8000010F14BF2343A3432B603368BDE8704039
:108D9000184700BFF7FD010025FE010010B5134C78
:108DA0004FF400312046FFF7B5FF2046104CFFF787
:108DB0008DFF4FF400312046FFF7ACFF20460D4CED
:108DC000FFF784FF4FF400312046FFF7A3FF204652
:108DD000094CFFF77BFF4FF400312046FFF79AFF65
:108DE0002046FFF773FF002010BD00BF04E701001D
:108DF000FCE60100F4E60100ECE60100012870B594
:108E00002A4E04460D4631D80FF00EFC284B834203
:108E10002CD1284B1B68F4542449002211F8013B43
:108E2000012B03D10132052AF8D1234622490878C3
:108E300098421DD1012B37D81E4B1A601F4B0022C0
:108E40001A601F480021FFF765FF1E480021FFF749
:108E500061FF1D480021FFF75DFF1C480021FFF75F
:108E600059FF1348BDE870400EF052BE7455D3E769
:108E70000B7010490A60114A0021012B1160E0D9E2
:108E80000FF0D2FB0A4DA842044609D028460EF046
:108E90003FFEFFF783FF2846BDE870400FF024B97E
:108EA000FFF77CFF2046F7E770BD00BFAB2800202E
:108EB000A8C701200C190220D95802200819022045
:108EC00004E70100FCE60100F4E60100ECE6010025
:108ED00038B59D4D9D4C2B78023B0F2B17D8DFE802
:108EE00013F010001A00300040004F0064008600AC
:108EF0009600A600AC00BA00EA00040116012001A9
:108F00002A0142F2107211460020FFF7ADFE904890
:108F10000EF0FEFDDFE72268013202F0010248BFD9
:108F2000524242F21071002022604A43FFF79CFE39
:108F30002368012B14BF4FF46170642012F0F1FD1F
:108F4000C9E72268013202F0010248BF524242F2F0
:108F50001071226000204A43FFF786FE4FF4FA703A
:108F6000ECE72268013202F0010248BF524242F2AD
:108F70001071226000204A43FFF776FEC820DDE72B
:108F80002368013313F0010F42F210710CBF0A463F
:108F9000002200202360FFF767FE2368072BEDD136
:108FA00000210120FFF72AFF95E72268531C002AC1
:108FB000236013DDC3F1CA01CA2B4FF0320342F222
:108FC000107203FB01F108BF00220020FFF74CFEE6
:108FD0002368CA2B07D100210846E3E7002242F2AA
:108FE00010711046F2E7012B4BD1FA20A6E7236857
:108FF000013313F0010F42F210710CBF0A46002238
:1090000001202360FFF730FE2368052BC7E72368A4
:10901000013313F0010F42F210710CBF0A46002217
:1090200001202360FFF720FE2368092BB7E742F2F7
:1090300010724FF4FA61012067E72268013202F0F2
:10904000010248BF524242F2107322604FF4FA61AB
:109050005A43032080E722684FF47A73013292FB6F
:10906000F3F103FB1122B2F5FA7F2260C8BF9A1A0E
:10907000C72A08DC1E235A4342F210710320FFF76F
:10908000F3FD05205AE7B2F5967F06DAC83A1421B7
:1090900041F2707301FB0232EEE7B2F5C87FABBF5D
:1090A00002EB8202C2EB021202F5EA5202F6AC5265
:1090B000A8BF0C32E0E72368013303F001031A462E
:1090C00042F2107148BF5A42002B22604FF000005C
:1090D0000CBF0A460022FFF7C7FD2368002B42F2AF
:1090E000E45008BF4FF4967028E722680A23013243
:1090F00092FBF3F103FB11222260032AD4BF02F09A
:109100000102002242F210714A43022024E7226841
:109110000A23013292FBF3F103FB11222260052A9C
:10912000ECE722680A23013292FBF3F103FB1122E0
:109130002260072AE2E72268013202F0010248BFFA
:1091400052422260DEE700BFD958022008190220EF
:10915000A8C7012070B5164D2C68E10704F007067A
:1091600007D50E200321FFF749FE41F2883012F0A7
:10917000E8FCA20707D50F200321FFF73FFE41F2CD
:10918000883012F0DEFC630707D510200321FFF7BB
:1091900035FE41F2883012F0D4FC002EDCD10321E0
:1091A0000120FFF72BFE642012F0CBFCD4E700BFB8
:1091B0001019022070B5404D04462B680E46002958
:1091C00066D0034308282B6009D850B1441E072CF1
:1091D00007D8DFE804F01C2C063F060606461028D8
:1091E0004FD008202C6802F033FA40B1334BC0E96D
:1091F000053403230374002343748374C374BDE8EC
:1092000070402F4900234FF4C65213F07FBC062054
:1092100002F01EFA38B12B4B436102230374002382
:1092200043748374C37400234FF482520EE006200B
:1092300002F00EFA38B1244B436102230374002379
:1092400043748374C37400234FF484521C4913F095
:109250005DFCC6E7062002F0FBF90028E3D01B4BBB
:10926000DAE7062002F0F4F938B1194B4361022322
:109270000374002343748374C37400234FF4865231
:10928000E4E7062002F0E4F90028F6D0114BEDE700
:1092900023EA000308202B6002F0DAF938B10E4B04
:1092A0004674C0E90534032303748674C67400232E
:1092B0004FF4C652CAE700BF101902207E08020010
:1092C000B4E40100130802002E0802003F08020067
:1092D0004D0802005B0802006B080200F0B52F4E3B
:1092E000377885B0002F56D12D4C2E48A0624FF410
:1092F0005A21216001AA13F0AEFF054698B106205D
:1093000002F0A6F930B1284B43610223037447747D
:109310008774C774254900234FF4825213F0F6FB7B
:10932000012005B0F0BD029BA38120460423E38108
:1093300001F0B2FC10F12D0F29D1062002F088F9BE
:1093400030B11B4B43610223037445748574C574AB
:10935000164900234FF4845213F0D8FBA289E38905
:10936000A06A21685A4313F0CAFD68B1062002F0D2
:109370006FF90028CED00F4B436102230374002302
:1093800043748374C374C5E7054801F085FC002865
:10939000ECD1012333700020C3E700BFDA5802206C
:1093A0001419022044E00100A1080200BCE40100FD
:1093B000B9080200E408020070B5044615461E46CE
:1093C000FFF78CFF33462A4621460248BDE870402D
:1093D00001F036BE1419022070B50D46164604463B
:1093E000FFF77CFF33462A4621460248BDE870401D
:1093F00013F032BB1419022010B588B00C46694630
:1094000012F018FC04AA2146684612F0AAFB9DED52
:10941000040AF7EE007AB4EEE70AF1EE10FA05DC82
:1094200011F0B2F930EE000A08B010BD9FED010A4C
:10943000FAE700BF0000000038B52DED048B90ED79
:10944000009A9FED210AF7EE008AF0EE689A49EE45
:10945000499A04460D4639EE800A11F03BFA88EE2F
:10946000808AB0EEC90A69EE889A89EE800A11F006
:109470002DF8DFED167AB5EE409AF1EE10FA20EEF7
:10948000270A07D019EE103AFFEE007A002BB8BF7A
:10949000F0EE678A68EE007A94ED017A67EEA87ABA
:1094A00027EE277A85ED007A94ED027A27EE277A67
:1094B00085ED017A94ED037A67EE277AC5ED027A9D
:1094C000BDEC048B38BD00BFBD37863583F9223F24
:1094D00038B52DED028B90ED018A90ED007AD0ED3C
:1094E000027A9FED1C0A28EE088A07EE078A0D46CD
:1094F000044607EEA78A38EE000A11F0EBF9F7EE02
:10950000007AC7EE808ADFED147A28EE278A28EEEB
:10951000288AB0EE480A11F0F1F868EE808AB0EEC1
:10952000480A11F0A7F885ED000AD4ED007A67EE3D
:10953000A87AC5ED017AD4ED017A67EEA87AC5ED77
:10954000027AD4ED027A67EEA87AC5ED037ABDEC13
:10955000028B38BDBD378635DB0FC93F10B5094CCE
:109560000A44914200D110BD11F8013B5840030953
:109570000001E35CC0B2434018091B01205CDBB270
:109580005840EEE7F808020070B589B30668304627
:1095900012F09DFB012201460446304612F05FFBAB
:1095A000C30708D413491448AF2212F00BFEAF21B1
:1095B000104812F0FEFD2146304612F066FB2518D9
:1095C00029460022304612F04AFB2D1AAC4206D042
:1095D00008490948B72212F0F5FDB721E8E721460E
:1095E000304612F058FB2146BDE8704012F094BCA2
:1095F00070BD00BF0809020025FE0100B2F5802FF2
:109600002DE9F0410CD2042A20D83D493D484FF4C1
:10961000077212F0D7FD4FF40771394812F0C9FDF7
:109620000823D21ACC1D114424F0070421F00701AD
:10963000091B17294FEAD1060AD83149314840F2AF
:10964000252212F0BFFD40F22521E6E70423E8E7DA
:10965000002704603146A660E760304612F04AFBFE
:109660000121421D8046304612F03BFB9200D51D81
:10967000ED082844B0423AD8B8F1FF3FA2F11002F9
:109680003946B8BF3A4604F1100014F0F5F92A46FD
:109690003946204612F017FB3B463A4639462046EB
:1096A00012F0E8FAA6EB050820463946012212F02E
:1096B000F2FA4246294612F006FB2B463A46294664
:1096C000204612F0D7FA3146204612F0FCFA434603
:1096D0003A463146204612F0CDFA31462046012264
:1096E00012F0D9FA2946BDE8F04112F0D3BB044983
:1096F000044840F23A2212F065FD40F23A218CE72C
:109700000809020025FE01002DE9F04F91B0840701
:10971000009302F004030293C2F3C20303F10103B6
:10972000DDF86880039205460E46059340F0E1811E
:10973000041D30B1072909D86FF01B0011B0BDE836
:10974000F08F01F007063444C6F10806009B4FF085
:109750000009591E4FF0040A4FF0FF330193CDF872
:1097600010904F46CB4653460DB1009820600598A7
:10977000002800F3D7809C48009A824203D39B487C
:109780008242C0F0CF80039AA4EB050E92074FEA05
:109790009E0040F1DE804FF0000CCCE07A285DD8CE
:1097A0004B280ED8472859D829282DD8252852D0FB
:1097B00054D820287AD02338D0F1000B4BEB000B83
:1097C00074E04C382E2849D8DFE800F0704848484B
:1097D00048484848484848484B4848484848484806
:1097E0004859484B4B595959704B6D487048184B64
:1097F00018484883804B48484B48800000204FF071
:10980000000B4FF0040A38E02A38C0B2012202FAF5
:1098100000F010EA0E0F49D110F0625C2FD110EA6F
:10982000020B43D06046013C5444B4FBFAF40AFBFB
:1098300004F4002D60D0A3EB050CA444B4453FF61E
:109840007BAF002867D1042B48D158F8043B236034
:10985000043404232AE0019A013A01924FF0000BEC
:1098600024E011F8010C6C2835D111F8023C0020DD
:109870006C2B8346C5D14FF0080A5346D3E708F155
:10988000070828F007080734F8E802AB24F00704BB
:1098900035B106982044B0423FF64EAFC4E900AB64
:1098A00008344FF0000B4FF0080A534611F8010F2F
:1098B000002800F0AA80BBF1000F7FF46FAF2528CD
:1098C000F4D1019B013301934FF0010B4FF0040AD7
:1098D000EBE7584693E700208346A4E7082B40F0C7
:1098E0008B8008F1070828F00708B8EC027B84EDAC
:1098F000007B08340823D9E768B9042B02D108F1AA
:109900000408A5E7082B77D108F1070828F0070815
:1099100008F10808EDE705980138059058F8040BA0
:10992000009021E7039A900744D5A4EB050E4FEA77
:109930009E004FF0010CBEF5007F1BD32C492D4833
:109940004FF41F7212F03EFC4FF41F71284812F0C2
:1099500030FC0F2F10D8002D38D007F140020DEB4E
:10996000020C019A0CF8200C0CF8102C0498013011
:1099700004901EE00F2F08D91D491E4840F2812295
:1099800012F020FC40F28121E0E7D5B107F140025E
:109990000DEB020EC0B2019A0EF8200C0EF8102C3E
:1099A000BCF1000FE2D060F07F000EF8200C09F14E
:1099B00001090137C5F10802043406924FF6DA7E38
:1099C00074E7BCF1000F01D00136F2E7029A0236CB
:1099D000002AEED10098CDE90631F8F707FEDDE95F
:1099E00006310644E5E700BFD4DE01003826020058
:1099F0002809020025FE01003F49404840F2C622E6
:109A000012F0E0FB40F2C621A0E7631BB3F5806FC4
:109A100008D33949394840F2D22212F0D3FB40F240
:109A2000D22193E71DB9A6F10804E01886E6029A50
:109A300028609B082B709DF81030C2B1EB7085F840
:109A40000290B9F1000F05D008A80022C5F1010C61
:109A500097420ED1C5F101030DF120084FF0000A25
:109A600001930DF1300B574512D1601B66E66B7008
:109A7000E5E710F8013B190608D50CEB040EB645D6
:109A800003F07F033FF658AE04F8013B0132DFE7F5
:109A9000B9F1000F03D098F90020002A17DB029BD0
:109AA000D3B11AF80B2004F8012B0022019B1819DE
:109AB0001044B0423FF640AE98F8000004F8010BA5
:109AC00000990392204613F0C9FF039A14440AF147
:109AD000010A08F10108C6E798F8002055F822307D
:109AE0000093029B45F822300098F8F77FFD421C56
:109AF000DCE76FF00D0021E62809020025FE0100D9
:109B00002DE9F04F97B000AF8946D7F880B0FA62E0
:109B10003B62044650B9A849A84840F2993212F075
:109B200051FB40F29931A44812F043FBCBF3C00340
:109B300090F802A07B6141B9457800780AEB80007B
:109B400020444D4517D8A0EB0409E378FB61BAF136
:109B5000000F02D01BF0010F16D1FB6953BBFB6A4B
:109B60001BB13A6A4946204698474D4628465C371D
:109B7000BD46BDE8F08F461C3046F8F737FD013092
:109B8000304409F10109DCE7237862687A62FA6AF5
:109B90009900B96104EB8301002A40F001814D4630
:109BA0000E4601EB0A094FF000084E454CD101EB7F
:109BB0000A0610E01BF0020FD1D023789A00BA6198
:109BC00062687A62FA6A04EB8301002A77D14D4613
:109BD00001EB0A0690461BF0050F0CBF0223012380
:109BE000FB62FB6906EB430A0BF00203BB625645BE
:109BF000BCD016F8021B16F8013C54F82390704BA9
:109C0000994502D36F4B994536D37B69002B40D0E1
:109C1000786A12F029FA00283BD0E9468AB06A46F1
:109C2000694B53617B6AC2E906314FF400731384B8
:109C3000664B42F8103F664800234FF4125101F082
:109C4000ADFE023DCD46D2E716F8013BF96254F86D
:109C50002300F8F7CBFCD7F88430F96A01304BB118
:109C6000D7F8883098453EBFD7F8843023F81800DD
:109C700008F10108054498E77B6923B1786A12F07E
:109C8000F3F90028C9D11BF0010F05D1FB6AED1AC9
:109C9000ADE7BB6A002BAAD04846F8F7A7FCD7F877
:109CA000843053B1D7F8883098453FBFD7F8842027
:109CB000431C22F8183008F10108054497E7BAF16F
:109CC000000F73D01BF0040873D0D04607F1480092
:109CD000002652463B61B96213F0C0FEB96A3B6987
:109CE00001EB0A02BA62FA69F9695200FA60BA6ACB
:109CF00002EB41023A610BF00202BA60BA6A3969BA
:109D00008A4267D162787A621BF0020F32440CBF3C
:109D10004FEA580100211BF0010FD2B240F0DF8062
:109D20001BF0040F14BF404600207B616270A070DE
:109D3000E1703A6AB969FB6A20469847051EFFF64A
:109D400015AF7B6923707B6A6370FB69E3704146E2
:109D50003A6AFB6A84F802A007F148009847B0F11C
:109D60000008C0F2F080BB693A6AA9EB0A01C91A7F
:109D7000FB68C91AD7E90A0398470028C0F2E580B2
:109D8000A84408EB00054FF0000B07F1380AB34573
:109D9000C0F0A78000213A6AFB6A08469847E5E6CA
:109DA000564607F138004FF0000892E7D046564675
:109DB00096E7464694E700BF2809020025FE010009
:109DC000D4DE01003826020053090200040000011D
:109DD00004E40100BA6A12F8021BBA6212F8015CCC
:109DE0005B4A54F82500904202D35A4A904217D356
:109DF0007A693AB1786A7B6012F036F97B6800289C
:109E00007FF47CAFBA68002A49D00F2E3DD9524961
:109E1000524840F24D4212F0D5F940F24D4182E6EF
:109E20007A693AB1786A7B6012F01EF97B68002883
:109E30007FF464AF1BF0010F0AD00F2E25D94649DD
:109E4000464840F2434212F0BDF940F243416AE60F
:109E50001BF0040F3FF452AFB8F10F0F08D93E4981
:109E60003E4840F2464212F0ADF940F246415AE611
:109E700008F1280207F1300008F1010102EB0008A7
:109E800008F8105C5FFA81F838E706F1280207F15C
:109E90003000711C161806F8205CCEB22EE7B8F11F
:109EA0000F0F08D92C492D484FF48A6212F08AF915
:109EB0004FF48A6137E608F1280207F1300C08F107
:109EC0000100944407F1580252FA80F008F10208A8
:109ED0000CF8101C5FFA88F800F8105C0EE7002000
:109EE00023E71BF80A3087F8373054F82390D7F867
:109EF00084302BB3D7F888309B4521D2D7F88430F3
:109F000033F81B803A6AFB6A012107F13700984752
:109F100000281ADB0544B8F1000F06D14846F8F7CF
:109F200065FB00F101081FFA88F83A6AFB6A4146AE
:109F300048469847002808DB05440BF1010B26E74B
:109F40004FF00008DEE7454610E605460EE600BF86
:109F5000D4DE0100382602002809020025FE010097
:109F6000014B1860704700BF5826002030B587B0FD
:109F70000025CDE903010446009503A90548059590
:109F8000FBF7FAF9DDE904309842B8BF255407B071
:109F900030BD00BFB7C00100F0B5094E01680246F0
:109FA0000A2700200B4601311C78355D6D0701D46E
:109FB0001360F0BD07FB0043A3F13000F2E700BFE0
:109FC000042402002DE9F84F15469A46D378234A17
:109FD00012F803B06F2B81460F460BF0030B2BD00A
:109FE00026D8582B0CBF10260A26DDF828803246CA
:109FF000002348463946F8F7D5FA092A08F1FF3810
:10A00000D4B21ED83034B145E4B277F1000788F8F5
:10A01000004001D3D04511D82B789B0605D5082EDA
:10A0200015D1AB7843F00803AB704046BDE8F88F1C
:10A0300003F0F703702BD5E70826D6E781460F46D5
:10A04000D5E7BBF1010F0CBF37345734DBE7102ED7
:10A05000EBD1AB7843F01003E6E700BF0424020025
:10A0600038B50D4604462022002113F005FDEB68AB
:10A07000E361AB68A3612B6823626B6863620022B3
:10A08000A2622A6923B1591E194208BF42F0010297
:10A0900022610122002104F12C0013F0DBFB40B10E
:10A0A000044905482F2212F08DF802482F2112F0A2
:10A0B00080F838BD0D0A020025FE01002DE9F04FA1
:10A0C00089B0CDE90123436A00268B4204468846C5
:10A0D00005960796B24652D300F114074FF0400B95
:10A0E000EFF3118300938BF31288BFF36F8F384621
:10A0F000DDF800900EF0BAFC40B946494648882287
:10A1000012F060F88821434812F053F838460EF0F8
:10A11000D1FC079A2AB13146204612F03AF90023C1
:10A12000079306A9204612F05AF8069941450546BC
:10A130002ED32268236A13F8221021F0030103F8BA
:10A14000221003EB820A21684246204612F06BF887
:10A15000E3682060984216D0002538460EF094FC43
:10A1600050B389F31188BFF36F8F059929B1A369A3
:10A170000BB12046984700230593002DB0D15046DF
:10A1800009B0BDE8F08F236943F008032361E3E7DA
:10A1900018B1204612F061F8DFE7DDE90132134320
:10A1A00030D0039113F084FB039958BB009B4BBB49
:10A1B00038460EF069FC40B91649174840F2311292
:10A1C00012F000F840F231119DE785F31188BFF3DA
:10A1D0006F8FDDE9012304F12C000CF0C7FE05466A
:10A1E000EFF311898BF31288BFF36F8F38460EF0AF
:10A1F0003DFC002881D03846B5FA85F50EF05AFCB2
:10A200006D09AAE707AB05AA2046266812F042F8B6
:10A210000546A2E7300A020025FE01002DE9F041C3
:10A220000446C36908460D46984704F114060746DC
:10A23000EFF31188402383F31288BFF36F8F30460A
:10A240000EF014FC40B916491648882211F0BAFFE6
:10A250008821134811F0ADFF30460EF02BFC2B780F
:10A2600043F001032B7061683A46204611F0DBFF92
:10A270006060204612F0A8F830460EF005FC40B9A8
:10A280000749084840F2311211F09CFF40F23111A9
:10A29000DFE788F31188BFF36F8FBDE8F08100BF5F
:10A2A000300A020025FE01002DE9F843044600F1C2
:10A2B0001407EFF31188402383F31288BFF36F8FE5
:10A2C00038460EF0D3FB054640B930493048882265
:10A2D00011F078FF88212D4811F06BFF38460EF001
:10A2E000E9FB2369A26813F0080F02D163689A4260
:10A2F00000D9636A9B1A002B3AD0216A11F82230E8
:10A3000013F0030001EB820935D0022803D151F884
:10A310002260B60805D1D8071AD4E36948469847A1
:10A320000646A1683246204611F07DFF3146A06006
:10A33000204611F086FF38460EF0A6FBE8B9134917
:10A34000134840F2311211F03DFF40F23111C2E7E3
:10A3500043F0020301F822304846E369A5689847B4
:10A3600029460246204611F05EFF0025A060E2E784
:10A370001D46A946DFE70546FBE788F31188BFF3D2
:10A380006F8F002D95D14846BDE8F883300A020052
:10A3900025FE01002DE9F0410446C36908460D463B
:10A3A000984704F114070646EFF31188402383F31E
:10A3B0001288BFF36F8F38460EF058FB40B923491F
:10A3C0002348882211F0FEFE8821204811F0F1FE7A
:10A3D00038460EF06FFB2B786FF300032B70236968
:10A3E0009B0705D5E268236A03EB82039D421DD1DA
:10A3F0002B786FF341032B70D4E90231994204D1D9
:10A400003246204611F00FFFA0603146204611F081
:10A4100018FF38460EF038FB68B90C490C4840F27A
:10A42000311211F0CFFE40F23111CEE72B6866F306
:10A430009F032B60EDE788F31188BFF36F8F04F162
:10A440002C00BDE8F0410CF02DBD00BF300A020029
:10A4500025FE010070B5044600F11405EFF31186E6
:10A46000402383F31288BFF36F8F28460EF0FEFA65
:10A4700040B916491648882211F0A4FE88211348D5
:10A4800011F097FE28460EF015FB2369A06813F023
:10A49000080F02D1636898420ED9646A241A2846CC
:10A4A0000EF0F2FA50B90949094840F2311211F0A0
:10A4B00089FE40F23111E2E71C1AF0E786F31188B9
:10A4C000BFF36F8F201E18BF012070BD300A02003D
:10A4D00025FE010008B50446EFF31183402383F302
:10A4E0001288BFF36F8F08F08FFC204604F07EFDCA
:10A4F000024811F0F4FD12F030FDFCE75A0A0200A8
:10A500002DE9F84F04460846A38B1907164612D4C6
:10A51000022803F0070162D1204611F07DFF88B1C7
:10A520000138042800F22581DFE810F059002301EA
:10A530007E00C800F50001280CBF43F0100143F075
:10A540002001A18304F114000EF09EFA002800F00F
:10A55000AB8086F31188BFF36F8FBDE8F88F03F0EF
:10A560000702501F01281ED80020062A2768C4E9C8
:10A57000000014D13A4603E0E08B0130E08312681A
:10A58000002AF9D123F0070343F00202A2832046F8
:10A5900011F042FF90B342F02002A2832EE023F09C
:10A5A00007039AB2F2E7042A33D123F007039AB2E1
:10A5B000A283204611F030FF10B142F02002A283A6
:10A5C000A38B03F00709894540F0DC80A18BCA0604
:10A5D00040F1218121F01003A38301F00701D4F899
:10A5E0001880A38BB8F1000FB9DA0022276823F096
:10A5F0000703C4E9002243F00103A383A38B03F004
:10A600000709894540F0BF80002FDFD00025AA460A
:10A6100040E08549854840F21B1211F0D3FD40F21D
:10A620001B11814811F0C5FD41B17F497F484FF4AE
:10A63000AB7211F0C7FD4FF4AB71F2E7236843B979
:10A6400079497A4840F2571211F0BCFD40F2571197
:10A65000E7E723691D6845B9734974484FF4AD7243
:10A6600011F0B0FD4FF4AD71DBE7A38B23F00703CE
:10A6700043F006039BB2A3830F4688464FF00609BA
:10A68000A268002A40F08180002F40F08180002DD8
:10A690009CD0BA4643F0080304F1140BA383584638
:10A6A0000EF0F2F9002875D16149604840F231128C
:10A6B00011F088FD40F231115D48B3E7022908D05E
:10A6C00059495A4840F25D1211F07CFD40F25D118B
:10A6D000A7E7E78B47B1544954484FF4AF7211F0E4
:10A6E00071FD4FF4AF719CE723695D6845B94E4930
:10A6F0004E4840F2611211F065FD40F2611190E7A1
:10A70000A38B23F0070343F004039BB2A383B84653
:10A710004FF00409B4E7012908D0434943484FF4F6
:10A72000B27211F04FFD4FF4B2717AE7236843B96A
:10A730003D493E4840F2651211F044FD40F265117A
:10A740006FE723699D6845B9374938484FF4B472BB
:10A7500011F038FD4FF4B47163E7A38B23F00703C6
:10A7600043F005039BB20027A383B8464FF00509C9
:10A7700086E72D492D4840F26B1211F023FD40F27F
:10A780006B114EE7002700257AE74FF0010A81E7B9
:10A7900092467FE786F31188BFF36F8FBAF1000FFF
:10A7A00016D147BB15B123492046A847EFF31186C0
:10A7B000402383F31288BFF36F8F58460EF056F98B
:10A7C00008BB1B491948882211F0FCFC882173E75B
:10A7D000A1680029E5D00E680029E2D0D1F804A0D4
:10A7E00043464A462046D0471EB1336831461E468E
:10A7F000F2E73346FAE7394643464A4620463F6881
:10A8000011F036FECDE758460EF054F9A38B23F035
:10A810000803A383DAE68B067FF594AE21F02003CC
:10A82000A38301F0070177E6830A020025FE0100F9
:10A83000300A020039A80000F8B504460D4600F1C0
:10A840001406EFF31187402383F31288BFF36F8F51
:10A8500030460EF00BF940B909490A48882211F038
:10A86000B1FC0748882111F0A4FC30460EF022F913
:10A87000A5613A4620460121BDE8F840FFF740BEF9
:10A88000300A020025FE01002DE9F04704460F467C
:10A8900011F0DEFD051E5DDB04F11409EFF3118AF2
:10A8A000402383F31288BFF36F8F48460EF0DEF823
:10A8B000804638B933493448882211F083FC882116
:10A8C00030483CE048460EF0F5F8E38BA68B4FF697
:10A8D000FF72934206F007063FD0022E10D10133DB
:10A8E000E383354648460EF0CFF800283BD1254992
:10A8F000254840F2311211F065FC40F23111DFE7DA
:10A90000062E13D8DFE806F0092C121209040900FC
:10A910006FF085054FF00008E4E700233B606368B3
:10A920007BB9C4E900777EB13546F3E7174916488D
:10A930004FF4E47211F046FC14484FF4E47111F046
:10A9400038FC1F606760EEE7524602212046FFF7A1
:10A95000D7FD35462846BDE8F0876FF00A05D9E7F0
:10A960006FF00405D6E78AF31188BFF36F8FB8F153
:10A97000000FEFD0002332463946204611F078FD13
:10A98000E8E700BF300A020025FE0100830A02004A
:10A99000F8B5054600F11406EFF31187402383F361
:10A9A0001288BFF36F8F30460EF060F838B9204937
:10A9B0002048882211F006FC88211D4825E03046F9
:10A9C0000EF078F8AC8B04F00704022C12D0012CA6
:10A9D0000CBF6FF004046FF0850430460EF054F89D
:10A9E00008BB1349134840F2311211F0EBFB40F25F
:10A9F0003111E2E7EB8B53B90F490E4840F2EF12E9
:10AA000011F0E0FB0C4840F2EF1111F0D2FB013BDA
:10AA10009BB2EB83002BE0D13A4621462846FFF754
:10AA20006FFD2046F8BD87F31188BFF36F8FF8E7FD
:10AA3000300A020025FE0100830A02002DE9F041E0
:10AA40000E460546002845D0002943D000F11407E2
:10AA5000EFF31188402383F31288BFF36F8F3846DA
:10AA60000EF004F838B91D491D48882211F0AAFBE0
:10AA700088211A4816E038460EF01CF83146284660
:10AA8000AC8B11F0AEFC78B104F00704231F022B4D
:10AA90000CD91449124840F22D2211F093FB1148B1
:10AAA00040F22D2111F085FB6FF0770438460DF050
:10AAB000EBFF40B909490A4840F2311211F082FB1C
:10AAC00040F23111D5E788F31188BFF36F8F20462C
:10AAD000BDE8F0816FF01504F9E700BF300A02000D
:10AAE00025FE0100830A020008B54268816002F079
:10AAF0000302032A034602D02AB1002000E00068C6
:10AB000000225A6008BD04490448452211F05AFB4E
:10AB10000148452111F04DFBA50A020025FE010068
:10AB20002DE9F34106460F4615464FF000082A4628
:10AB300001A9304611F0EEFC044640B10246394608
:10AB4000019812F08BFF2D1BA0442744EFD1424601
:10AB5000311D304611F0FCFC40B106490648482240
:10AB600011F030FB0348482111F023FB404602B0AE
:10AB7000BDE8F081C80A020025FE01002DE9F3417D
:10AB800007460E4615464FF000082A4601A93846EA
:10AB900011F0CFFC044648B12EB10246019930466F
:10ABA00012F05CFF26442D1BA044EED1424607F173
:10ABB0000A01384611F0CCFC40B106490648632230
:10ABC00011F000FB0348632111F0F3FA404602B094
:10ABD000BDE8F081C80A020025FE01002DE9F74317
:10ABE0000F4606460821C06ADFF8509011F05EFD5E
:10ABF0003C68241A80463C6004EA0905AC4203D84C
:10AC0000002003B0BDE8F08308236A4621463046A1
:10AC100011F0D5FC0028F4D16946304611F050FD02
:10AC200040B1BDF80230BDF804203C6005EA0905DA
:10AC300013441D44A4EB0804E0E700BF0000FFFF3D
:10AC400073B504460821C06A124E11F02FFD4FF66D
:10AC5000FF726368ADF800208DF80620A2891918EC
:10AC600033401344181A002560606846ADF802109E
:10AC7000ADF8045011F011FD6946204611F0E0FDD9
:10AC80002046211D11F0D4FC636828463340A360A0
:10AC900002B070BD0000FFFF2DE9F04704468AB006
:10ACA00000F11407384612F0B7FDA06A8368DB682C
:10ACB00098470546E06258B9062000F0C9FCD8B1B3
:10ACC0009F4B43610223037445748574C57413E07C
:10ACD000A06A8368DB6898470368013B1F2B17D97C
:10ACE000062000F0B5FC38B1964B43610223037493
:10ACF000002343748374C374934900234FF4825236
:10AD000011F004FF6FF0150528460AB0BDE8F08782
:10AD1000A06A216807AA12F09EFA30B1062000F05E
:10AD200097FC0028E8D0894BDFE7A5892DB1089B67
:10AD3000B5FBF3F203FB125535B1062000F088FC99
:10AD40000028D9D0824BD0E7E389012B06D8062012
:10AD500000F07EFC0028CFD07E4BB2E7E36A01957D
:10AD600093F805904FF0FF334FF0FF3238460BF069
:10AD700005FEE06A082111F099FCA8460646E38921
:10AD80001FFA85FA53451BD8E389434500F04C81EF
:10AD900053450BD1019908234A46891B204611F0DF
:10ADA0001CFC18B901A9204611F042FC01A920465B
:10ADB000FFF714FF054608B338460BF095FEA3E7EE
:10ADC000A1892B04891B13FA81F14A4608232046E6
:10ADD000019111F002FC78B101A9204611F028FC84
:10ADE00008F10108019908234A4620461FFA88F80D
:10ADF00011F0F3FB0028C7D00135C0E7019B636069
:10AE00004FEA13484FEA0848C4F80880D4E9011310
:10AE100099420FD3082303AA204611F0D0FB054620
:10AE20000028C9D103AB13F8012B914535D1013569
:10AE3000082DF8D163681B0C1B0401A9204601935F
:10AE400011F0F6FBA38901994A46204611F0C5FB93
:10AE5000051EB1DB636800F08F8006EB03084FF638
:10AE6000FF79A389CDF804801FFA88F29B1B9A42D0
:10AE70002FD300236168002B45D0090C09040191F0
:10AE8000204601A911F0D4FB0199204611F0DDFB09
:10AE90000546002D00F08D808EE703A9204611F0B5
:10AEA0000FFC626810B9921B6260AFE7BDF81050EA
:10AEB000BDF80E10E06AC4F80880294411F0F6FBD2
:10AEC00040449042A060EED1002DECD06FF01C0504
:10AED000A5E0082305AA4146204611F070FB05466F
:10AEE00000287FF469AF05A9204611F0E9FB30B1D5
:10AEF000BDF814304B4502D1BDF818300BB1B04449
:10AF0000AFE70123B6E7204611F09FFB0546002876
:10AF10007FF452AF6368104AA18913400B44A3EB3E
:10AF200046031A40A260636004F12C0204F50B7121
:10AF300042F8043F9142FBD1204611F0B5FCA7E74F
:10AF4000040B0200260B02004CE40100430B02003C
:10AF50005B0B02006F0B02000000FFFF5B1A4A460A
:10AF6000204611F03AFB051EFFF626AF08D0E26A34
:10AF7000A36812681344A360D4E901318B42EDD871
:10AF80006168A38901EB46029A4282D1DFF8AC8066
:10AF9000A26801EA08039A423FF47BAF204611F011
:10AFA00054FB054600287FF407AF636803EA0803F3
:10AFB000A3604FF40072FF2104F1300012F05CFD39
:10AFC000636802934FF6FF7805AA02A92046DDF8D0
:10AFD000089011F0B2FB054600287FF4EDAEBDF8F5
:10AFE000140040450DD011F0CDFA04EB80052B6B19
:10AFF000013306D105A9204611F062FB08B1C5F85E
:10B0000030906368029A9342DED1A2899BB2A2EB90
:10B01000460293420BD1204611F02FFC05463846DC
:10B020000BF062FD35B16FE66FF02C05C4E63846D3
:10B030000BF05AFD01232374002565E60000FFFF95
:10B040002DE9F04F91B0067C019204460F461D4653
:10B05000B6B9062000F0FCFA30B1734B436102230D
:10B06000037446748674C6744FF482526F49002389
:10B0700011F04CFD6FF00C02104611B0BDE8F08FDE
:10B08000C26A0821104611F011FB294602901046B1
:10B0900011F00CFBA389029AA3EB8203AB42064694
:10B0A000C0F0BF8055B9384611F06CFA0C3054F836
:10B0B0002030059301334DD10022DDE7019B002BA9
:10B0C00000F0AF80384611F05DFA0C3054F82030B3
:10B0D000059301333ED1002E40F08D8004F1140A17
:10B0E0004FF0FF324FF0FF3350460BF047FC4FF06C
:10B0F0000009E389994500F09180A168626873189E
:10B100009A427CD3FF23019A8DF8263020462B46A5
:10B11000ADF82210ADF82070ADF8245011F057FBB7
:10B1200029460246E06A11F0C1FAA3680344A3600D
:10B1300052B908A811F0B1FA08A9204611F080FB15
:10B14000002814BF02462A46019250460BF0CCFC60
:10B15000019A91E706AA05A92046DDF814A011F08E
:10B16000ECFA0246002887D1BDF81830BB4206D061
:10B170006268059B9A42EDD1002DACD19CE706A9EF
:10B18000204611F09DFA0028F2D0BDF81A90BDF8C3
:10B190001C304DB39D429ED1E36ADDF804B01B68BC
:10B1A0004FEA1A4A5B424FEA0A4A03F02003D144AD
:10B1B0000393AA46039B534528BF534608AA494612
:10B1C0002046984611F0FBF9021E11D1424608A90B
:10B1D000584612F033FC00287FF47DAFBAEB080A22
:10B1E000C144C344E6D167E7002B7FF474AF63E743
:10B1F0003FF771AF40E7029B1E44B6B26EE72046B0
:10B20000FFF71EFD024600289ED1204611F04CFBA0
:10B210000246002898D109F101096AE76FF01B0284
:10B2200092E76FF0150227E7F00A02004CE40100F4
:10B230002DE9FF47057CBDF8309004460E46904648
:10B240001F46ADB9062000F003FA30B1344B43611C
:10B250000223037445748574C574324900234FF486
:10B26000825211F053FC6FF00C0004B0BDE8F0877F
:10B27000C06A082111F01AFAA389A3EB4003BB426C
:10B280004AD3304611F07EF90C3054F820A0CDF8A6
:10B2900004A0BAF1FF3F1AD16FF00100E5E702AA5E
:10B2A00001A9204611F049FA0028DED1BDF8083086
:10B2B000B34206D102A9204611F002FA08B10135C5
:10B2C000ADB26268019B9A4202D1514608E0002566
:10B2D0004D455146DDF804A0E1D96368534503D1DB
:10B2E000BDF80830B342D7D1BDF80C30002BD3D015
:10B2F000A945D1D8BDF80A00090CBB424FEA01416B
:10B3000028BF3B4601444246204611F058F9002828
:10B31000ABD1BDF80C00A8E76FF01500A5E700BFA2
:10B32000F00A02004CE4010030B51049104889B021
:10B33000002212F045FB0F4D0F4900220023CDE9FA
:10B34000062300240E23CDE90334CDE901440B4B41
:10B3500000944FF4806228460CF012FA08492846FF
:10B360000CF088F9204609B030BD00BFB9B4000028
:10B3700050CE012068C9012080710220CDB70000A5
:10B38000990B02002DE9F047DFF858800446074684
:10B390004FF0010914B93846BDE8F08794FAA4F5D6
:10B3A000B5FA85F509FA05F32E0108EB05156FEAE4
:10B3B000030A24EA03042B7B002BEBD058F8063059
:10B3C0001B694BB94644032273682846196807EA8B
:10B3D0000A0711F07CFBDDE7284698470028D9D101
:10B3E000F0E700BFF4E401002DE9F047DFF8C49076
:10B3F0002C4CA9EB04038F2B80460F460AD92A490F
:10B400002A484FF4A77210F0DDFE4FF4A7712648CA
:10B4100010F0CFFE264811F03AFB064658B300253F
:10B420002846BDE8F087237B83B12368DB680BB136
:10B4300020469847636883F806A023681B6993B980
:10B44000636803221968204611F041FB013610346D
:10B450004C4514D9144915484FF4AD7210F0B2FEA2
:10B460004FF4AD71D3E7204698470028E8D00AFA98
:10B4700006F31D43EAE705464FF0010AE8E7D2D399
:10B48000B8F1000FCCD0002DC9D02846FFF77AFFC5
:10B490000546002FF7D000214FF4A4700DF024F8DA
:10B4A000F1E700BFF4E40100A10B020025FE01005A
:10B4B000581B022014E5010001480BF0F3BC00BF4B
:10B4C000102A0020014B53F82000704720E70100AC
:10B4D00008B5034608462BB1044A136000F07AFD14
:10B4E000002008BD6FF01500FBE700BF5C260020C0
:10B4F00010B5044C237813B903480BF0D3FC012397
:10B50000237010BDDB580220102A002010B504461D
:10B510000B4811F0BCFA5CB1BFF35B8F094B53E8E9
:10B52000001F013943E80012002AF8D1BFF35B8FF6
:10B53000054812F051FA0548BDE810400BF0B2BCC6
:10B54000501B0220541B022050CE0120102A002044
:10B550000020064BBFF35B8F014653E8000F43E822
:10B560000012002AF9D1BFF35B8F7047501B0220F5
:10B5700070B5FFF7EDFF0E4C0E4E0546B44215D9DF
:10B580000D490E4840F20E2210F01CFE0A4840F20F
:10B590000E2110F00EFE63685B792BB123685B68A7
:10B5A00013B12946204698471034E7E7F3D370BD1E
:10B5B000F4E4010014E50100A10B020025FE0100E6
:10B5C00010B5044C04492046FEF74AFD034B1C60AD
:10B5D00010BD00BFC42800200CE70100441B02205E
:10B5E000134A1448002310B51370134A1360134A0A
:10B5F0004FF400411360FFF76BFFFFF7E1FF104BC3
:10B60000104918468B4211D90F49104840F22912AF
:10B6100010F0D8FD0C4840F2291110F0CAFD1A1A9A
:10B620005C681211013222711033EBE7F7D310BDC1
:10B63000DC5802208BCA0100501B0220541B022040
:10B64000F4E4010014E50100A10B020025FE010055
:10B650000146002201480023FEF730BDC428002027
:10B660000148FEF721BE00BFC4280020024B01465E
:10B670001868FEF78FBE00BF441B02200148FEF78A
:10B68000E9BE00BFC428002070B52F4B18780028F1
:10B6900059D0FFF7E5FF0546002840D12B4B2C4C35
:10B6A0001B68002B19DD12F089F94FF47A72A0FBA8
:10B6B000020302FB0131C30BD4E9002043EA4143FA
:10B6C0009B1A4FEAD13140F2E93261EB000193421B
:10B6D00071F1000101D3FFF74BFFD4E9003213F5FC
:10B6E0007A7342F10002C4E90032BDE87040FFF70E
:10B6F000C5BF63685B7923B1236829461B68204670
:10B7000098471034B4420DD91249134840F202222E
:10B7100010F058FD0F4840F2022110F04AFD0F4C86
:10B720000F4EEFE7E5D32846FFF7A0FFBFF35B8F8F
:10B730000C4B53E8001F013943E80012002AF8D1EE
:10B74000BFF35B8FAAE770BDDB580220501B0220BD
:10B7500048CE0120A10B020025FE0100F4E4010007
:10B7600014E50100541B022070B5134D297809BB64
:10B770000120FFF739FE114C114EB44213D9114983
:10B78000114840F2C71210F01DFD0E4840F2C711DB
:10B7900010F00FFD63685B791BB1236820469B683E
:10B7A00098471034E9E7F5D3FFF76EFF0028FBD187
:10B7B00001232B7070BD00BFDC580220F4E40100AF
:10B7C00014E50100A10B020025FE01002DE9F04760
:10B7D0002C4B2D4FFB1A1B090AD12C492C4840F247
:10B7E000AB3210F0EFFC40F2AB31284810F0E1FC36
:10B7F00000210846FFF7F8FD044640B340F26768B1
:10B800004FF000090CF010FF224B186030B1224BB2
:10B810001B68092B02DD21480BF044FBDFF87CA0FC
:10B82000002544B12046FFF7ADFD044618B94FF09E
:10B83000FF384FF0FF39FFF727FF064628B95DB9FB
:10B8400042464B4650460BF091FB3546E9E74FF038
:10B85000FF384FF0FF39D5E70A4D08E0F0D22B68EA
:10B860009B691BB100221146284698471035BD42FE
:10B87000F4D90649064840F29F3210F0A3FC40F28A
:10B880009F31B2E7F4E4010014E50100A10B0200CE
:10B8900025FE01004C1B0220541B0220102A002010
:10B8A00013B5264811F0F3F8254B1B785BB3EFF383
:10B8B0001184402383F31288BFF36F8F21480DF06A
:10B8C000D5F840B920492148882210F07BFC882116
:10B8D0001D4810F06EFC1B480DF0ECF8FFF7D4FE8D
:10B8E00018480DF0D1F840B91749184840F2311204
:10B8F00010F068FC40F23111EAE784F31188BFF3DD
:10B900006F8F02B010BD124B1B68002BF9D050B9DD
:10B9100000220023CDE900230E4840F6CD4200234B
:10B920000DF0A4FBEDE70928EBD10A4812F054F81A
:10B93000094802B0BDE810400BF0B4BA541B022015
:10B94000DC580220481B0220300A020025FE0100BC
:10B950004C1B022050CE0120102A002010B5064BAF
:10B960001B68044698472146A0600448FEF756FC31
:10B97000BDE81040FFF794BF5C260020C4280020DB
:10B98000044A054B9B1AB1EBD30F34BF52F8310078
:10B990000020704704E40100F4E401002DE9F04FB9
:10B9A0008FB004AFC1F34A28B8600D4691467B6062
:10B9B0000C0DB8F1000F67D0002607F114034FF00B
:10B9C000040B4FF00A0AC7F80C80C7E907667E62CD
:10B9D0000193CDF808B0CDF800A007F11C03F96879
:10B9E00032464846FEF78CF8B0F5006F03461CD38C
:10B9F0006C468AB0D9F8041004AB2C48C3E90501A1
:10BA000040F2FF71D9611A464FF400711984284B36
:10BA100042F8103F274833464FF41251FFF7BEFF5C
:10BA2000A5462C37BD46BDE8F08FC0F30A0804F1E7
:10BA30001700184420F0070080083B60FFF708FE5D
:10BA400068F35325044638B33B681B4AC7E90836F8
:10BA500000F1100107F11403F961CDE900A3CDF85D
:10BA600008B0F96807F11C034846FEF749F80028BA
:10BA700012DA124912484FF4A37210F0A3FB0F48D8
:10BA80004FF4A37110F095FB04F1170020F00700AC
:10BA90008008FFF7DDFD044668F353257B68B9682D
:10BAA0002A46204611F032F8BBE700BFD80B02004F
:10BAB0000400000164E40100E1CA0100170C020067
:10BAC00025FE01002DE9F04F87B0DDE91279DDE9AF
:10BAD000106A04460391934698468FB3CDF80090C0
:10BAE0003B46524610210020CDF81490FDF70CFE85
:10BAF000051E0ADA2A492B4840F2651210F062FB53
:10BB000040F26511264810F054FBB5F5006F18DBC4
:10BB10000820FFF79DFD50B1234B436140F2FF73B6
:10BB2000836103230374002343748374C3741F4924
:10BB300000234FF4C45207B0BDE8F04F10F0E6BF49
:10BB40003D4606F11700284420F0070004F00704E2
:10BB50008008FFF77DFD0BF0070BE40044EA8B142F
:10BB600044EA452444EA0654064698B197B1CDF814
:10BB700000903B46524629461030FDF7C5FD00288F
:10BB800008DA074907484FF4C47210F01BFB4FF462
:10BB9000C471B7E70399434622463046CBE700BF5E
:10BBA000170C020025FE0100400C020064E40100B5
:10BBB000406820B1034BC01A40F3CF0070474FF0EC
:10BBC000FF30704704E401000EB403B503AB014637
:10BBD00053F8042B0448019310F0CCFF02B05DF839
:10BBE00004EB03B0704700BF09BC0000CA0605D4CF
:10BBF0008B064CBF02490349FFF7E6BF704700BF01
:10BC0000790C0200780C020038B54B681A68CB68D2
:10BC10009A4205460C4602D1084610F09EFF636822
:10BC2000BFF35B8F53E8002F511C43E8001000283E
:10BC3000F8D1BFF35B8FA3689D5463681A68E3680B
:10BC40009A4208D905490648722210F0BBFA034807
:10BC5000722110F0AEFA002038BD00BF7B0C02004C
:10BC600025FE01002DE9F04F8BB09A46169B0693F6
:10BC70009DF854B0179B0593189B199E0493044696
:10BC80000D469046BBF1000F00F0AC80BBF1040FF5
:10BC90000AD9A349A34840F2462210F093FA40F291
:10BCA00046219F4810F085FA06F00103089306F03C
:10BCB0000803079306F48073099310F006FF06F05B
:10BCC0000209024600283BD097492046FFF77CFF37
:10BCD0000746B9F1000F08D016F0440F32D193494E
:10BCE0002A462046FFF770FF0744089B53B1904B4C
:10BCF000904953F82B20904B2046002A08BF1A4643
:10BD0000FFF762FF099B002B48D0079B002B62D1F5
:10BD1000B8F1000F64D0894942462046FFF754FF2E
:10BD20000546069B3D44002B6BD1049B002B7FD125
:10BD3000F30700F1EE8031462046FFF757FFE2E0BF
:10BD40000746C6E77E4B18680028CDD07D4B4FF4E0
:10BD50007A791B68B5FBF3F54FF46163B5FBF0F13D
:10BD600000FB115509FB05F54FF03C0CB1FBF3F25C
:10BD700003FB1211B5FBF0FEB1FBFCF300FB1E55FB
:10BD80000CFB131109FB05F50091B5FBF0F56E49AD
:10BD9000CDE901E52046FFF717FFA5E7079BEBB1CB
:10BDA0006A4B6B4953F82B202046FFF70DFF0546E1
:10BDB000B8F1000F05D0614942462046FFF704FF65
:10BDC0000544BAF1000FACD0624952462046FFF755
:10BDD000FBFE0544A5E74FF0000AE1E7079DE7E712
:10BDE00045469EE7BAF1010F069B06D1D3B9049BE5
:10BDF000002B00F0888000251AE0002BF7D0564871
:10BE000011E05648069B5649224610F0FCF80028DF
:10BE10000BDA434943484FF4287210F0D3F94FF43A
:10BE200028713EE74D485D46ECE7049B002B66D049
:10BE3000DFF84081DFF84091049F3146102F204603
:10BE400028BF1027FFF7D2FE4FF0000A554543DC0C
:10BE5000059B49461A782046FFF7B6FE4FF0010AC7
:10BE60001AF0070F03D141462046FFF7ADFE5745B4
:10BE700039D9059B494613F80A202046FFF7A4FE4E
:10BE80000AF1010ABAF1100FEAD1364920464FF003
:10BE9000000AFFF799FE5246059B9A5C324B995C6B
:10BEA00011F0970F08BF2E2230492046FFF78CFE75
:10BEB0000AF1010ABAF1100F1AD01AF0070F03D1D4
:10BEC00041462046FFF780FE57455246E4D841469A
:10BED0002046FFF779FEEBE741462046FFF774FE68
:10BEE0000AF1010AB2E722492046FFF76DFEC7E7D3
:10BEF000059B3B440593049BDB1B04939CD1BBF146
:10BF0000000F7FF415AF20460BB0BDE8F04F10F0E6
:10BF100024BE094A07492046FFF756FE0BE700BF3B
:10BF20007B0C020025FE0100AC0C0200B00C0200EC
:10BF300030E70100BDF80100A70C0200D50C02009B
:10BF4000601B02205C1B0220B90C020044E70100C8
:10BF5000D90C0200DF0C020083CB010009BC0000F9
:10BF600075CB0100EE0C020004240200F00C02006C
:10BF7000EA0C0200EC0C0200E40C020073B542F281
:10BF80000F738B4228BF0B4605680F4A04460521F4
:10BF9000684610F0B1F863680C495B6806460B22EE
:10BFA000284610F0CCFD63683246694628465B6837
:10BFB00010F0C5FD636806495B681B22284610F037
:10BFC000BEFD02B070BD00BFB8EF01000F0D020052
:10BFD000F30C0200074A00210123904206D8064ACA
:10BFE00001B901231360054B1860704740085B00DE
:10BFF0000121F2E740420F005C1B0220601B02207F
:10C00000014B01221A707047DD580220014B0020BD
:10C0100019607047781B02200148FFF7AFBF00BFCF
:10C0200074E7010010B5064B18680C46FFF74AFA92
:10C0300021460346BDE8104002480F22184700BFC2
:10C04000781B022074E70100F8B5094D094B0A4E30
:10C05000D5E9004701221A700CB92C60F8BD2146C1
:10C0600030463A4600F01EF8241A0644F4E700BFB2
:10C070006C1B0220DE580220DF58022010B9074B4B
:10C0800018707047064B1B781BB141F2883011F0D5
:10C0900068BBA42000210CF027BA00BFDD580220A5
:10C0A000DE5802202DE9F047DFF87C901D4F8046D6
:10C0B0000E46042499F80050A5B911F045FB32460C
:10C0C0008246414628460AF043F80546504611F09C
:10C0D00043FBE5B101233B7099F8003073B930465A
:10C0E000BDE8F0873246414600200AF031F80546A7
:10C0F000EFE72046FFF7C2FF651E2C4600200AF03E
:10C10000B1F80028EBD03B78002BF2D1E7E73B7881
:10C11000002BE4D0013C2046FFF7B0FF3B78002B1A
:10C12000C8D1DCE7DD580220DE580220F8B5074F01
:10C130000D4604464618B44201D12846F8BD14F80D
:10C14000011BBB6801485B689847F4E704E0010005
:10C1500010B543681C68084811F007FB40B907494F
:10C160000748992210F02EF80448992110F021F880
:10C1700023685B685C6010BD04E00100470D0200AD
:10C1800025FE0100014B036000207047B8E7010065
:10C190002DE9F0471A4CDFF87480DFF874900546FB
:10C1A0000E461746444525D9164917484FF4BB6239
:10C1B00010F008F813484FF4BB610FF0FAFF626803
:10C1C000D9F824309A4213D3A3698BB1A988907807
:10C1D000C9B2884205D13A4631462846BDE8F04703
:10C1E00018475279012A03D13A46314628469847E2
:10C1F0002434D7E7E3D36FF08500BDE8F08700BFB4
:10C20000502B00209C0D020025FE0100982B0020E1
:10C21000A01B02202DE9F041134B144F5E6A144B12
:10C22000BB421BD91349144840F2BB520FF0CAFF5E
:10C23000104840F2BB510FF0BCFF5C68B4420BD316
:10C240001D694DB194F802C08488E4B2A44503D1BD
:10C250002B46BDE8F04118472433E1E7EDD36FF0FA
:10C260008500BDE8F08100BFA01B0220982B0020B4
:10C27000502B00209C0D020025FE0100024B0022E5
:10C280001A605A60704700BF5B1C02202DE9F04124
:10C29000114CDFF8508005460E461746444516D926
:10C2A0000E490F484FF4C1620FF08CFF0B484FF45A
:10C2B000C1610FF07EFF63690BB92434EEE73A46A3
:10C2C0003146284698470028F7D1BDE8F081F2D3DF
:10C2D0006FF08500F9E700BF502B00209C0D020095
:10C2E00025FE0100982B0020430670B51CD0114B91
:10C2F000114CA3421AD9114911484FF47D720FF025
:10C3000061FF0E484FF47D710FF053FF196A1E7FD5
:10C3100000220439D5B2AE4201D82433E9E7013214
:10C3200011F832508542F5D1012001E0EED3002012
:10C3300070BD00BF502B0020982B00209C0D0200E8
:10C3400025FE0100F7B58488E4B220460F468DF83B
:10C350000740FFF7C9FF054680B114F07F0F0E4E6E
:10C3600002D096F8BA30ABB1204657B103F096FE32
:10C37000F3691BB10DF1070108209847284603B067
:10C38000F0BD03F0CBFEF369002BF7D00DF10701F0
:10C390000920F2E71D46F1E7A01B022010B5044674
:10C3A0000820FFF755F940B1084BC0E905340323D5
:10C3B0000374002343748374C374054900234FF44A
:10C3C000C25210F0A3FB002010BD00BFCB0D020035
:10C3D000D4E4010038B5054610F070FE10F1780F76
:10C3E00004461ED10820FFF733F940B1184BC0E9CD
:10C3F000053503230374002343748374C374154900
:10C4000000234FF4C45210F081FB284610F02FFC9B
:10C41000114AD2F8C43023EA0003C2F8C430002421
:10C4200014E00028F1D00820FFF712F940B10B4BBF
:10C43000C0E9053503230374002343748374C37474
:10C44000044900234FF4C25210F060FB204638BD6F
:10C45000E60D0200D4E40100A01B0220070E02003A
:10C4600008B509480378C3F341130A3350F8233061
:10C470003BB100F1080200F110019847C043C00F22
:10C4800008BD1846FCE700BFA01B022004282DE9C8
:10C49000F74FDFF8D89004460F4616D0012830D168
:10C4A000DFF8C48098F8B9305BB300F0FDFF2B4D86
:10C4B0004D4532D92A492B4840F2C2420FF082FE44
:10C4C00040F2C24126480FF074FEFFF7D7FEE7E7BF
:10C4D00002EBC6060192307910F0F0FD8346307908
:10C4E00010F0C5FBD8F8C430019A23EA0003BBF171
:10C4F000000FC8F8C4300AF1010A12DA002388F8E4
:10C50000B930164D4D451BD91549164840F2EE423B
:10C510000FF058FE40F2EE41D4E7EFD22A6A4FF016
:10C52000000A2B7F5FFA8AF6B342D1D82435BFE7E1
:10C53000EB681BB13A462146284698472435E1E787
:10C54000F6D3094B1B6A2BB13946204603B0BDE830
:10C55000F04F184703B0BDE8F08F00BF502B00200C
:10C560009C0D020025FE0100A01B0220982B00203C
:10C5700073B5044680788DF8000023796279404DC8
:10C5800043EA0223ADF80230E37803F003038DF8A9
:10C59000043010F06CFBD5F8C430184206460CD0BD
:10C5A000A478204600F062FF2046FFF713FF11F049
:10C5B0007FF910B996200BF0D3FF684603F034FDE5
:10C5C00010F1780F9DF8004037D10820FFF740F8B0
:10C5D00040B12C4BC0E9053403230374002343749A
:10C5E0008374C374284900234FF4C45210F08EFAA8
:10C5F0009DF8000003F0CEFD10F1780F35D1082032
:10C600009DF80040FFF724F840B1204BC0E9053405
:10C6100003230374002343748374C3741A490023EF
:10C620004FF4C45210F072FAD5F8C43001203343ED
:10C6300085F8B900C5F8C43015E00028D8D0082026
:10C64000FFF706F840B1124BC0E905340323037429
:10C65000002343748374C3740B4900234FF4C25204
:10C6600010F054FA002002B070BD0028DCD0082081
:10C670009DF80040FEF7ECFF0028EDD0054BE3E706
:10C68000A01B0220290E0200D4E40100700E02005B
:10C690004C0E0200900E02002DE9F047A44DAB694C
:10C6A00004460E461746C3B9207800F01F00012843
:10C6B00077D0022800F0DE8000BB94F900103A68C1
:10C6C000637800292EDA062B0CD0082B25D0ABB9C5
:10C6D000537001231370022306E198470028E3D129
:10C6E00000200DE06388190A0A1F012A8C4605D92B
:10C6F000072903D8DAB26B6A1C781CB96FF01500F1
:10C70000BDE8F0875D78654503D1824200F0E7809F
:10C7100001302344F0E71B78E6E095F8BA30137057
:10C720000123E1E0052B11D0092BE7D163886E6A64
:10C73000002B33D1FFF7A2FD638885F8BA30EB698F
:10C74000002BCDD07B4903209847C9E76088C0B251
:10C7500003F0E6FB0028C3D0D0E77378042B10D099
:10C76000052B11D0022B04D177796388BB4208BF17
:10C77000012033781E443378002BEED10028BDD041
:10C78000D8E796F80380F4E76388BB42F1D1B8F1AB
:10C79000000FEED13046FFF7EBFEEAE7FF27B84681
:10C7A000E9E795F8BA30D7F800C0002BA6D0A288E8
:10C7B0006F6A5FFA82FE3B46187800289ED059784F
:10C7C000022904D193F80480F04500F28F800344DD
:10C7D000F2E78CF800308CF80130316080E71F44BC
:10C7E00090E00B2B8AD100264FF0FF08C146B246DD
:10C7F00006E07B78042B0FD0052B21D03B781F441B
:10C800003B78002BF5D1EB6913B1514607209847CF
:10C81000002E7FF465AF71E797F80280A38897F840
:10C8200003909845EAD163889945E7D1B8F1070F9D
:10C830001DD805EB0803BA4683F8BB900126DDE757
:10C84000A3884345DAD16388DBB24B450AD0BE7872
:10C85000304600F00BFE3046FFF7BCFDB0FA80F624
:10C860007609CBE73846FFF783FE0646C6E7BA46A9
:10C870000026C3E794F900206378002A19DA002B18
:10C880007FF43CAFA4883F68E4B22046FFF72CFD5C
:10C8900000283FF433AF630604D095F8BA30002B7C
:10C8A0003FF42CAF3946204603F058FC00237B7040
:10C8B00011E7012B08D0032B7FF420AF6388002BF6
:10C8C0007FF41CAF012103E0618800297FF416AFDB
:10C8D0002046FFF737FD00287FF402AF0EE702295C
:10C8E0003B607FF418AF5B883360F9E694F9000091
:10C8F00063780028BFF675AF002B3FF46AAF0A2BB0
:10C900007FF4FCAE3B78002B3FF4F8AE7978042935
:10C910007FF465AFB9788A427FF461AF072A96BF8A
:10C920005219002392F8BB308CF80030F8E600BFB3
:10C93000A01B02205A1C022070B5164D95F8B83085
:10C94000FBB103F0CDFA002822DB00F0ADFD00249E
:10C95000D5F8C430E340DA07E6B214D4D5F8C430D1
:10C9600004F11002D340DB0705D546F08000FFF745
:10C9700031FD00280CDB0134102CE9D1002385F8AF
:10C98000B830002004E03046FFF724FD0028E5DA47
:10C9900070BD00BFA01B02202DE9F84FDFF854B096
:10C9A000DFF854A005460F469046994604264B46AC
:10C9B00042463946284603F017FC10F10B0F044697
:10C9C00015D10820FEF744FE38B10323C0E905B5B0
:10C9D0000374002343748374C37400234FF4C4525C
:10C9E000514610F093F80BF099FC013EDFD1204640
:10C9F000BDE8F88FB10E0200D4E4010013B5164C67
:10CA0000237DF3B9E268A168019201AB8020FFF7B2
:10CA1000C3FF019AA3681344A360E3689B1AE36011
:10CA20006BB962B12369E2889A4208DD94F8C820A4
:10CA300093FBF2F102FB11330BB90123237502B012
:10CA400010BD00231A4619468020237502B0BDE8A8
:10CA5000104003F0C9BB00BFA01B02207FB500231C
:10CA60000D460193064600286ED1002946D10822C2
:10CA70000B460DEB020110F03AFB002803DA802090
:10CA800003F00CFB2BE03B4C029A2260039A62609D
:10CA900004F13802A2609DF90820BDF80E3025751A
:10CAA000002AC4E903551CDB802B15D90620FEF7AC
:10CAB000CFFD30B1304B436102230374457485745C
:10CAC000C5742E4900234FF4825210F01FF88020C5
:10CAD00003F0E4FA0020D3E71BB1C4E9033304B048
:10CAE00070BDFFF7BDFC0028C9D0E28823699A42D7
:10CAF000D4BFE260E360FFF781FFF0E71D4CD4E9AB
:10CB00000212002A01AB05DC024610F0F0FA002800
:10CB1000E5DAB4E710F0EBFA002804DA802003F03D
:10CB2000BDFA3046ACE7019AA3681344A360E368FA
:10CB30009B1AE360002BD2D104F13803A360FFF706
:10CB40008FFC0028D7D19AE7802807D1094BDA68F3
:10CB5000002AD0D11B7D002BCDD1C0E70849094860
:10CB60004FF4C5720FF02EFB05484FF4C5710FF05E
:10CB700020FB00BFA01B0220D80E0200D4E401005D
:10CB80009C0D020025FE0100054B064A9A62064AEA
:10CB9000DA62064A1A63064A58629A6100207047B0
:10CBA000A01B022099C6000015C200008DC2000023
:10CBB00091C100002DE9F3410646664D66484FF0ED
:10CBC000FF334FF0FF3209F0D9FE95F8B830D3B1FA
:10CBD0000620FEF73DFD38B1604B4361022303742C
:10CBE000002343748374C3745D4900234FF484525B
:10CBF0000FF08CFF6FF07704574809F075FF20465F
:10CC000002B0BDE8F0816B6ACBB900F0FFF8FFF726
:10CC1000BBFF6C6A9CB90620FEF71AFD30B1514B80
:10CC200043610223037444748474C4744C49002324
:10CC30004FF482520FF06AFF4FF0FF34DCE74A48AE
:10CC4000E8616F6A2E6203F051FC03F017F9041ECD
:10CC5000D2DB00F04BFC041ECEDB7B78012B01D134
:10CC6000FB79A3B90620FEF7F3FC38B13F4B4361D3
:10CC700002230374002343748374C374384900236C
:10CC80004FF482520FF042FF6FF01504B4E7002614
:10CC9000684685F8C830ADF802308DF804608DF82C
:10CCA000006003F0C1F9041EA6DB802768468DF8FA
:10CCB000007003F0B9F9041E9EDB2D49304603F0E5
:10CCC00001FC041E98DB2A49384603F0FBFB041ED6
:10CCD00092DB284CDFF8A88044451DD92649274817
:10CCE0004FF4C3620FF06EFA23484FF4C3610FF0A4
:10CCF00060FA276A0026227FF3B29A4201D82434D0
:10CD0000EAE707EBC30257F83310107903F0DAFBB8
:10CD100001360028EFD08FE7EBD3002003F03AFA7A
:10CD2000041EFFF669AFD5F8C430802043F001033C
:10CD3000C5F8C43003F02EFA041EFFF65DAFD5F837
:10CD4000C43043F48033C5F8C430012385F8B830CB
:10CD5000002451E7A01B0220EC290020F10E020064
:10CD6000D4E40100140F02008DC40000390F02004A
:10CD70005DCA0000502B00209C0D020025FE010022
:10CD8000982B002030B51F4B8BB005AA03F110057E
:10CD900018685968144603C40833AB422246F7D1D9
:10CDA0001B7823701022002101A810F065FE1222CA
:10CDB0000021154810F060FE102101A810F0ACFA17
:10CDC00000281BDD0828B8BF0820093801AB0E4930
:10CDD0001A18002012F8013F0AAC04EB131403F0F8
:10CDE0000F0328336B44013014F8144C13F8143C2F
:10CDF0000C7008284B7001F10201EBD102480BB016
:10CE000030BD00BF730F0200F15802202DE9F04F32
:10CE1000AD4B93F8009087B0B9F1000F03D0AB4849
:10CE200007B0BDE8F08FA94C00264FF0011801961D
:10CE30003546374623783BB9A54B02349C42F3D1A3
:10CE4000A14A01231370EAE76378052B29D8DFE8AC
:10CE500013F0EC0006006601EC002B007500402387
:10CE600004A88DF81090ADF812308DF8149003F0EE
:10CE70007DF898B1082304A8ADF8123003F076F8D5
:10CE800060B194499448ADF8129040F28F120FF0BF
:10CE900099F940F28F118F480FF08BF9BDF81230DD
:10CEA000E37123781C44C5E7E378002BF9D1A3781C
:10CEB000002B3ED1894D03E06B689C4234D0243571
:10CEC000874B9D4208D9834983484FF49B720FF0EA
:10CED00079F94FF49B71DEE7EED30820FEF7B8FB3B
:10CEE00040B1804BC0E9053403230374002343742D
:10CEF0008374C37400234FF4C2527B490FF006FEC3
:10CF00000620FEF7A5FB38B1784B4361022303747A
:10CF1000002343748374C374734900234FF4825213
:10CF20000FF0F4FD00207BE7AB6813B101992046B8
:10CF30009847019B0133DBB20193B2E7002D71D119
:10CF40000620FEF785FB30B1694B43610223037471
:10CF500045748574C57400234FF48252CDE72A6A64
:10CF600094F802C002EBC3021079844548D14FF017
:10CF7000010AE07800F003008DF81400207994F89D
:10CF800005C040EA0C20ADF8120094F90200002818
:10CF90005FFA8AFB28DA0AF1100001FA00F010EAC1
:10CFA000080F28D14BF080008DF8100004A8CDE9BF
:10CFB000023202F0DBFFDDE902320121D8B99DF82F
:10CFC0001030A37013F0800F18BF0BF1100B13710A
:10CFD00018BF5FFA8BFB0B460CBF03FA0AF301FA8A
:10CFE0000BF348EA03085CE701FA0AF010EA080FBD
:10CFF00001D15846D8E70AF1010ABAF1100FB8D1A9
:10D0000001332A7F9342AAD30620FEF721FB002892
:10D01000A1D0384B4361022303740023437483740B
:10D02000C37498E700230121EBE7032E2FD1FFF70C
:10D03000A9FE8346F8B1F5F7D9FA8246D8B110288F
:10D0400011D00620FEF704FB38B12B4B43610223BD
:10D050000374002343748374C374234900234FF47F
:10D0600084520FF053FD5246102AA8BF1022594691
:10D07000A01C10F0F3FC23786FF00200E218001BF4
:10D0800004EB5303D04214D50136F6B209E7002E63
:10D09000F1D1002F3BD10620FEF7DAFA00283FF449
:10D0A0005AAF164B43610223037447748774C774E5
:10D0B00051E7197820395E2922D906490648CB2242
:10D0C0000FF080F8CB21E6E6F05802205C2A002021
:10D0D000502B0020840F020025FE0100502B002061
:10D0E000982B0020B70F0200CCE401009D10020035
:10D0F000D70F020018100200351002008010020045
:10D1000002F8019C13F8011902F8021DBAE7E31BAB
:10D11000BB70C3F30723FB70019B3B71B4E7274649
:10D12000BFE600BF10B5094B00211A461C788442A7
:10D1300004D15C6814B102EB811010BD01310429E7
:10D1400003F14003F2D10020F7E700BF6C1C02207E
:10D150002DE9F34150F8283C10F82C6C10330446AC
:10D160000BD1036950F8202C13F002074BD0D2B931
:10D17000590715D5002344F8283C54F8283C1033AF
:10D180000BD054E9077554F8148C10F091FB00286B
:10D1900073D04048214610F07BFB02B0BDE8F0811F
:10D1A00043F00403036154F8241C01AB3046FFF73D
:10D1B000F3FB0546B0B10820FEF74AFA48B1364BFA
:10D1C000C661C0E9053504230374002343748374E6
:10D1D000C374002331494FF401520FF097FC6FF0F4
:10D1E0001503C8E7019A54F8243C134444F8243C3E
:10D1F00054F8203C9B1A44F8203C54F81C3C13443F
:10D2000044F81C3CB9E750F8241C01AB304603F04D
:10D2100097F8054670B10820FEF71AFA0028D8D012
:10D220001D4BC661C0E90535042303744774877438
:10D23000C774CEE7019D54F8243C2B4444F8243CA9
:10D2400054F8203C5B1B44F8203C54F81C3C2B4415
:10D2500044F81C3C002D8DD0304603F04DF9B5FB51
:10D26000F0F303FB1055002D84D154F8203C002B23
:10D2700080D0304603F0CCF87FE744F8180CA4F1D6
:10D28000100009F00FFE002D87D042463946304687
:10D29000A84782E788CE0120CB100200ECE4010011
:10D2A0004B1E012B73B506460D4620D8FFF73AFFFB
:10D2B0000446F0B9012D1AD101AB01220DF1030191
:10D2C000304603F03DF8019C002CF5D10620FEF716
:10D2D000BFF930B1104B436102230374447484746A
:10D2E000C4740E4900234FF482520FF00FFC02B0B9
:10D2F00070BD10F0DDFA04F12C0108B1012D05D14B
:10D30000084602B0BDE87040FFF722BF044802B0F3
:10D31000BDE8704010F0BCBAE8100200ECE4010077
:10D3200088CE01202DE9F74F054601911646984613
:10D330000FF0DBFC0446002840F08980EFF31183F6
:10D340000093402383F31288BFF36F8FDFF81491AB
:10D3500000220023484609F009FE08BBDFF808A1B7
:10D360000AEB841BA701DBF8044014F1100F39D13C
:10D3700001900820FEF76CF940B1364A019B4374D6
:10D38000C0E90525032202748374C3743249002363
:10D390004FF4C2520FF0BAFB484609F083FD18E083
:10D3A0000134042C09F14009D2D10620FEF750F9CE
:10D3B00038B12A4B436102230374002343748374FE
:10D3C000C374254900234FF482520FF09FFB6FF086
:10D3D0000B04009B83F31188BFF36F8F204603B0CB
:10D3E000BDE8F08F0C9B019ACBF814300D9BCBF865
:10D3F0001000CBF8183028466FF00F03CBE9022657
:10D400000AF80750CBF83C80CBF8043003F074F8EE
:10D4100068B1284603F070F8B6FBF0F303FB106622
:10D420002EB1DBF83C3043F00403CBF83C3018F06D
:10D43000020F07D007F12C010948514410F028FAD7
:10D440000024C6E7284602F0E3FF0446C1E76FF078
:10D450000F04C3E71D110200ECE4010002110200F9
:10D4600088CE0120881C02206C1C022010B5EFF32E
:10D470001184402383F31288BFF36F8FFFF752FEAE
:10D4800050B14368103307D16FF08B03436000F154
:10D490002C01044810F0FCF984F31188BFF36F8F5E
:10D4A00010BD00BF88CE0120F8B50E4C04254027E2
:10D4B000EFF3118687F31288BFF36F8F6368103321
:10D4C00007D16FF08B030848636004F12C0110F062
:10D4D000DFF986F31188BFF36F8F013D04F140043B
:10D4E000E6D1F8BD6C1C022088CE012070B50A4C34
:10D4F0000A4E00253146204609F04CFF0122A4F1D6
:10D5000010001146013510F0A5F9042D04F1400476
:10D51000F0D1002070BD00BF981C022051D1000046
:10D520000169012381F84B300B6833B191F8493020
:10D530001BB10248083110F0ABB9704788CE01200A
:10D540000169012381F84A300B6833B191F8483002
:10D550001BB10248083110F09BB9704788CE0120FA
:10D5600070B50569EFF31186402383F31288BFF38A
:10D570006F8FD5F89000FDF7D3FA044686F3118833
:10D58000BFF36F8F30B104480022002305F118016A
:10D590000AF004F8204670BD88CE012070B5012342
:10D5A00082F8483013680D4614463BB192F84A3071
:10D5B00023B10E4802F1080110F06AF9D4F8903056
:10D5C000DA885B899A4205D17DB904F1180140F6E9
:10D5D000CD4204E004F11801002DF8D00022BDE88E
:10D5E00070400248002309F0D9BF70BD88CE0120E9
:10D5F00070B50E4681880446C9B2154815460FF02D
:10D6000050FB10B394F900206378002A16DB202B1E
:10D6100004D0222B0ED06FF085000AE02B681A6828
:10D6200040F8102C9A8820F80C2C9B7900F80A3CC2
:10D63000002070BD638800F8093CF9E7212BEAD18E
:10D640001038072328603360F2E76FF01200F0E72C
:10D650006C1D022008B5014603480FF030FB10B1E5
:10D66000012300F8073C08BD6C1D02200D4A03464B
:10D670000021A0F848101068C3F8940090889279AF
:10D68000A3F8980083F89A2083F89C1083F89B10E5
:10D69000A3F89E1083F8A010402203F14C0010F074
:10D6A000EBB900BFC4E5010010B504690023C4F85C
:10D6B000A8300C4BC4F8A400596804F1A80269B959
:10D6C000C3E9002204F10800074909F063FE04F1F0
:10D6D0001800064909F03CFF002010BD0A605A609E
:10D6E000F0E700BF6C1D022015CD0100A5D700009A
:10D6F00030B54FF40033426805690D4C85B042F2F5
:10D70000A100CDE90103002385F89D30106AADF832
:10D710000C1000790A2201A9FFF73EF995F89D3017
:10D7200023B9012010F01DF8013CF7D105B030BD40
:10D73000A186010073B504698DF80710002384F8F1
:10D7400048304025EFF3118685F31288BFF36F8FC1
:10D750000122D4F890000DF10701FDF7E1F986F3FD
:10D760001188BFF36F8F01280AD010F0A1F810B90B
:10D7700094F8A1306BB9094B1A780AB901221A70D2
:10D780002122002304F11801054809F007FF02B027
:10D7900070BD002121200AF0A7FED3E70359022023
:10D7A00088CE0120F0B5D0F88C305B681B6A1F7DF5
:10D7B00085B0054638460FF098FA064650BB95F8F6
:10D7C00086303BB3A86F0146C38831F80A2F9B1AF5
:10D7D0009BB2B3F5806F28BF4FF4806303AA0EF0AD
:10D7E00081FE0446B0B18306A5F1180308BF00F11D
:10D7F000FF3485F830600193074B0399009322466C
:10D8000002233846FFF78EFDA86F224600F10A0179
:10D810000EF09EFE05B0F0BD9DD5000037B5144654
:10D820000A1E054621DDD4F88C0004F14C01FDF7F9
:10D8300077F9012384F8493023683BB194F84B30E1
:10D8400023B1114804F1080110F022F8D4F88C201B
:10D850009388918912695B1A9BB2D31A3F2B04D823
:10D86000012384F8A03003B030BD94F89E30002B23
:10D87000F9D0064B009301940123402204F14C019E
:10D880002846FFF74FFDEEE788CE01201DD80000A7
:10D89000F7B50D4601461D480FF0F7F9044610B3E1
:10D8A0000646691E56F8A4395F6805291BD8DFE8CB
:10D8B00001F01C1A031C222610F8061C99B901233A
:10D8C00000F8063C3B6A3246187BFFF7A7FF14F8C6
:10D8D0005C2C42B93B6A187D0D4B009301960223E4
:10D8E0001146FFF71FFD03B0F0BD304603B0BDE8A1
:10D8F000F040FFF7BBBE012304F8053CF3E710F846
:10D90000053C002BEFD00023F6E700BF6C1D022082
:10D910009DD5000037B5094D0949002400944FF00A
:10D92000FF334FF48062284609F0ACFD05492846D4
:10D9300009F0A0FE204603B030BD00BF88CE012014
:10D94000007602206011020010B5084C216811B168
:10D9500007480FF074FF4FF0FF324FF0FF330548D8
:10D9600009F02AFA2060053010BD00BF741D0220A6
:10D97000202A0020482A002038B5094C094D2046AD
:10D9800029460FF05CFF05F1880120460FF057FF94
:10D9900020460549BDE83840002204F0ABBA00BF7C
:10D9A000202A0020781D0220482A002008B50548BA
:10D9B0000EF095FB04480EF092FBBDE808400348CA
:10D9C0000EF08DBB78110200BE110200FA110200A8
:10D9D00001480BF0C3BC00BFB8E7010038B50446EE
:10D9E00018B90F4B0F485B6898476168B1F5683FFD
:10D9F00010D0B1F5680F0DD00B4DA9420AD011F42B
:10DA00006861206807D00146084808F003FF00233A
:10DA10002360656038BD142210F02EF8F9E700BFCE
:10DA2000C0270020281202002C5F5CA98823022056
:10DA300008B520B34368B3F5683F10D101220368ED
:10DA4000BFF35B8F53E8001F002903D143E8002098
:10DA50000028F7D1BFF35B8F0DD1002008BD094A24
:10DA600093420AD000684FF0FF324FF0FF3308F0C6
:10DA700085FF0028F1D00448F0E70448EEE76FF492
:10DA8000E040EBE72C5F5CA9E98FFFFFEA8FFFFF27
:10DA900008B5D8B14368B3F5683F10D100220368D8
:10DAA000BFF35B8F53E8001F012903D143E8002037
:10DAB0000028F7D1BFF35B8F0BD1002008BD074AC8
:10DAC000934208D0006809F00FF8F6E76FF4E040E1
:10DAD000F4E70348F2E70348F0E700BF2C5F5CA9D6
:10DAE000E98FFFFFEA8FFFFF10B5044618B91D4B01
:10DAF0001D485B6898476368B3F5683F2FD0B3F55E
:10DB0000680F2CD0194A934219D1236803BB1848D7
:10DB10004FF0FF324FF0FF33214608F009FE08B9FD
:10DB200023681BB90F4B13485B6898472068142281
:10DB300000210FF0A1FF4FF46863636008E0B3F5C4
:10DB4000683F0DD83A2B03D040F6BA629342DED13B
:10DB500020680FF061FE636843F03A03636010BD14
:10DB6000054AF3E7C0270020281202002C5F5CA9B9
:10DB7000882302204E1202003A00003A08B50649F6
:10DB80000648402314220FF030FEBDE80840044947
:10DB900004480BF055BC00BF881E022088230220D9
:10DBA000C0E70100D4E701002DE9F74F07460C4616
:10DBB000002900F09C800A20D1E900868D68FDF7DD
:10DBC00047FD50B1594BC0E90765C0E90538052349
:10DBD0000374002343748374C374554900234FF4C2
:10DBE00021520EF093FF0A20D4E903866569FDF700
:10DBF0002FFD50B14F4BC0E90765C0E9053805233B
:10DC00000374002343748374C374494900234FF49D
:10DC100021520EF07BFF0820E569FDF719FD40B1A8
:10DC2000454BC0E905350323037400234374837413
:10DC3000C3743F49DFF8109100234FF4C2520EF035
:10DC400065FF00252646A846326A736A01920E20B7
:10DC5000D6E90ABA0093FDF7FBFCA8B1009B43622A
:10DC6000AB1C019AC261C0E90A3BC0E90595EB1CF7
:10DC7000C0E90C3A6A1C0A230262037480F811801E
:10DC800080F8128080F813802949002345F2400271
:10DC900004350EF03BFF102D06F11006D4D10820FC
:10DCA000256EFDF7D5FC40B1244BC0E905350323B3
:10DCB0000374002343748374C3741D4900234FF419
:10DCC000C2520EF023FF0820A569FDF7C1FC40B148
:10DCD0001B4BC0E90535032303740023437483748D
:10DCE000C374134900234FF4C2520EF00FFF012FEB
:10DCF00015D1EFF305850820FDF7AAFC48B1114BBB
:10DD000043610323103D03740023856143748374CE
:10DD1000C374074900234FF4C2520EF0F7FE2146A8
:10DD2000384603B0BDE8F04F08F010BB7B1202008C
:10DD300094E40100AA120200D91202002B1302007F
:10DD40003A13020068130200E812020030BFFFF726
:10DD5000FDBF00BF054B9A699B689A421FBF044AEA
:10DD6000536843F080535360704700BF2035022052
:10DD700000ED00E02DE9F041064606200F4615466D
:10DD8000FDF766FC38B16F4B436102230374002337
:10DD900043748374C37400236B494FF482520EF0B2
:10DDA000B5FE6A4B9B6AD80662D50620FDF750FC8B
:10DDB00038B1674B436102230374002343748374B7
:10DDC000C374614900234FF482520EF09FFE4FF05E
:10DDD00011085E4B9B6A190713D50620FDF738FC26
:10DDE00038B15C4B43610223037400234374837492
:10DDF000C374554900234FF482520EF087FE4FF052
:10DE00001208524B9B6A9A0735D50620FDF720FC75
:10DE100038B1514B4361022303740023437483746C
:10DE2000C374002348494FF482520EF06FFE474BF3
:10DE30005C6B9B6A1B0674D50820FDF709FC40B19A
:10DE4000464BC0E9053403230374002343748374F1
:10DE5000C3743D4900234FF4C2520EF057FE27B160
:10DE60003A4A936A23F0800393624FF0130804E068
:10DE70004FF01008ADE76FF01504344B9B6AD807DC
:10DE800013D50620FDF7E4FB38B1354B436102237F
:10DE90000374002343748374C3742B4900234FF429
:10DEA00082520EF033FE4FF01408284B9B6A9906FD
:10DEB00013D50620FDF7CCFB38B12A4B4361022372
:10DEC0000374002343748374C3741F4900234FF405
:10DED00082520EF01BFE4FF015081C4FBB6ADA068B
:10DEE00002D4BB6A9B070BD57B68180508D5314661
:10DEF000204600F013FDB8B180F309884FF0020806
:10DF0000124B9A6A920642BF5A6A22F400525A622F
:10DF10009A6A42F0FF029A6200232B704046BDE8E5
:10DF2000F0816FF01504A0E7BB6AD906E8D50E4969
:10DF30000E484FF492720EF045F90B484FF492716F
:10DF40000EF037F97B13020094E4010000ED00E0CD
:10DF500091130200C4130200D7130200EF13020052
:10DF600005140200241402005314020025FE0100CF
:10DF700008B50620FDF76CFB38B1514B4361022315
:10DF80000374002343748374C3744E4900234FF415
:10DF900082520EF0BBFD4C4B9B6A990140F18E8082
:10DFA0000620FDF755FB38B1484B4361022303744B
:10DFB000002343748374C374424900234FF4825294
:10DFC0000EF0A4FD1E20404B9B6ADA0112D50620FC
:10DFD000FDF73EFB38B13E4B43610223037400233F
:10DFE00043748374C374374900234FF482520EF094
:10DFF0008DFD1F20344B9B6A1B0312D50620FDF7B5
:10E0000027FB38B1334B436102230374002343746D
:10E010008374C3742B4900234FF482520EF076FDB3
:10E020002120294B9B6A590312D50620FDF710FBCE
:10E0300038B1294B43610223037400234374837472
:10E04000C374204900234FF482520EF05FFD22205A
:10E050001D4B9B6A9A0312D50620FDF7F9FA38B1D9
:10E060001E4B436102230374002343748374C374FF
:10E07000144900234FF482520EF048FD2320124B26
:10E080009B6ADB0312D50620FDF7E2FA38B1144B88
:10E09000436102230374002343748374C3740949E6
:10E0A00000234FF482520EF031FD2420064A936A79
:10E0B0006FEA03436FEA1343936208BD1D2082E7B2
:10E0C0008214020094E4010000ED00E09A140200C2
:10E0D000AD140200C7140200E51402000A15020084
:10E0E0002415020070B5054606200C46FDF7B0FA6F
:10E0F00038B1604B4361022303740023437483747B
:10E10000C37400234FF482525B490EF0FFFC5B4B5B
:10E110009B6ADA0440F196800620FDF799FA38B13F
:10E12000574B436102230374002343748374C37405
:10E13000514900234FF482520EF0E8FC17204F4B58
:10E140009B6A1B0512D50620FDF782FA38B14D4BAC
:10E15000436102230374002343748374C3744649E8
:10E1600000234FF482520EF0D1FC1820434B9B6ADF
:10E170009E0530D50620FDF76BFA38B1424B43615E
:10E1800002230374002343748374C3743A49002345
:10E190004FF482520EF0BAFC384B9E6B9B6A190406
:10E1A00018D50820FDF754FA40B1384BC0E90536C0
:10E1B00003230374002343748374C3742E49002320
:10E1C0004FF4C2520EF0A2FC25B12C4A936A23F4FC
:10E1D000004393621920294B9B6A5A0512D50620E9
:10E1E000FDF736FA38B12A4B43610223037400234A
:10E1F00043748374C374204900234FF482520EF099
:10E2000085FC1A201D4B9D6A15F480751CD00620D4
:10E21000FDF71EFA38B11F4B43610223037400233C
:10E2200043748374C374144900234FF482520EF074
:10E230006DFC1B20114A936A43F47F4393620023D1
:10E24000237070BD16207AE79B6A9B04F2D50620E6
:10E25000FDF7FEF930B1104B43610223037445749E
:10E260008574C574044900234FF482520EF04EFCAD
:10E270001C20DFE74F15020094E4010000ED00E0F0
:10E2800065150200C4130200761502008F15020006
:10E29000A4150200BF150200241402002DE9F0416C
:10E2A000A44B9CB00546586800AFC0F30803002695
:10E2B00086F31188BFF36F8F02F07F44B4F17F4F74
:10E2C00014D102F00C04082C1BD10620FDF7C0F974
:10E2D00030B1994B43610223037446748674C6744B
:10E2E000964900234FF482520EF010FC9449954851
:10E2F00040F211420DF066FF40F2114190480DF0DE
:10E3000058FF12074CBF0D460126002DEED000220B
:10E31000FA71DA1E092A00F2EC80DFE812F00A0036
:10E32000D500D800C000EA00EA00EA00EA00EA00EE
:10E33000DB000620FDF78CF938B1834B43610223E3
:10E340000374002343748374C37400237B494FF424
:10E3500082520EF0DBFB4FF00008764B87F8078007
:10E36000DC6A14F0020415D00620FDF771F948B1FB
:10E37000764B43610223037480F8118080F8128089
:10E3800080F813806D4900234FF482520EF0BEFBDB
:10E39000002447E0DA6A002A0CDA0620FDF758F973
:10E3A0000028EFD06A4B43610223037444748474E1
:10E3B000C474E7E7DB6A5B007DD50620FDF748F90A
:10E3C00030B1644B43610223037444748474C47495
:10E3D0005A4900234FF482520EF098FB554BA9691D
:10E3E0005A6942F480725A61BFF34F8FBFF36F8F47
:10E3F0005A6931F8021C22F480725A61BFF34F8FC0
:10E40000BFF36F8F4DF60272914227D108202C681E
:10E41000FDF71EF960BB494900234FF4C2520EF0CC
:10E4200075FB2C68FB79ABB96822294607F1080017
:10E430000FF014FB7B6A002E77D0C3F3080222B9D9
:10E440006FEA53236FEA43237B6207F108012046FA
:10E45000FFF7AAFB7037BD46BDE8F0819A6AD2B2D9
:10E4600082B1FA1D01212846FFF784FC0446D9E752
:10E47000394BC0E9053403230374002343748374C8
:10E48000C374C8E79A6A12F47F4F04D0F91D0120C3
:10E49000FFF728FEEAE79B6AB3F5803F02D3FFF758
:10E4A00067FDE3E72649274840F2EA220DF08AFE9D
:10E4B00040F2EA2122E72249224840F2ED220DF003
:10E4C00081FE40F2ED2119E7FA1D0021CBE7F91D8D
:10E4D0000020DDE70620FDF7BBF800283FF452AF2F
:10E4E0001E4B436102230374002343748374C3747B
:10E4F00048E71B4A1B4910F4F87F6C468AB018BFE6
:10E5000011466A46103BD36117484FF400731384D9
:10E51000164BC2E9050142F8103F084800234FF4AA
:10E520001151FDF73BFAA54632E723F4FF7323F0C0
:10E53000010389E700ED00E00516020094E4010004
:10E540005314020025FE0100301602004716020097
:10E55000681602007616020095160200B116020037
:10E56000EC150200D7150200D516020004000001C8
:10E57000044B5A6942F010025A615A6922F00802AB
:10E580005A61704700ED00E0EFF30880EFF3098176
:10E5900001B57246FFF782FE01BD00BF002080F387
:10E5A0001488BFF36F8F134880F3088806F092F940
:10E5B000002011490860BFF34F8F00F033F840206E
:10E5C00080F311880D484FF0AA014FF490620FF0CC
:10E5D000EEF80A484FF49061401880F30988EFF391
:10E5E00014800221084380F31488BFF36F8F00F07A
:10E5F00025F900008087022094ED00E0007F0220D2
:10E600000749D1F890200023C2F30722184693420D
:10E6100000DB7047C1F89830C1F8A0000133F6E77D
:10E6200000ED00E008B572B6002383F31388FFF70E
:10E63000E7FF144B4FF0FF32C3F88020C3F884206B
:10E64000C3F88820C3F88C20C3F89020C3F8942026
:10E65000C3F89820C3F89C20C3F88021C3F8842114
:10E66000C3F88821C3F88C21C3F89021C3F8942102
:10E67000C3F89821C3F89C2162B6BFF34F8FBFF354
:10E680006F8F08BD00E100E0084B9B6883420BD10F
:10E69000EFF3058343B1064B5A6842F080525A604B
:10E6A0005A6A22F400425A6209F0C4BF203502209F
:10E6B00000ED00E022498A6882F8DDE04FF030008A
:10E6C0001044EFF3098C80E8F01F1EF0100F03D107
:10E6D00002F19C0080EC108A402080F31288BFF386
:10E6E0006F8F184F4FF000668A698A603E6092F91A
:10E6F000DDE0D2F894000023C2F8943080F3118852
:10E700001EF0100F03D00023E1EE103A03E002F1F7
:10E710009C0090EC108AEFF3148323F0040383F33E
:10E720001488BFF36F8F04B5104600F089F9BDE877
:10E73000044002F1300090E8F01F8CF30988704724
:10E740002035022004ED00E01EF0040F0CBFEFF3B3
:10E750000880EFF30980816911F8021C0229FFD0BB
:10E7600001B572460EF0E3FB01BD00BF40B20028C8
:10E7700007DB044A4109012300F01F00834042F8EF
:10E780002130704700E100E040B200280CDB430973
:10E79000064900F01F0020330122824041F8232067
:10E7A000BFF34F8FBFF36F8F704700BF00E100E0F2
:10E7B000054B420900F01F0053F82220012303FA01
:10E7C00000F01040704700BF00E100E008B5D3073B
:10E7D0000BD40231072909D90E490F486B220DF0DD
:10E7E000F1FC0C486B210DF0E4FC002140B2002844
:10E7F000ACBF00F16040094B4FEA4111B8BF00F0D7
:10E800000F00C9B2AABF00F56140195480F8001387
:10E8100008BD00BFE816020025FE010014ED00E06F
:10E82000044B054A23F07F039360BFF34F8FBFF380
:10E830006F8F70470010000000ED00E008B5FFF793
:10E84000EFFF104BD3F8882022F47002C3F8882021
:10E85000D3F8882042F4A002C3F888204FF0404249
:10E86000C3F83422BFF34F8FBFF36F8F0023E1EE65
:10E87000103A07F08BFE0AF025F900F0B7F807F020
:10E88000CBFE00BF00ED00E042F8203C009B42F8C8
:10E890001C3C019B42F8183C0A49029B42F8143C7C
:10E8A0004FF0807342F8043C21F00101002342F84C
:10E8B000081C203AC0F894304FF47D430265C0F83C
:10E8C000DC30704713C10100037B13F0020F124BC1
:10E8D00003D190F8DD20D20611D45A6B42F0804269
:10E8E0005A63D0F8DC3019075CBF43F00803C0F866
:10E8F000DC30037B43F002030373802070475A6BC4
:10E9000022F080425A63D0F8DC301A0744BF23F06B
:10E910000803C0F8DC30F0E700EF00E00A4A0346E5
:10E92000906878B113F1160FD0F8840005D0A0F1EB
:10E9300080029A4205D8834203D2814228BF002038
:10E9400070470020704700BF20350220104B9B68A5
:10E9500083421AD1EFF30580B8B9EFF31181402259
:10E9600082F31288BFF36F8F1A7B22F002021A73B0
:10E97000EFF3148323F0040383F31488BFF36F8F42
:10E9800081F31188BFF36F8F70476FF015007047E8
:10E990002035022008B515460E460022E1EE102A69
:10E9A000EFF3148222F0040282F31488BFF36F8F16
:10E9B000BFF36F8F074A906000F042F82C4686F351
:10E9C00009880020044B984720460021002200239C
:10E9D000024C2047203502204DCF010013C1010019
:10E9E000014B10221A61704700ED00E0044800233B
:10E9F0004021C2180133302B82F80013F9D170473F
:10EA000000E100E008B5EFF30583064A103B02EB96
:10EA1000C30152F8330049688847BDE80840FFF752
:10EA200099B900BF84E00100024B034A0348012169
:10EA300000F0B2B80000042000000020E4E701006C
:10EA400010B50446FFF740FFD4F88420034605487C
:10EA5000D21AC0E90023044B8360BDE810400121B5
:10EA600000F0B6B8A823022000000B1510B504462C
:10EA70000820FCF7EDFD40B1084BC0E90534032345
:10EA80000374002343748374C374054900234FF453
:10EA9000C2520EF03BF86FF0150010BD20170200B7
:10EAA00084E4010010B40F4CD4F89030C3F3072372
:10EAB000013B984203D95DF8044BFFF7D7BFC4F878
:10EAC00098000B6823F01F03034343F01003C4F8BE
:10EAD0009C308B6843F00103C4F8A0305DF8044B10
:10EAE000704700BF00ED00E0F0B50E4685B01F4650
:10EAF00004460025B54211DA606830B3B7B1431E51
:10EB000018420ED00820FCF7A3FD08BB15490023CE
:10EB10004FF4C2520DF0FAFF6FF01502104605B027
:10EB2000F0BD7F28EED921680B42EBD12368019319
:10EB30000EF020FAA36801A90343D0B20393FFF7B4
:10EB4000B1FF10F1160FE7D0421C01350C34D1E7AC
:10EB5000054BC0E905350323037400234374837414
:10EB6000C374D3E784E4010046170200044B052276
:10EB7000C3F89420BFF34F8FBFF36F8F704700BF70
:10EB800000ED00E0BFF35F8F024B0022C3F894203A
:10EB9000704700BF00ED00E010B50A4C0123227859
:10EBA000FFF7A2FF207016300AD1074907484FF43B
:10EBB000BB720DF007FB04484FF4BB710DF0F9FA7E
:10EBC00010BD00BF045902206917020025FE010094
:10EBD00008B5114A00231278FFF786FF10F1160FCF
:10EBE00008D00E4A0021D2F89030C3F30723984290
:10EBF0000BDB08BD0A490B4840F295120DF0E2FA12
:10EC0000074840F295110DF0D4FAC2F89800C2F806
:10EC1000A0100130E7E700BF0459022000ED00E03A
:10EC20006917020025FE01002DE9F04F7048714977
:10EC3000D0F890300D68C3F307239D4285B00AD900
:10EC40006D496E4840F2AD120DF0BCFA40F2AD11C4
:10EC500069480DF0AEFAFFF795FF4968002295422A
:10EC600001F10C0129D1664C664F25706846FDF70D
:10EC700089FADFF89481DFF8949106460025AE42C8
:10EC80002ED123785A490020D1F89020C2F30722D0
:10EC90009342C0F2A380FFF769FFD1F89030C3F32D
:10ECA0000723082B00F0A0805349544840F21F224C
:10ECB0000DF088FA40F21F21CAE7C0F8982051F8F9
:10ECC0000C3C23F01F03134343F01003C0F89C30A7
:10ECD00051F8043C43F00103C0F8A0300132BEE714
:10ECE000009A02EB05132901D3F80CA00AEA0700E9
:10ECF000B0F5000F58D00AD8B0F5001F34D0B0F5E9
:10ED0000800F46D0B0F5801F12D00135B7E7B0F1C3
:10ED1000807F54D0B0F1007FF7D19868D3F804A079
:10ED200052580EF027F9CDE901A240F480200BE003
:10ED30009868D3F804A052580EF01CF9CDE901A24E
:10ED400040F0885040F430200390207801A9FFF76C
:10ED5000A9FE00283EDA2849284840F2D7120DF0D3
:10ED600031FA40F2D71173E79868D3F804B05258DB
:10ED70000EF000F91AF0010F40EA0800CDE901B2E7
:10ED80000390E2D01C491D487B220DF01BFA7B2129
:10ED90005EE79868D3F804A052580EF0EBF8CDE97E
:10EDA00001A240EA0900CFE79868D3F804A05258BE
:10EDB0000EF0E0F8CDE901A240F08270C4E7986857
:10EDC000D3F804A052580EF0D5F8CDE901A240F0D6
:10EDD0008870B9E723780133237096E7C1F898303B
:10EDE000C1F8A00001334FE7002005B0BDE8F08F67
:10EDF00000ED00E0F0E701006917020025FE0100C8
:10EE0000045902200000F0FF000008110000020277
:10EE100008B5094BC3F1005303F58023B3F5006F28
:10EE200008D20649064892220DF0CCF903489221F7
:10EE30000DF0BFF9002008BD009B0220A4170200BE
:10EE400025FE0100014B1860704700BFCC26002052
:10EE5000F8B5084F06460D460024AC4208DA3B6878
:10EE600098470A28305504F1010401D00D28F4D147
:10EE70002046F8BDC8260020F8B50A4F0D46461EAC
:10EE8000C0F10104A3199D4201DC2846F8BD737846
:10EE90000A2B02D13B680D2098473B6816F8010FFA
:10EEA0009847EFE7CC26002010B5074C2368C2181E
:10EEB0000648C0F1005101F580218A423ABF226024
:10EEC000C0184FF0FF3010BDB4230220009B022079
:10EED00010B5044650B90E490E4840F297120DF095
:10EEE00071F940F297110A480DF063F914200AF005
:10EEF000D9FB206040B90649064840F29F120DF048
:10EF000061F940F29F11EEE7BDE810400EF084BCBD
:10EF1000A417020025FE010010B550B909490A489E
:10EF200040F2C7120DF04EF9064840F2C7110DF03D
:10EF300040F94FF0FF32BDE810404FF0FF3307F0CB
:10EF40001DBD00BFA417020025FE010008B550B981
:10EF50000749084840F2E3120DF034F9044840F242
:10EF6000E3110DF026F9BDE8084007F0BDBD00BF74
:10EF7000A417020025FE010008B505480DF0AFF802
:10EF8000002383F31188BFF36F8F0423184602DF39
:10EF9000D11702000E4A0123C2F840354FF08042DB
:10EFA0004FF08051C2F87835D1F83001082808D1E7
:10EFB000D1F83411052904D80648415C09B1C2F8DA
:10EFC00038364FF080430122C3F880250020704777
:10EFD00000E00140DA17020020B1034B800143F04A
:10EFE00001031847704700BFD0E50100BFF34F8F02
:10EFF0000549064BCA6802F4E0621343CB60BFF3D5
:10F000004F8F00BFFDE700BF00ED00E00400FA05F0
:10F010002DE9F843914690F900200378002A05462F
:10F020000E4603DB6FF01500BDE8F88303F01F0305
:10F03000012BF7D14378062BF4D1B0F80480478830
:10F040001D485FFA88F841460DF02BFE3F0A044642
:10F0500090B90820FCF7FCFA38B1184B4474C0E9A9
:10F060000538032303748474C474154900234FF4D2
:10F07000C4520DF04BFDD5E7212F04D0222F10D024
:10F080006FF08500D0E70368E9885B685B6813F878
:10F09000092F914294BF31603260C9F800300020DE
:10F0A000C2E7A0F5A264EB8862689A4294BF32601E
:10F0B00033602368F1E700BFD0280220E417020084
:10F0C000DCE4010010B504460820FCF7C1FA40B1A9
:10F0D000084BC0E90534032303740023437483748D
:10F0E000C374BDE81040044900234FF4C4520DF02E
:10F0F0000DBD00BF0B180200DCE4010070B5044632
:10F100000D4601460A480DF0DAFD20B92046BDE85B
:10F110007040FFF7D7BF022D09D1A0F5A2639B680D
:10F120002BB11B691BB1BDE870400068184770BD6A
:10F13000D028022010B504460820FCF789FA40B117
:10F14000084BC0E90534032303740023437483741C
:10F15000C374BDE81040044900234FF4C4520DF0BD
:10F16000D5BC00BF31180200DCE401002DE9F041FC
:10F170000F4681880546C9B2624890460DF091FD60
:10F180000446B0B90820AD88FCF762FA38B15E4B8E
:10F190004474C0E90535032303748474C4745B4963
:10F1A00000234FF4C4520DF0B1FC6FF01200BDE823
:10F1B000F08195F9003000686E78002B51DA022E4C
:10F1C00010D0032E20D0012E3AD1A4F5A264A3685A
:10F1D00073B31C6864B343463A462946A446BDE867
:10F1E000F04160476888C0B2012338B96FF481727A
:10F1F0001444C8F800403B600020D8E7A0F58270B6
:10F200002044C8F80000F6E76B88A3B10620FCF79D
:10F210001FFA38B13E4B4361022303740023437449
:10F220008374C37400234FF4825238490DF06EFC8E
:10F230006FF08500BBE7033CC8F800400123DAE724
:10F240000820FCF705FA40B1324BC0E9053603232C
:10F250000374002343748374C37400234FF4C252B5
:10F26000E3E70A2E0AD00B2E2DD0092EE8D1A4F503
:10F27000A264A368002BDBD05C68ABE76E88310A20
:10F2800016F0FF06A4F5A26714D16FF481734FF452
:10F290008072E0180EF0F0FB4FF480623146A4F269
:10F2A00004500EF0E9FB6B88003B18BF012387F880
:10F2B0000C34A1E7BB19013607EB860683F80C1462
:10F2C00000237360EFE76D88012D08D90820FCF753
:10F2D000BFF90028C1D0104BC0E90535B7E714F8D5
:10F2E000032CAA42A4F5A26386D0E9B204F8031C59
:10F2F0009B68002B80D09B68002B3FF47DAF984724
:10F300007AE700BFD0280220E4170200DCE4010005
:10F3100052180200651802007E18020038B5044633
:10F320000D46014623480DF0B0FC20B92046BDE84B
:10F330003840FFF7FFBE691EA0F5A264092921D855
:10F34000DFE801F005201D2127292020202F0023A0
:10F3500084F80E3584F80F3594F80D35D4F810057F
:10F3600001218B4284F80D1504D0A36813B19B686A
:10F3700003B198472046BDE838400DF02DBE01236B
:10F3800084F80E3538BD002384F80E3584F80F3527
:10F39000F8E70123FAE794F80F35002BF2D00023A9
:10F3A000F4E794F80C34002BECD02046BDE838404C
:10F3B0000DF026BED028022010B50469C4E9001261
:10F3C000A3600023C4F81435064BC4F8100559682F
:10F3D00004F2145211B9C3E9002210BD0A605A6048
:10F3E000FBE700BFD028022070B54468006990F8A0
:10F3F0000E5545B190F80F0528B9206ABDE8704058
:10F400000079FDF7C9BA0620FCF722F938B1084B9C
:10F41000436102230374002343748374C374054956
:10F4200000234FF484520DF071FB6FF00A0070BDA1
:10F4300097180200DCE40100020600F07F0312D5F9
:10F44000082B05D1010700F00F0306D50E487047C1
:10F4500010F0780F12D100F00F034C2000EB431096
:10F460000A4B18447047082B05D1020700F00F0320
:10F4700006D50748704710F0780FF6D00020704787
:10F48000044800EB43107047242A0220D8280220A9
:10F49000442B0220442A0220014902480EF0F8B908
:10F4A0000029022088CF0120014601480EF0C7B98B
:10F4B000342A002008B50620FCF7CAF838B10C4BF6
:10F4C000436102230374002343748374C3740949A2
:10F4D00000234FF482520DF019FB074907484FF4FF
:10F4E000E3720CF06FFE04484FF4E3710CF061FE20
:10F4F000B8180200E4E40100D418020025FE01005F
:10F5000010B51049BFF35B8F002351E8002F012A8B
:10F5100003D141E800300028F7D1BFF35B8F0CBF67
:10F52000012018460DD151F8044C14392046FBF740
:10F5300085FA10F1780F04D12046BDE81040FBF7A2
:10F5400027BA10BDF828022002480022002307F045
:10F5500033BC00BF342A002013B5124801F010FA62
:10F56000114B98421AD1114806F03AF9002410487C
:10F5700006F08AF90F49104800944FF0FF334FF41A
:10F58000806207F07FFF0D490B4808F073F80C48C4
:10F590000C4907F0FFFE204602B010BD6FF00400DA
:10F5A000FAE700BF3DF800000000AD0B1A1B020097
:10F5B00014E80100807A022088CF0120051902009A
:10F5C00000290220EDF9000038B5002464F07F0026
:10F5D000C0B2FFF731FF50B91B491C4840F27A22F4
:10F5E0000CF0F0FD40F27A2117480CF0E2FD0134F6
:10F5F0000DF04DFD082CE9D1154D0024E0B2FFF7C8
:10F600001BFF40B9104911484FF420720CF0DAFD8D
:10F610004FF42071E8E7036903B9056101340DF087
:10F6200036FD082C05F14005E8D10A480DF02FFD04
:10F63000094BD3F87C2212B9084AC3F87C22084847
:10F640000DF025FD002038BDD418020025FE010074
:10F65000682F0220242A0220D8280220682B0220AA
:10F66000442B022010B5054CFFF76EFF20B1416816
:10F67000204607F0CFF8F7E710BD00BF4029002073
:10F6800013B500221848002301A907F051F840B330
:10F690000620FBF7DDFF38B1144B436102230374EE
:10F6A000002343748374C374114900234FF48252BE
:10F6B0000DF02CFAFFF7D6FF0B480022002301A91A
:10F6C00007F036F8044608B1FFF7F4FE019804236A
:10F6D00040600374FFF7E8FEFFF7DEFE204602B04D
:10F6E00010BD01984060FAE740290020101902007F
:10F6F000E4E40100022810B5044611D8134B1C5C49
:10F70000FFF7BEFF08B3002202740472FFF7CCFEBD
:10F710000F4B93F82430C3B1BDE81040FFF7BCBED7
:10F720000820FBF795FF40B10A4BC0E905340323DD
:10F730000374002343748374C374BDE81040064906
:10F7400000234FF4C2520DF0E1B910BD171B0200A7
:10F75000D82802202E190200E4E401002DE9F0412E
:10F76000877806463846FFF767FE3B06F47805467D
:10F7700029D5BCB1032C59D00820FBF769FF48B14B
:10F780002B4BC761C0E90534042303740023437481
:10F790008374C374BDE8F041264900234FF401523D
:10F7A0000DF0B4B9FFF76CFF034600283ED00122EC
:10F7B000AC770274032202739D60FFF775FEBDE80B
:10F7C000F041FFF769BE4CB1012CD5D1FFF758FFCE
:10F7D000034658B36C7704740473EDE7FFF750FFEA
:10F7E00020B3B278144B12F0800F02F0080111D050
:10F7F00041B1D3F8A836EB600123037402230373ED
:10F800008560DAE702F00F02142101FB0233D3F81E
:10F810000836F0E711B1D3F8A837ECE702F00F0291
:10F82000142101FB0233D3F80837E4E7BDE8F08187
:10F8300049190200E4E40100007002402DE9F041A2
:10F84000804688B01422002103A80EF015F998F81C
:10F850000030062B25D8DFE803F0B804121717A7ED
:10F8600019000224FFF70CFF0346D0B1047400F125
:10F870000802DDE9050182E8030018463CE00323A5
:10F880008DF814300024EDE70423F9E798F80270AE
:10F890003846FFF7D1FD857A06462DB1013D022D90
:10F8A0007CD908B0BDE8F0813B0698F803402AD522
:10F8B000BCB1032CF5D00820FBF7CAFE40B1444B85
:10F8C000C761C0E905340423037445748574C574A5
:10F8D000404900234FF4015208B0BDE8F0410DF05B
:10F8E00015B9FFF7CDFE03460028DAD00122B47720
:10F8F0000274032202739E60FFF7D6FD08B0BDE8D4
:10F90000F041FFF7C9BD54B1012CD4D1FFF7B8FEC7
:10F9100003460028C5D0747704740473EBE7FFF73F
:10F92000AFFE05460028BCD00123037402230373F5
:10F93000866098F8020006F10C010DF0E7FB07461F
:10F94000E0B10820FBF784FE38B1234B4474C0E9D2
:10F950000537032303748474C4741E4900234FF4D1
:10F96000C2520DF0D3F81D491D4840F29D320CF0F3
:10F9700029FC1A4840F29D310CF01BFC194AF16831
:10F98000B2F88C328B4206D95B1AA2F88C3201F0A5
:10F9900031FC2846B0E7A2F88C02FAE7404608B0EE
:10F9A000BDE8F041FFF7DABE01A801F001FC9DF8C7
:10F9B0000530052B05D19DF8043013F0600F3FF49E
:10F9C00070AF094B059301244CE703244AE700BFBD
:10F9D00049190200E4E4010075190200D41802007C
:10F9E00025FE0100D8280220442A02202DE9F043F8
:10F9F0009E4DDFF87C9285B08046FFF7A5FD074657
:10FA000010B905B0BDE8F08395F825303C7C3BB9D2
:10FA1000002C00F0CB807968954806F0FBFEECE7FF
:10FA2000042C00F20482DFE814F0C1000500860116
:10FA30009C01CA0118F8044C9CB9BB6808205E7A86
:10FA4000FBF706FE38B18B4B4474C0E9053603233F
:10FA500003748474C474884900234FF4C2520DF0B7
:10FA600055F8BC6854B9854985484FF44B720CF081
:10FA7000A9FB4FF44B7181480CF09BFB3B7B032BA4
:10FA800042D8DFE803F002487B80A27A42B17B498A
:10FA90007B484FF439720CF095FB4FF43971EAE76B
:10FAA0006669784B32607260D3F880143170D3F895
:10FAB00084147170D3F88814D3F88C0441EA0021BF
:10FAC0007180D3F89014D3F8940441EA0021B180F6
:10FAD000D3F89814D3F89C3441EA0323F380082325
:10FAE000E36030687168684B03C311462368607A2D
:10FAF000984796F90030002B09DBF3889AB232B1AF
:10FB0000A5F88C3201F076FB7968484685E700233A
:10FB1000A5F88C32F8E7637F002BF5D0237F002B0C
:10FB2000F2D000266677594826774FF0FF324FF023
:10FB3000FF330DF0BFFA636901936368CDE90236C4
:10FB400001A9607A00F094FF514B9842044611D00D
:10FB50000820FBF77DFD38B14E4B4674C0E90534F3
:10FB6000032303748674C674434900234FF4C252BE
:10FB70000CF0CCFF45480DF09FFAC5E72368012142
:10FB8000607A9847C0E7A37A6BB9E37F5BB93F48D7
:10FB90004FF0FF324FF0FF330DF08CFA01F030FBE5
:10FBA0003A480DF089FA23680221E9E73A7A042AF3
:10FBB000AAD8DFE802F090032DA9B50000F05AFEA4
:10FBC00004460028A0D100F061FDBFF35B8F3249ED
:10FBD000012351E8002F002A03D141E8003000281A
:10FBE000F7D1BFF35B8F8FD141F8084C41F8104C2F
:10FBF000E8696B611439FAF747FE002884DA1F4977
:10FC00001F4840F2AA220CF0DDFA40F2AA2132E7A6
:10FC1000002464F07F00C0B2FFF70EFC40B9174922
:10FC2000174840F231220CF0CDFA40F2312122E7A0
:10FC3000037A13B1407A01F09BFC0134082CE8D11F
:10FC400095F854311BB195F8550101F091FC002451
:10FC5000E0B2FFF7F1FB08BB0849094840F2432234
:10FC60000CF0B0FA40F2432105E700BFD82802208B
:10FC70004029002095190200E4E40100D418020094
:10FC800025FE010000700240DC280220102902201D
:10FC90000000AD0BBB190200F8280220037A13B153
:10FCA000407A01F065FC0134082CD1D195F874320A
:10FCB0001BB195F8750201F05BFC012000F0AAFD74
:10FCC000012385F825302B68002B3FF41DAF002160
:10FCD0000220984718E7002485F8254001F08EFBA4
:10FCE000FFF70EFCA04208DA5B495C4840F2C222F2
:10FCF0000CF068FA40F2C221BDE62B68002B3FF4FD
:10FD000003AF21460420E4E7002B3FF4FDAE00F0F2
:10FD1000BBFD2B68002B3FF4F7AE00210520D8E790
:10FD20002A68002A3FF4F0AE002B3FF4EDAE00212C
:10FD300006209047E8E608F110044FF0FF334FF03B
:10FD4000FF3220460DF0B6F9FFF73EFC20460DF0DD
:10FD5000B3F958F8283C002B3FF4D6AE002101201F
:10FD6000B7E795F87432CBB1012685F8896285F83A
:10FD70008862FFF785FC0446C0B90620FBF768FCE3
:10FD800030B1374B43610223037444748474C474E8
:10FD9000344900234FF482520CF0B8FE58F8283C46
:10FDA000002B3FF4B1AE00210A2092E72E4B0674DF
:10FDB00006738360FFF778FBFFF76EFBEEE7062024
:10FDC000FBF746FC38B1294B43610223037400233F
:10FDD00043748374C374234900234FF482520CF09C
:10FDE00095FE0DF0C3FB01F009FB00F031FCFFF7BD
:10FDF00039FCFFF7E9FB40B11749184840F2864249
:10FE00000CF0E0F940F2864135E60DF0A8FB184809
:10FE100000F0B6FD174B98423FF476AE0E490F48FE
:10FE200040F28D420CF0CEF940F28D4123E60820DD
:10FE3000FBF70EFC40B1104BC0E9053403230374FB
:10FE4000002343748374C374064900234FF4C252E1
:10FE50000CF05CFE58E600BFD418020025FE01003D
:10FE6000E1190200E4E40100442B0220F51902002C
:10FE70003DF800000000AD0B0C1A020038B5164D1D
:10FE800095F824402CBB05F138000DF0C5FC204648
:10FE900001F064FD22460121E8612720FEF796FC6F
:10FEA0000DF05DFBFFF790FB044610B9012385F8C8
:10FEB00024300A4B1B680BB1FFF7EEFA4FF080437A
:10FEC000D3F83834DB0702D50020FFF713FC2046B7
:10FED00038BD0024FBE700BFD8280220342A0020C8
:10FEE00010B50D484FF0FF324FF0FF330DF0E2F840
:10FEF000FFF7B8FB00F0BEFC08B101F07FFAFFF796
:10FF0000FFFA0DF033FB0548002480F82440383018
:10FF10000DF0D2F8204610BD10290220D82802206A
:10FF200008B50E4B93F824209AB193F8253083B18D
:10FF30000B4BD3F87034DBB283420DD009490A4829
:10FF400040F259520CF03EF9064840F259510CF07B
:10FF500030F96FF0120008BD0020FCE7D82802201D
:10FF600000700240D418020025FE010010B503788D
:10FF7000047903F00F02ACB9002A37D00620FBF752
:10FF800067FB30B1234B43610223037444748474D0
:10FF9000C47400234FF482521F490CF0B7FD4FF098
:10FFA000FF3010BD082A0DD90620FBF751FB0028B1
:10FFB000EFD01A4B4361022303740023437483740C
:10FFC000C374E6E7012C11D113F008041FD10620F9
:10FFD000FBF73EFB30B1124B4361022303744474C0
:10FFE0008474C47400234FF48452D5E713F00800DE
:10FFF000D7D00620FBF72CFB0028F3D0094B436138
:020000021000EC
:1000000002230374002343748374C374EAE700205B
:10001000C7E700BF241A0200E4E40100431A02000B
:10002000621A0200781A020038B5194B93F824308E
:1000300004464BB305782846FFF7FEF9E8B1457250
:1000400023798372638843602078618810F0080503
:1000500016D14B1E0B4213D00620FBF7F9FA30B134
:100060000C4B43610223037445748574C5740A49BB
:1000700000234FF482520CF049FD6FF0150038BD9B
:1000800000F038FC0020FAE76FF01200F7E700BF3D
:10009000D8280220951A0200E4E4010038B51C4B70
:1000A00093F8242005467AB393F8253063B3FFF71D
:1000B000C3F9044610B96FF0150038BD837A012BDF
:1000C0000FD007D9023B012B07D96369A361002038
:1000D000E060F2E701F09AF8F7E7284601F018F837
:1000E000F3E70620FBF7B4FA38B10A4B4361022369
:1000F0000374002343748374C374074900234FF4CB
:1001000082520CF003FDD6E76FF01200D5E700BF76
:10011000D8280220BD1A0200E4E4010038B50E4BD5
:1001200093F82420054682B193F825306BB1FFF790
:1001300083F968B115F008040AD1284601F01CF8CB
:10014000284601F04DFA204638BD6FF01200FBE75B
:100150006FF01500F8E700BFD828022038B50C4B27
:1001600093F8242005460C4662B193F825304BB134
:10017000FFF762F948B144B1284600F0E3FF207070
:10018000002038BD6FF01200FBE76FF01500F8E7B4
:10019000D828022070B5134E96F824300446C3B117
:1001A000FFF74AF90546B8B1230705D4204600F009
:1001B000E3FF204601F014FA2B7A83B901232B7256
:1001C00096F825300BB9002070BD204601F0D0F91B
:1001D000F9E76FF01200F7E76FF01500F4E76FF042
:1001E0007700F1E7D82802202DE9FF47DFF84C819E
:1001F0001E4698F8243007468A461546002B00F024
:10020000908098F82530002B00F08B8003061DD5D8
:10021000FFF712F90446C8B190F80890B9F1000F41
:100220001AD10820FBF714FA50B13F4B80F8119017
:10023000C0E905370323037480F8129080F8139007
:100240003A4900234FF4C2520CF060FC6FF01504E1
:10025000204604B0BDE8F0874FF0FF334FF0FF3287
:1002600008F138000CF026FFA37F33B108F1380005
:100270000CF022FF6FF00A04EAE7A37A7DB3002BAB
:100280003DD00123A37738464FF0000801A9CDE9FE
:1002900001A5CDF80C8000F0EBFB254B98420746FA
:1002A0003BD084F81E800EB1C6F800800820FBF712
:1002B000CFF940B11F4BC0E9053703230374002376
:1002C00043748374C374194900234FF4C2520CF071
:1002D0001DFC6FF0040418480CF0EEFEB8E7E27F56
:1002E00002B1E577002BCCD100F096FF8742C8D051
:1002F00000F086FF10480CF0DFFE0024A8E7B8F8F5
:100300000A309D42F0D26268B5FBF2F302FB135350
:10031000002BE9D10123E377E6E706B1356000243D
:10032000D9E76FF0120493E7DF1A0200E4E401005A
:100330000000AD0BFE1A020010290220D82802206E
:100340002DE9F8431D462E4B174693F8242080468E
:100350000E46002A51D093F82530002B4DD010F0D6
:10036000800F20D101B9F7B94046FFF765F8044680
:10037000C8B190F80890B9F1000F17D10820FBF729
:1003800067F950B11F4B80F81190C0E9053803237D
:10039000037480F8129080F813901B4900234FF4E7
:1003A000C2520CF0B3FB6FF0150013E04FF0FF33B7
:1003B00016484FF0FF320CF07DFEE3689F42B846CE
:1003C00028BF984646B93FB905B12B600F480CF0DD
:1003D00073FE0020BDE8F883A169424630460DF067
:1003E0003DFBA3694344A361E368A3EB0803E36017
:1003F000002DEBD0C5F80080E8E76FF01200E9E7C8
:10040000D8280220DF1A0200E4E4010010290220AB
:10041000F8B5284D95F824300746002B46D095F8BE
:100420002530002B42D0030617D4FFF705F8044609
:1004300098B1067AA6B90820FBF70AF938B11E4B25
:100440004674C0E90537032303748674C6741B49D8
:1004500000234FF4C2520CF059FB6FF01500F8BDA9
:100460004FF0FF334FF0FF3205F138000CF022FE61
:10047000E368B3B9012663692677A361637F83B11B
:10048000FFF7FEF830B905F138000CF015FE6FF0FB
:100490000B00E4E7067484600673FFF705F8FEF7C7
:1004A000FBFF07480CF008FE0020D8E76FF01200B1
:1004B000D5E700BFD8280220DF1A0200E4E40100DB
:1004C0001029022010B5084B93F824300C462BB1AC
:1004D000FEF7B2FF28B10460002010BD6FF01200DB
:1004E000FBE76FF01500F8E7D8280220014B1860F1
:1004F000704700BFD828022008B5074B93F8243076
:1005000023B1FEF799FF20B1406808BD6FF01200DB
:10051000FBE76FF01500F8E7D82802204FF0805372
:10052000D3F83021082A06D1D3F83431052B04D86A
:10053000034AD05C7047002070470120704700BF1D
:10054000691B0200EFF31180402383F31288BFF38D
:100550006F8F0A4BD3F8001C032261B949F2753141
:10056000C3F8001CC3F8142DC3F8001C80F31188D5
:10057000BFF36F8F7047C3F8142DF7E700E0064014
:10058000EFF31180402383F31288BFF36F8F0A4B80
:10059000D3F8001C61B949F27532C3F8002CC3F8D6
:1005A000141DC3F8002C80F31188BFF36F8F7047C0
:1005B0000022C3F8142DF6E700E0064000F00F0219
:1005C000082A08B50AD90B490B484FF4D7720BF02B
:1005D000F9FD08484FF4D7710BF0EBFD074B10F015
:1005E000800F03F1D80118BF0B46182000FB023022
:1005F00008BD00BF241B020025FE0100A831022017
:1006000008B500F00F03082B0AD90849084840F242
:10061000C1120BF0D7FD054840F2C1110BF0C9FD26
:10062000C043C0F3C01003EB001008BD241B020040
:1006300025FE01004FF08053D3F83031082B02BF64
:10064000024B0022C3F81C2C704700BF0070024010
:1006500008B50A4B1A78012A0AD00949094840F21C
:1006600074420BF0AFFD064840F274410BF0A1FD5F
:10067000054900220A601A7008BD00BF095902200E
:10068000241B020025FE01006033022010B5574CE8
:100690002378012B0AD05649564840F27C420BF091
:1006A00091FD40F27C4152480BF083FD524B4FF4D8
:1006B0000062C3F80024FFF731FF08B1FFF742FFE3
:1006C0004FF08053D3F83031082B18D1EFF311805D
:1006D000402383F31288BFF36F8F484BD3F8001C7D
:1006E000C02200296DD149F27531C3F8001CC3F84E
:1006F000142CC3F8001C80F31188BFF36F8F3E4B9E
:100700000122C3F80025D3F800241205FBD54FF4CD
:100710000062C3F800244FF08053D3F83031082B27
:1007200017D1EFF31180402383F31288BFF36F8F4B
:10073000324BD3F8001C002946D149F27532C3F878
:10074000002CC3F8141CC3F8002C80F31188BFF3ED
:100750006F8FFFF7E3FE30B1FFF712FFFFF7DEFE0A
:1007600008B1FFF7EFFE4FF08053D3F83031082B7C
:10077000214B0AD140F2E372C3F800284022C3F8AB
:100780000428BFF36F8FBFF34F8F8022C3F81C255F
:100790000122C3F830251A4B40F2FF121A60194BA0
:1007A00000211960184B1970184B9B68012B0FD052
:1007B0000F4910484FF495620BF004FD4FF495611A
:1007C00071E7C3F8142C96E70022C3F8142CBCE799
:1007D000FFF730FF0E4B197002232370FFF79EFEC8
:1007E00018B1BDE81040FFF7CBBE10BD095902207B
:1007F000241B020025FE01000070024000E00640BC
:100800005C3302205833022005590220002A0020C0
:100810000759022010B5104B1B78022B0AD00F4944
:100820000F4840F2DC420BF0CDFC0C4840F2DC41BA
:100830000BF0BFFC0B4B0C4C00221A700B4A0C4BFC
:10084000002808BF1346C4F800332720FDF78EFFA9
:100850000123C4F8043510BD09590220241B0200ED
:1008600025FE01000859022000700240FDFFDF0153
:10087000FDFFFF01034B1878012894BF00200120E1
:10088000704700BF0959022010B54FF0FF324FF0FA
:10089000FF33154806F06AFBEFF31181402383F321
:1008A0001288BFF36F8F114B1B7803F0FF0483B1E5
:1008B0000F4BD3F8002412F400720AD10120C3F8C0
:1008C0002C05D3F82C05D3F80004800502D5C3F815
:1008D0002C25002481F31188BFF36F8F024806F0A6
:1008E000E1FA204610BD00BF002A0020085902206E
:1008F000007002404B1E0B4210B500F008030C467E
:100900000CD001071ED11B491B4840F269520BF065
:1009100059FC40F2695117480BF04BFC91B90207A2
:1009200008D11449144840F26B520BF04BFC40F2D2
:100930006B51F0E713B1114BD3F81C35FFF73EFEB6
:10094000848210BDA3B10D4BD3F81C1540F2FF32C9
:1009500040F2FF13802918BF13469C42EED9054987
:10096000054840F26D520BF02DFC40F26D51D2E77C
:10097000402CF3E7241B020025FE0100007002401A
:10098000F8B550B92149224840F24D420BF01AFC0B
:100990001E4840F24D410BF00CFC1E4B1C7894BBE2
:1009A0001D4A106001221A7040F2FF17264664F0BB
:1009B0007F0514F0080FEDB214BF394640212846D8
:1009C000FFF798FF2846FFF7F9FD0134092C8675DB
:1009D00006730661EBD1002440F2FF17254614F0A0
:1009E000080FE6B214BF394640213046FFF782FFB8
:1009F0003046FFF7E3FD0134092C85750573056169
:100A0000EDD10648F8BD0648FCE700BF241B0200F4
:100A100025FE010009590220603302200000AD0BC1
:100A20000500AD0B08B543B200F00F0008280AD945
:100A30000C490D4840F281520BF0C4FB094840F2CA
:100A400081510BF0B6FB002B084BB4BFD3F8102537
:100A5000D3F8142501238340134214BF0120002042
:100A600008BD00BF241B020025FE010000700240EB
:100A70002DE9F84381460C46FFF7C2FDEFF31188DC
:100A8000402383F31288BFF36F8F54B92649274858
:100A900040F2BC520BF096FB40F2BC5122480BF0E6
:100AA00088FB19F00F0F03D1214B1B784B4537D131
:100AB000204B214F1B683D68DB4301269BB28640DB
:100AC0002B4333422ED14846FFF778FD19F0800FB3
:100AD00003460FD122686AB102F06042B2F1005FB2
:100AE00008D0114911484FF4BA620BF06BFB4FF478
:100AF000BA61D3E701221A7394E8070083E807007C
:100B000000221A619A750D4B0D48354380223D60D5
:100B1000C3F8042188F31188BFF36F8FBDE8F88311
:100B20000848F7E70848F5E7241B020025FE010006
:100B3000075902205C3302205833022000E100E014
:100B40000000AD0B0A00AD0B0B00AD0B10F0080F51
:100B5000074B06D0D3F8C00410F4803F18BF002024
:100B6000704700F00F0000F5947053F820007047B4
:100B7000007002402DE9F74FA04BA14DD3F854214E
:100B8000DAB10022C3F85421D3F80413890214D532
:100B90008DF80420D3F82025ADF80620D3F8C03412
:100BA000002B2B6814BF4FF001224FF480721343C7
:100BB0002B60944B01A81B689847904BD3F8604179
:100BC00034B10022C3F86021D3F86C44C3F86C44FC
:100BD000D3F828214AB10022C3F828218A4B18787B
:100BE000FFF70EFD012383401C43884F97F80080D8
:100BF00097F9009008F00F03082B0AD9844985481B
:100C00004FF491720BF0DEFA4FF4917180480BF0C3
:100C1000D0FA18F00801804E42D1B9F1000F2FDA56
:100C20007E4A52F8230020B342F823101422534383
:100C300003F1804303F51C33D3F80836784A117862
:100C400003F001034B401370FFF7F4FC754806F006
:100C500029F94046FFF7B2FC837D032B38D140468B
:100C6000FFF7CEFC012303FA00F0336823EA000308
:100C70003360DFF890A14FF001084FF006095DE006
:100C8000694A52F823000028F3D042F823101422B6
:100C9000534303F1804303F51C33D3F80837CDE702
:100CA000B9F1000F554B09DBD3F85021002AE0D0F1
:100CB0000022C3F85021D3F8A837BFE7D3F82C217E
:100CC000002AD6D00022C3F82C21D3F8A836B5E7E5
:100CD000037BE3B94046FFF793FC012303FA00F0DE
:100CE0003368B9F1000F23EA0003336002DAB8F188
:100CF000880FBED106238DF8043000238DF807300D
:100D0000404B8DF806801B6801A89847B1E7B8F101
:100D1000000FAED1394B0122DA64AAE794FAA4F0AD
:100D20002A68B0FA80F008FA00F31A430F282A6004
:100D300024EA0304326849DD134256D0002CEDD179
:100D40002E4BD3F800215AB1C3F80041374B1C7029
:100D50002D4B1C70012301932A4B01A81B68984757
:100D6000264BD3F85821002A6DD00022C3F8582111
:100D7000D3F80044C3F80044E20508D52B4B012208
:100D80001A70022301931F4B01A81B689847A30503
:100D900008D5264B00221A7003230193194B01A892
:100DA0001B68984760054ED5204A1378002B4AD01F
:100DB000124BD3F82C1500293AD01549154840F2AA
:100DC000F5220BF0FFF940F2F5211FE71340B5D1F2
:100DD00060F07F018DF804908DF806108DF80730D3
:100DE000DAF8003001A89847A8E7A0F110018DF8C3
:100DF00004908DF806108DF80780F1E7007002402E
:100E00005C33022060330220075902200659022079
:100E1000241B020025FE0100583302200871024005
:100E200005590220002A0020307102400859022092
:100E300011700122C3F808259A6504230193AD4B74
:100E400001A81B689847AC4BD3F85C31FBB1AB4BA6
:100E50009B6813B93B78590619D0A74B0022C3F8F9
:100E60005C21D3F88034A64A23F07F0313703368E3
:100E700023F0011333602B6823F4803343F0010324
:100E80002B60052301939B4B01A81B689847326890
:100E90002B681A4200F01C8198480022002306F0BB
:100EA00065F8002840F01481934BD3F82C35002BC3
:100EB00000F09A80914803B0BDE8F04F05F0F2BF12
:100EC00049F0800B5846FFF779FB037B0446002B63
:100ED00000F0AA804368B0F814800168984528BFE4
:100EE000984601F06043B3F1005F23D12268636844
:100EF00042442260A268A3EB0803D2074FFA8BF0AA
:100F0000636040F1A680B8F1000F40F0A580002397
:100F10002373A1E05846FFF719FEB4F814C06045EA
:100F20001AD97849784840F263120BF04BF940F235
:100F300063116BE6B8F1400F08D9724972484FF45B
:100F4000C1720BF03FF94FF4C1715FE66F48424642
:100F50000CF084FD6D49C9E723686BB103F0604371
:100F6000B3F1005F08D0674967484FF4B2720BF0E5
:100F700029F94FF4B27149E66368226898429BBF31
:100F80001B1A02EB000E4FF0000863609CBFC4F810
:100F900000E08046604511460FD1003B18BF012399
:100FA0006AB9B8F1000F52D0564957484FF45A72F7
:100FB0000BF008F94FF45A7128E60023F0E740459A
:100FC0003BD9012303FA09F32AEA0303022233601F
:100FD0000623A2758DF80430464B8DF806B01B68C9
:100FE0008DF8072001A89847D6F800A02B681AEAC8
:100FF00003093FF45FAF19F0012314BF93FAA3F97B
:1010000099FAA9F9B9FA89F9B9F10F0F7FF658AF32
:10101000A9F1100B5FFA8BFB5846FFF7CFFA037B61
:101020000446002B7FF476AF3649374840F25732FA
:101030000BF0C8F840F25731E8E508D031493248A2
:1010400040F279320BF0BEF840F27931DEE54FFA2A
:101050008BF0002B3FF45BAF4FF080530126D3F8A9
:101060003031082B02BF244B8222C3F81C2C2B6882
:1010700087F800B006FA09F923EA09032B6023690F
:10108000434423610BF00F04082C08D91D491E4866
:101090004FF4A4720BF096F84FF4A471B6E51BF070
:1010A000080F154B17D100284FF0140202FB043231
:1010B000A9BF0A3403EB8403C2F80017C2F80487FF
:1010C000AFBF43F82460C2F80016C2F804865E6021
:1010D00003B0BDE8F08F0028B5BFC3F8A016C3F871
:1010E000A017C3F8A486C3F8A487B4BF5E629E6449
:1010F000EEE700BF6033022000700240002A0020AB
:1011000007590220241B020025FE0100683102203D
:1011100008B503070AD50849084840F207620BF0F2
:1011200051F8054840F207610BF043F8044B40F4D6
:101130008070C3F8180508BD241B020025FE0100BD
:1011400000700240030713D400F00F0310F0800F6B
:10115000084A0BBF03F5887303F5847302EB83021F
:1011600052F8230008BF5068003818BF01207047AC
:10117000002070470070024008B503070AD50949EE
:10118000094840F229620BF01DF8064840F2296137
:101190000BF00FF8054BC3F80C0540F48070C3F852
:1011A0000C0508BD241B020025FE01000070024052
:1011B0000023036043600E4BD3F880240270D3F801
:1011C00084244270D3F88824D3F88C1442EA012294
:1011D0004280D3F89024D3F8941442EA012282800A
:1011E000D3F89824D3F89C3442EA0323C380704791
:1011F00000700240014B0122DA6470470070024027
:10120000014B01221A65704700700240014B012218
:101210005A65704700700240014B1878704700BF54
:101220000759022038B50446EFF31185402383F3B4
:101230001288BFF36F8F03060AD51249124840F295
:1012400053620AF0BFFF0F4840F253610AF0B1FF4A
:10125000FFF7D6F90D4A012303FA00F0136823EAD9
:101260000003136014F0080201BF04F00F04084BE0
:1012700004F5947443F8242085F31188BFF36F8F2D
:1012800038BD00BF241B020025FE01005C33022094
:10129000007002402DE9F04F044685B0EFF311874E
:1012A000402383F31288BFF36F8FFFF787F914F0A1
:1012B000800F414E05462BD12046FFF7A1F9D6F805
:1012C00000804FF0010909FA00F030EA08000BD065
:1012D0002046FFF7A7FF0323AB7587F31188BFF301
:1012E0006F8F05B0BDE8F08F28732046FFF788F9AF
:1012F00009FA00F028EA000030602046FFF780F984
:101300002E4A136809FA00F923EA09031360E2E799
:10131000230715D4802C2A4B41D004F00F0202F28F
:10132000DA325200C3F80028D3F80428D3F804189E
:10133000D2B242F002020A43C3F80428D3F80438B8
:10134000DFF87890D6F800B0D9F800A020466BEA14
:101350000A030193FFF754F94FF00108019B08FAC3
:1013600000F00342B9D02BEA000030602046FFF7BE
:1013700047F900232B73032308FA00F8AB758DF8A7
:101380000F30104B8DF80E4048EA0A000622C9F8CB
:1013900000001B688DF80C2003A898479DE740F2D9
:1013A000B472C3F80028D3F80428D3F80418D2B2D2
:1013B00042F00402BFE700BF583302205C33022032
:1013C000007002406033022038B50446094D4FF0EA
:1013D000FF324FF0FF33284605F0C8FD2046FFF7E7
:1013E00059FF284605F05EFD034B8022C3F8042117
:1013F00038BD00BF002A002000E100E02DE9F041E7
:101400003A4D2B7853B93A493A4840F2BA420AF079
:10141000D9FE40F2BA4136480AF0CBFE4FF0FF3316
:1014200035484FF0FF3205F0A1FD2B78022B08D094
:101430002F49304840F2FC420AF0C4FE40F2FC4121
:10144000E9E72E4B8022C3F884212720FDF7B0F96D
:10145000A0B12B4F2B4B3C681B68240C24041C436D
:101460004FF0010864BB284E40F2FF133B60272079
:10147000C6F80445FDF788F9C6F80043234A1378F7
:101480008BB1214B0021C3F808110121C3F80026BC
:10149000C3F804165960D3F808110029FBD00021C5
:1014A000C3F808111170184B0022C3F80025FFF78C
:1014B000C1F8114805F0F6FC01232B70BDE8F0815E
:1014C00094FAA4F6B6FA86F60F2E3046C6BFA6F1F9
:1014D0001000C0B240F08000030701D4FFF7DAFE2D
:1014E00008FA06F624EA0604BCE700BF0959022000
:1014F000241B020025FE0100002A002000E100E07C
:101500005C3302205833022000700240055902204B
:1015100010B504464FF0FF324FF0FF33114805F08D
:1015200025FD2046FFF7B6FE04F00F02012393408D
:101530000D4A14F0800F14BFD2F81015D2F814150C
:101540006FEA030315BF0B400B40C2F81035C2F819
:101550001435044805F0A6FC044B8022C3F804218E
:1015600010BD00BF002A00200070024000E100E032
:1015700070B50446FFF756FA68B904F00F0201256A
:1015800014F0800F144B05FA02F205D0D3F81015B1
:101590000A43C3F8102570BDD3F814150A43C3F8E5
:1015A0001425631E062BF6D8EFF31186402383F330
:1015B0001288BFF36F8F2046FFF734FE2046FFF7F7
:1015C0001FF8064A1368854023EA0503136086F373
:1015D0001188BFF36F8FDEE700700240583302209E
:1015E000020710B504460AD50B490C4840F20F62B9
:1015F0000AF0E8FD084840F20F610AF0DAFD030640
:1016000005D4FFF79FFD10B12046FFF70BFE044BFA
:10161000C3F8184510BD00BF241B020025FE0100C1
:101620000070024037B50C460A490B4A411A402364
:10163000009349110546234608480BF07EFD011E24
:1016400005DA2846234603B0BDE83040184703B00A
:1016500030BD00BF78330220A3D10100A4DF010018
:10166000C9B2012908B508D9084909487F220AF0FA
:10167000A9FD06487F210AF09CFD03690C2201FBAD
:101680000233986C00F0070008BD00BF7F1B02000A
:1016900025FE010070B5C9B2012903690AD91849AC
:1016A000184840F2C5120AF08DFD154840F2C511E8
:1016B0000AF07FFDEFF31185402484F31288BFF315
:1016C0006F8F0C2606FB0134A46C14F0C00408D004
:1016D000A24206D085F31188BFF36F8F4FF0FF3021
:1016E00070BD71430B4401229A6485F31188BFF3E6
:1016F0006F8F43680B445B6898470020F0E700BF9A
:101700007F1B020025FE010070B50D460649411AF7
:101710000446491105484022FFF7BCFF2B4601460D
:101720002046BDE87040184778330220A4DF01004E
:10173000002270B5012104461046FDF747F80F4816
:1017400003F06AFA0E4B984215D103F075FA266938
:101750000C4930460AF0A2FE00280BDB0125B564D7
:101760002469084904F120000AF098FE002801DBF2
:101770006565002070BD6FF00400FBE78D18010067
:101780000000AD0B18E801001FB500220123CDE9D0
:101790000223094ACDF800D06B46CDF804D00BF0F7
:1017A000F9FC002805DB4FF480420023684605F071
:1017B000DDFB05B05DF804FBAFD1010008B50020EA
:1017C00003F0CEFA05490648F9F738F9783004D124
:1017D000BDE808400248F9F7DBB808BDD033022065
:1017E0007833022010B507490748002401234C60D4
:1017F000CC608B60F9F748F82046BDE8104003F054
:1018000043BA00BFD03302207833022010B5EFF383
:101810001184402383F31288BFF36F8F074A136844
:1018200023F00201DB07116002D4012003F098FAD3
:1018300084F31188BFF36F8F10BD00BFE033022027
:1018400030B4104B0C2202FB003301460020D3E9D8
:1018500010521864EFF31180402484F31288BFF310
:101860006F8F9C6C04F0C00444F002049C6480F30D
:101870001188BFF36F8F1DB12B46034830BC18474A
:1018800030BC704778330220A4DF0100012808B57E
:1018900006D0032808D090B90E4B9B6C5B0717D17C
:1018A000BDE80840FFF7CCBF0B490C484FF4397234
:1018B0000AF088FC4FF4397107480AF07AFC0649AF
:1018C00006484FF43D720AF07DFC4FF43D71F3E79A
:1018D00008BD00BF783302207F1B020025FE0100F7
:1018E00010B4EFF31182402383F31288BFF36F8F9C
:1018F0001848016841F002040460C80708D482F364
:101900001188BFF36F8F01205DF8044B03F0BCB961
:101910004FF08041D1F80C04D1F80C14C907EED572
:10192000EFF3118083F31288BFF36F8F0A498B6C3A
:1019300003F0C00343F002038B6480F31188BFF30C
:101940006F8F82F31188BFF36F8F00205DF8044B17
:10195000FFF776BFE033022078330220024BC0B29B
:1019600003EB4010704700BF7833022038B52F4991
:10197000BFF35B8F0446012251E8003F41E800209D
:101980000028F9D1BFF35B8F9BB9294929484B60E7
:10199000CB608A60F8F778FF00280ADA26492748E2
:1019A0004FF426720AF00EFC4FF4267122480AF01A
:1019B00000FC0CB3631E012B2ED80BF079FFE0B9AD
:1019C0001F4B1B78CBB14FF080430222C3F8082392
:1019D00003464FF08041D1F81854D1F81824ED0394
:1019E000F9D502F00302022A01D0012CF3D168B12B
:1019F00083F31188BFF36F8F38BDEFF3118340225B
:101A000082F31288BFF36F8F0120E2E74FF080432B
:101A10000222C3F80423EFE70749084840F2AA224C
:101A20000AF0D0FB40F2AA21C0E700BF74330220C5
:101A300064330220983302207F1B020025FE010040
:101A4000B35A022010B5044C2046F8F789FA204614
:101A5000FDF7F8F9002010BD5D1A010073B5104EB6
:101A60008DF807000446032501220DF1070100202F
:101A700004F0DEFB20B101233370204602B070BDBC
:101A80003378002BF9D0013D08D00BF011FF00286E
:101A9000EAD10021422006F027FDE5E73570ECE7AA
:101AA0000A590220024883685B6A03B118477047ED
:101AB00004E001000146024883685B68184700BFE4
:101AC00004E0010008B507480BF04FFE38B10648A6
:101AD000FDF7B8F90448F8F743FA002008BD6FF0A5
:101AE0001200FBE704E00100D9D1010038B504463B
:101AF0000D460820FFF7DEFF3DB92020FFF7DAFF93
:101B0000BDE838400820FFF7D5BF0A480AF0E7FAD9
:101B10002544EDB2607804F8010BFFF7CBFFE3B288
:101B2000AB42F7D12020FFF7C5FFBDE8384002489F
:101B30000AF0D5BAE21B0200E61B02002DE9F74FBE
:101B40009C4F9D4ED7F80880D8F83C30BBB1384642
:101B50009847002813DDD8F8383083B138469847C5
:101B600000280CDDD8F82C304BB1384698470028B7
:101B700005DBE9D0D8F8103023B9FFF793FF03B0A5
:101B8000BDE8F08F01220DF1070138469847002883
:101B9000F3DB336893B3BFF35B8F884C2368BFF3E9
:101BA0005B8F13F0020F234600F0D6809DF807509C
:101BB000D6F80090BFF35B8F53E8002F22F00401AA
:101BC00043E800100028F7D1BFF35B8F50072AD5F8
:101BD0007B4BDFF8F8A15B5D13F0040F18D10123F4
:101BE000CAF80030482D5CD8422D5CD9433D052D04
:101BF00059D8DFE805F0766558945885714B186818
:101C00000022002305F0D8F830600028C3D1B6E7E1
:101C1000082120460BF0D1FA6B4B303D0022CAF868
:101C200000501A6090E7BFF35B8F2368BFF35B8FB0
:101C30001907D7D5624B5B5D5A0710D5BFF35B8F91
:101C40002368BFF35B8F13F0100F14BF5E4A5F4A27
:101C500013680A2101FB0353303B136074E73B2DEB
:101C600018D0BFF35B8F54E8003F23F0080344E82B
:101C70000032002AF7D1BFF35B8FBFF35B8F54E8CC
:101C8000003F23F0100344E80032002AF7D1BFF3ED
:101C90005B8FA7E7102120460BF08FFAC306E0D434
:101CA00052E77E2D44D0BFF35B8F54E8003F23F012
:101CB000020344E80032002AF7D1BFF35B8F43E709
:101CC0004348424A037811688B42ECD3414D2A784D
:101CD0005B1A52FA81F203703F482A700AF0FFF94A
:101CE000E1E73C48394B027819688A42DBD3CBB232
:101CF000D21A0270364A1078034413703748EDE761
:101D0000334D29780029CED033480AF0E8F9314A1A
:101D1000137829780B44137000232B70C3E72D4DE3
:101D200029780029BFD02D480AF0D9F9284AEFE7D1
:101D3000284D2B78002BB6D0284801210AF0CFF986
:101D4000234A2978107809F105090139C9B24844B4
:101D50002970FFF7CBFEA6E7BFF35B8F54E8003F87
:101D600023F0010244E800210029F7D1BFF35B8F83
:101D700013F0010F9DF807500BD05B2D7FF4E4AEFC
:101D8000022120460BF019FA042120460BF015FA27
:101D9000DAE60B4B5B5D13F0970F6CD10D2D1FD85E
:101DA000072D2ED9083D052D2BD8DFE805F01D5352
:101DB000342A2A3804E00100E4330220F033022000
:101DC00004240200FC330220E8330220EC3302201A
:101DD0000D5902200C590220EA1B0200F01B0200E0
:101DE0001B2D13D07F2D0CD13B4A13784BB1013BF7
:101DF000DBB213703068394A053311781844FFF7A5
:101E000075FE374B9DF807201A709DE6012120468C
:101E10000BF0D3F9F5E7324B1B780D2BF1D0DFF83F
:101E2000B8902E4D99F8001033682A780B4413446B
:101E300000245C710D20FFF73DFE0A20FFF73AFEFB
:101E4000284B3168186889F800402C700BF0F7FCBB
:101E50003460D6E7244B1B68002BD2D01F4A12787F
:101E6000002ACED11C4C3068217805309847237861
:101E700018442070C5E7194A174B147893F800B03E
:101E800004EB0B027E2ABCDCD6F800A00BF10102A9
:101E900028461A70FFF70EFE0AEB0B030CB95D71B2
:101EA000AFE793F8059011485D710AF018F90BF14E
:101EB000060B013CDA44E4B2013C4846E4B2FFF7C9
:101EC000F9FD4B46FF2C9AF800900AF8013BF3D13C
:101ED00007480AF004F994E70D5902200C59022032
:101EE0000B590220F8330220F4330220E21B0200D7
:101EF000E61B0200164B73B51860164B1960164BA3
:101F00001A60FFF7CFFD154DAC68A3690BB12846E9
:101F10009847236C1BB112491048002298470F4E76
:101F2000E36A23B9AB681B6A73B902B070BD30466F
:101F300098470028F6DD2369002BF1D001220DF12E
:101F4000070130469847EBE704489847EDE700BFA4
:101F5000FC330220F8330220F433022004E00100B5
:101F60003D1B0100024B0B6001231360704700BF53
:101F700000340220004870473CE8010038B50546AF
:101F800008200C46F9F764FB48B1094BC461C0E96D
:101F9000053504230374002343748374C374054913
:101FA00000234FF401520AF0B1FD6FF0150038BD67
:101FB000F61B020044E4010010B501221146064858
:101FC000064C0BF047FC0BF0BAFA20600BF0B3FAAA
:101FD0006060002010BD00BF0834022000340220E1
:101FE0004FF08042D2F81015D2F8103501F01E01E2
:101FF00023F01F030B4343F00103C2F81035024BDB
:1020000000221A70704700BF0E5902204FF0805313
:10201000D3F83031082B20D14FF08042D2F8101580
:10202000CB071AD5D2F8103501F01E0123F01F039B
:102030000B43C2F81035D2F808315BB1D2F8103535
:1020400023F01F030B4343F00103C2F810356FF078
:102050008B007047024B01221A700020704700BFAE
:102060000E5902202DE9F0410E4615460BF063FA99
:102070002946074630460BF0FBF8B04604460028D8
:1020800044D0B6FBF7F307FB136323B9B5FBF7F4B2
:1020900007FB1454B4B10820F9F7DAFA48B1234B1E
:1020A000C561C0E9053604230374002343748374B7
:1020B000C3741F4900234FF401520AF027FD6FF04B
:1020C00015041DE0AF421BD84FF0FF324FF0FF3335
:1020D0001848194F04F04AFF0BF02DFA0646FFF797
:1020E00095FF044678B9404603F016FB3B780BB1E8
:1020F000FFF776FFAD1BB044F1D10E4804F0D2FEDD
:102100002046BDE8F0816FF08B04F6E70820F9F770
:102110009FFA0028CDD0094BC561C0E905360423DC
:10212000037444748474C474C3E700BF131C0200B6
:1021300044E40100083402200E590220F61B02007C
:102140002DE9F8430E463046194617461C460BF05B
:102150008FF80546B8B90820F9F77AFA40B12A4B4A
:10216000C461C0E905360423037445748574C574DD
:10217000264900234FF401520AF0C8FC6FF0150401
:102180002046BDE8F88346EA040515F003050FD0A4
:102190000820F9F75DFA0028EAD01D4BC461C0E9B8
:1021A000053604230374002343748374C374DFE788
:1021B000002CE5D01748DFF864904FF0FF324FF065
:1021C000FF3304F0D3FE24F00304A54205EB060818
:1021D00009D1114AD2F80034DB07FBD500240D48A1
:1021E00004F060FECCE7FFF711FF50B97959404683
:1021F00003F0C6FA99F800300BB1FFF7F1FE043591
:10220000E3E76FF08B04EAE7F61B020044E4010009
:10221000321C02000834022000E001400E59022066
:1022200010B5036941B91C491C483F2209F0CAFF97
:102230003F21194809F0BDFF486830B916491748D1
:10224000402209F0BFFF4021F3E75868F8B1884207
:1022500019D19C6808685860A14200D1986000209C
:1022600008602AB15A680A609A68596002B9996090
:10227000002010E0814206D1086820609868814201
:10228000EDD19C60EBE7044600680028F2D1002AFB
:10229000E8D16FF0150010BD741C020025FE01008E
:1022A00008B503685909024613D0012906D103F085
:1022B0001F034FF6FF71D940C80712D40A490B48D3
:1022C00040F2C73209F07EFF074840F2C73109F0FB
:1022D00070FF4FF0FF31D940C907EFD54FF0A04054
:1022E00000E00348136008BDAD1C020025FE01009C
:1022F00000030050F0B54068057B01F01F0444EA7C
:102300004514056987B0002D77D0B2F5001F00F1A4
:10231000100506D1214628460BF0F1F8002007B041
:10232000F0BD01AE0027B2F5800F0197776034D180
:10233000B3F1007F14BF052304238DF8043000237C
:10234000CDE9046303938368CB40D9073AD4B2F153
:10235000A07F37D168460094FFF7A2FF009B03F5EA
:10236000E07350F82330DB072CD46A462146284618
:1023700002F0F6FF244B98421AD0CDF808D003AAF9
:102380002146284602F0B6FE204B984238D1012261
:102390002146284603F05EF8C0E7B3F1C06F05D0D0
:1023A000B3F1007F14BF01230223C6E70323C4E770
:1023B0006946284603F048F8144B9842DDD06FF088
:1023C0000B00ACE76A462146284602F0C9FF0F4BD6
:1023D00098420646D3D19DF80010284603F02EF807
:1023E000B042CCD00A490B484FF4E37209F0EAFE40
:1023F00007484FF4E37109F0DCFE6FF085008EE7CB
:102400006FF015008BE700BF0400AD0B0000AD0BB3
:10241000DD1C020025FE01002DE9F043466840F274
:102420000635337BD00687B001F01F0702EA0505A9
:1024300047EA431754BFC2F340130323B5F5837F24
:1024400014468DF8033045D00DD8062D16D005D88A
:10245000A5B1022D40D06FF0150038E0B5F5807FB2
:10246000F9D101250AE040F20222954236D0B5F5B5
:10247000407F35D0B5F5007FEDD102250123220341
:1024800003FA01F12ED57368C3F8081533697BBBD5
:1024900003A80397FFF704FF039B00EB830084F47A
:1024A0008033C3F30043C4F34044D0F8002744EA28
:1024B00043049DF8033022F4E16244EA830422F0ED
:1024C000070244EA05231343C0F80037002007B091
:1024D000BDE8F0830725D1E70425CFE70525CDE743
:1024E0000325CBE7630344BF7368C3F80C15CDE73E
:1024F00010360DF102023946304602F031FF14F475
:10250000403F804616D1394630460AF0F6FF244B4C
:102510009845DBD19DF80210304602F08FFF404510
:10252000D4D020492048E02209F04CFE1D48E0218B
:1025300009F03FFE01AB4FF0000903AA39463046CF
:10254000CDE90439CDE90199CDF80C9002F0D2FD26
:10255000134B9842BAD114F4003315D09DF80330D0
:102560008DF80E3084F48034C4F300444B4603AA43
:10257000394630468DF80C508DF80D4002F06EFE55
:10258000074B9842A2D1C2E7CDE9043303AA0DF16B
:10259000030339463046039302F0ACFDF0E700BF79
:1025A0000000AD0BDD1C020025FE0100420970B5E4
:1025B000034602D0012A1AD070BD124E326951680A
:1025C0000029F9D003F01F0301250C689D40002964
:1025D000F2D08A682A400ED04B6853B90A490B489A
:1025E000642209F0EFFD0848642109F0E2FD084E7D
:1025F000E4E7304698471CB1236821461C46E6E7CD
:102600002346FAE7E4DF0100741C020025FE010006
:10261000C4DF010038B545682B69B3B110352846D1
:1026200002F002FF044680B90146284602F0C2FECD
:10263000084B98420BD108492246284602F08AFEF0
:10264000224605210620FCF7C1F8002038BD6FF0B6
:102650000400FBE70000AD0BAD25010008B50368E1
:102660005909024613D0012906D103F01F034FF682
:10267000FF71D940C80712D40A490B4840F2C7324B
:1026800009F0A0FD074840F2C73109F092FD4FF074
:10269000FF31D940C907EFD54FF0A04000E0034813
:1026A000136008BDAD1C020025FE010000030050B0
:1026B0002DE9F04FDFF8DC80DFF8DC9085B01546BF
:1026C000044600EB810640F2FF17A64203D100202A
:1026D00005B0BDE8F08F23685904C3F3C322C3F3E8
:1026E000080B51D41B0E163B18F802A0BB4508BFBF
:1026F0004FF0FF3B032B4AD8DFE803F00235383BAD
:10270000C5F860B56388BBF1FF3F03F0010328D033
:10271000CDF80CB003A87BBBFFF7A0FF039A012301
:102720009340C0F80C352268019203A8CDF80CB094
:10273000FFF794FF039B019A00EB830082F40043B0
:10274000C3F3C033D0F8001743F00203C2F34122B1
:1027500043EA820301EA090143EA0A230B43C0F872
:1027600000370434B1E7C5F864B5CBE7C5F868B500
:10277000C8E7C5F86CB5C5E7FFF770FF039A0123FA
:102780009340C0F80835CEE76FF01500A0E76FF072
:1027900085009DE7221D0200F0F8FCFF08B50368E4
:1027A0005909024613D0012906D103F01F034FF641
:1027B000FF71D940C80712D40A490B4840F2C7320A
:1027C00009F000FD074840F2C73109F0F2FC4FF074
:1027D000FF31D940C907EFD54FF0A04000E00348D2
:1027E000136008BDAD1C020025FE0100000300506F
:1027F0002DE9F341BDF820C0466804690329074666
:102800000D4690460CF0010C10D90820F8F720FF77
:1028100040B15C4BC0E905350323037400234374C6
:102820008374C37400234FF4C25221E0B27F012AA3
:102830004FF0010104BF5B084FEA5808A940002B84
:1028400076D0984577D9226890452AD02079884358
:1028500016D00620F8F7FCFE38B14B4B436102233B
:102860000374002343748374C37400234FF48252AF
:1028700046490AF04BF96FF0150002B0BDE8F0814F
:102880004246B2F5004F45D2C4F800806071D6F8D8
:1028900000E096F81E80CEF80C05CEF80485CEF840
:1028A0000825627923FA02F292B24FF0010E78689D
:1028B0008CF00108806A42EAC83220F815205FFADD
:1028C00081F8BEF1000F45D1326805F5AC7552F8BC
:1028D0002520002A0FDBBCF1000F4FD0B3FA83F3A1
:1028E0005B096BBB01A80192FFF758FF019A012316
:1028F0009340C0F80C35217921EA0801217171B3A8
:10290000A3799BBB1023012206F12801304603F076
:10291000DFF929E0013008284FEA5202B1D1F8F777
:1029200097FE00283FF47EAF194BC0E9053873E7E6
:102930009E461A46BBE74FF0000E47F6FF72B6E719
:1029400001A80192FFF72AFF019A01239340C0F8E2
:102950000835D0E7237948EA03032371D0E7786884
:1029600003F018FA0123A371002086E70023A37166
:10297000304603F045FA0028FAD0C3E7003B18BF01
:102980000123AEE72A1D02003F1D02009CE4010066
:10299000541D02002DE9F041044682B0002200AF30
:1029A00001211C20FBF712FF60682369304A00F107
:1029B000080103F067F92F4B984219D023686C4641
:1029C00088B06A462C49C2E905134FF4007393831B
:1029D0002A4B42F8103F2A4800234FF4E251F8F7FF
:1029E000DDFF6FF00F00A5460837BD46BDE8F0815A
:1029F0006568AE6B3A1D002130460AF0A1FC002844
:102A000005DB7B68326819791868FFF751FE4FF0D3
:102A1000000846462B6806F5AC7253F82230002BAE
:102A200010DB7B60381DFFF7B9FE7A68D0F80435FB
:102A3000D34013F001031CBF0123B34048EA030352
:102A40005FFA83F80136042EE4D100230120626886
:102A5000916A00FA03F212EA080F0CBF0122002269
:102A6000D20321F813200133042BF0D10020BBE75F
:102A700067D301000000AD0B7E1D020003000001C2
:102A80009CE4010070B40E49D1E90034D01AC31897
:102A900044F1000422F07F46C1E90034A6F500139A
:102AA000B3F5400F09D2074B1B681A0A1B069C1985
:102AB000054B42F10005C3E9004570BC06F062B960
:102AC00098D0012040340220A0D001200D4B18687E
:102AD000010A0006BFF35F8F0B4BD3F804351818BB
:102AE00041F10001B3F5801F0AD2084BD3E900235E
:102AF000904271EB030303D210F1807041F10001A9
:102B0000704700BF4034022000100140A0D00120D7
:102B10002DE9F7432B4CD4F8043399070BD5D4F89F
:102B2000043143B1284A0023C4F80431D4F80431F5
:102B3000136801331360D4F80433DA0323D5BFF3E9
:102B40005B8F224B53E8002F22F0010143E8001075
:102B50000028F7D1BFF35B8FD30702D4D4F84031FC
:102B60008BB10025C4F84051D4F84031FFF7AEFFD7
:102B7000EFF3108272B6164BD3E90267B042B94147
:102B800004D282F3108803B0BDE8F0834FF0FF3821
:102B90004FF0FF39C3E90289D3E900101D604FF4FB
:102BA0008033C4F84833C4F84051D4F8403182F33C
:102BB00010880029E7D0009032463B4628468847D7
:102BC000E1E700BF00100140403402203834022009
:102BD00088D001202DE9F84F4B4DBFF35B8F06469F
:102BE0000F4655E8008F28F0010345E80032002A1F
:102BF000F7D1BFF35B8F454C4FF48039C4F808938D
:102C0000BFF35F8FBFF36F8FFFF760FFB04271EBD1
